:0800000C32322E332E312E3763
:1000000AF9141AFC40351BF63B474B2A052A3008DF
:1000000A4833370C1A1216141A161B1C175E524460
:1000000A0F645761461E3C3F21614E3D4026303306
:1000000A3833383333373B3633393D433E433E3E4C
:1000000A4246413E43484E494E49494D514C495456
:1000000A545754595454585C575477597B4C8271FD
:1000000A745A74785D9D7B60A99D8F5A907F82682F
:0500000A92966B90903E
:020000040800F2
:40800000E0C7002085C80E088DC80E086918170891C80E0893C80E0895C80E08000000000000000000000000000000002183000899C80E0800000000D98300083D84000868
:408040009FC80E089FC80E089FC80E089FC80E089FC80E089FC80E08C5A51608CFA51608D9A51608E3A51608EDA516089FC80E084BBD16089FC80E0855BD16089FC80E0839
:408080009FC80E089FC80E086DAB0D085F93160869931608739316089FC80E08F7A516089FC80E089FC80E089FC80E089FC80E089FC80E089FC80E089FC80E089FC80E082C
:4080C0009FC80E0847420E0851420E089FC80E089FC80E089FC80E089FC80E085FBD16081DA616089FC80E089FC80E089FC80E089FC80E089FC80E089FC80E089FC80E0841
:408100009FC80E089FC80E089FC80E089FC80E089FC80E089FC80E0851A61608E7A8160849AB0D0861AB0D0855AB0D089FC80E089FC80E089FC80E089FC80E087D9316082E
:4081400087931608919316089FC80E089FC80E089FC80E089FC80E089FC80E089FC80E089FC80E089FC80E089FC80E089FC80E089FC80E089FC80E089FC80E08000000002C
:408180009FC80E089FC80E089FC80E089FC80E089FC80E089FC80E089FC80E089FC80E0800000000000000009FC80E0800F002F800F06FF80AA090E8000C82448344AAF1C3
:4081C0000107DA4501D100F064F8AFF2090EBAE80F0013F0010F18BFFB1A43F0010318470C3010004C30100010F8013B0A4413F0030408BF10F8014B1D1108BF10F8015B54
:40820000641E05D010F8016B641E01F8016BF9D1002D15D010F8014B03F00C030C2BA1EB04040ABF10F8013BA4EB8314A4EB032405F1010314F8016B5B1E01F8016BF9D588
:40824000914238BF10F8013BD1D370470023002400250026103A28BF78C1FBD8520728BF30C148BF0B6070471FB5E7F008FC9DE8030069F1DCF969F128F869F1ABFA040089
:4082800000200021E6F06EF8401C6060E4F0D4FD1FBDE4F01EFF1146FFF7E6FF0FB437F1C5FE0FBC22F006FEE4F0BAFC03B437F1B8FE03BC52F17DF880F309887047EFF3BF
:4082C00009807047684680F3098804480078C00714BF0220032080F31488704738A01008DFF818C0EFF305831B0618BF6047EFF31483DB0708BF604700DF7047FB251708DD
:40830000DFF818C0EFF305831B0618BF6047EFF31483DB0708BF604700DF7047C5261708EFF30980816911F8021CE1BB90E80F1010B5E047BDE81040EFF3098C8CE807009A
:40834000214B93E80600914208BF704741B91EF0100F16D11D49086820F00100086010E01EF0100F06BF2CED108A0120002081F825002CE9F00FC1F828C00CB46AF1C6FB5D
:408380000CBC1A60D2F828C0BCE8F00F92F8250000280EBF6FF0020E6FF0120EBCEC108A8CF30988704710B5094A1268914209D8084C54F8214090E80F10A047EFF3098C4F
:4083C0008CE80F0010BD00001434002034EF00E0501817085018170810B5E5F061FDBDE81040154B93E80600914208BF7047EFF3098C1EF0100F06BF2CED108A0120002038
:4084000081F825002CE9F00FC1F828C00CB46AF17DFB0CBC1A60D2F828C0BCE8F00F92F8250000280EBF6FF0020E6FF0120EBCEC108A8CF3098870471434002010B5E5F022
:40844000FFFDCCE710B56AF1D7F8E5F0F9FDC6E710B50446204637F19CFE002084F8500084F851006065A0659FEDFE0A84ED170A20666066206881682046884710BD2DE931
:40848000F04104460D4616461F463946204637F1FDFD0446F44820602430E0601030206184F852602046FFF7D3FF1DB1012084F8200002E0022084F820002046BDE8F081C8
:4084C00010B50446204637F104FE0446204610BD70B504462046FFF7F3FF054669F122FB70BD10B50446103C2046FFF7F1FF10BD10B504460C3C2046FFF7EAFF10BD10B512
:408500000446103C2046FFF7DBFF10BD10B504460C3C2046FFF7D4FF10BD70B50546012406E0D24B00222146284664F197FB641C0B2CF6D30C2406E0CC4B00222146284635
:4085400064F18CFB641C0D2CF6D370BD2DE9F0412DED028B0446B0EE408A0F4615460026204637F1DCFEB4EEC80AF1EE10FA06D2204637F1D4FEB0EE408A022638E02046EF
:4085800037F1CDFEB1EE400AB4EEC80AF1EE10FA08DD204637F1C3FEB1EE400AB0EE408A022625E027B3204637F1F0FEB1EE400AB4EEC80AF1EE10FA1AD2204637F1E6FED6
:4085C000B4EEC80AF1EE10FA12DDB5EEC08AF1EE10FA07D2204637F1D9FEB1EE400AB0EE408A04E0204637F1D1FEB0EE408A032694ED0D0AB4EE480AF1EE10FA07D084ED3B
:408600000D8A2B4632460221204664F127FB3046BDEC028BBDE8F0812DE9F0412DED028B04460D46E06ADEF001F906464FF4967020639FED8C0AB0EE408A00270B2D0BD27D
:40864000DFE805F0060C0B4146474C5B738D92009FED870AB0EE408A8CE000BFB6F57A7F09D2204637F192FEF1EE040A30EE200AB0EE408A1FE041F27070864209D2204615
:4086800037F184FEF3EE040A30EE200AB0EE408A11E043F69820864209D2204637F176FEF3EE0E0A30EE200AB0EE408A03E09FED700AB0EE408A022D03D1B1EE480AB0EE5E
:4086C000408A012756E09FED670AB0EE408A51E000BF9FED680AB0EE408A4BE0204637F189FD012804D19FED630AB0EE408A03E09FED5C0AB0EE408A3CE0204637F146FECE
:40870000F3EE0E0AB4EEE00AF1EE10FA05DD204637F13CFEB0EE408A03E0B3EE0E0AB0EE408A4FF4FA60206324E0204637F12EFEF2EE040AB4EEE00AF1EE10FA07DD20462A
:4087400037F124FEB1EE400AB0EE408A03E0BAEE040AB0EE408A4FF4FA6020630AE09FED410AB0EE408A05E0204637F19CFDB0EE408A00BF00BF20683C4A3946B0EE480AA5
:40878000036920469847BDEC028BBDE8F08170B52DED048B84B004469FED320AB0EE408A9FED300AF0EE409A9FED2E0AF0EE408A9FED2C0AB0EE409A002003900290019046
:4087C0002A4D4FF4FA70206303A9204637F14DFD002871D002A9039800F07BFB00286DD003980068C16A039888470646029843F196F986427CD203980068016A03988847A5
:40880000039800F060FBB0EE408A204637F1F5FD20EE080AB0EE408A02980068416902988847B0EE409AB5EEC09AF1EE10FA11D003980068016B03988847C0EE090AF0EE16
:40884000608A03980068016903988847C0EE090AF0EE609A01A9029843F164F968B301980AE0000000000000C4A01708BB1817080000C8420000C8C200F0A9FBC8BBB0EE6D
:40888000080AF4EEC08AF1EE10FA18D2B5EEC08AF1EE10FA13DDB2EE040AB4EEC08AF1EE10FA0CD29FEDF80A28EE000AB0EE408A4FF47A70206346E075E047E065E0F5EEF0
:4088C000C08AF1EE10FA1CDDB2EE040AF4EEC08AF1EE10FA15D2B1EE040AF4EEC09AF1EE10FA0ED2B5EEC08AF1EE10FA09D201E046E029E09FEDE40A28EE000AB0EE408A2D
:4089000021E0B3EE040AF4EEC09AF1EE10FA1AD2F5EEC08AF1EE10FA15DDB5EEC08AF1EE10FA10D29FEDD90A28EE000AB0EE408A9FEDD70AB4EEC08AF1EE10FA03D29FED1C
:40894000D40AB0EE408A00E000BF00BFB5EEC08AF1EE10FA07DD204637F118FD30EE080AB0EE408A2CE0B5EEC08AF1EE10FA27D2204637F10BFD38EE400AB0EE408A1FE016
:408980001FED480AB0EE408A1AE094F82000012804D11FED480AB0EE408A11E01FED4F0AB0EE408A0CE094F82000012804D11FED4F0AB0EE408A03E01FED560AB0EE408AAF
:4089C00020682A460021B0EE480A03692046984704B0BDEC048B70BD0146486D704770B52DED028B0446AB4D4FF4FA70206394F8230094F8241088420AD094F8240084F874
:408A00002300A54800688047E062012084F827001FED6C8AA06D002810D9A06DDDF006FF00EE100AB8EE400AD4ED0D0A20EE200A5FED710A80EE201AB0EE418AA06D0028DD
:408A400062D994F8270000285ED194ED170A30EE080A84ED170AD4ED170A40F2DC5000EE100AB8EE400AF4EEC00AF1EE10FA06DD00EE100AB8EE400A84ED170A0AE094EDA8
:408A8000170AB5EEC00AF1EE10FA03D21FED8B0A84ED170A94F8520090B394F8230006282FD194ED0D0AB5EEC00AF1EE10FA03D100202066606627E094ED0D0AB5EEC00AFF
:408AC000F1EE10FA0BD200202066B1EE480ABCEEC00A10EE100A616E0844606614E094ED0D0AB5EEC00AF1EE10FA0DDD00206066BCEEC80A10EE100A216E0844206603E022
:408B0000FFE7002020666066634800688047A06594F823000D280CD2DFE800F0070C11161B20257C7D6D72777E0006212046FFF773FD76E001212046FFF76EFD71E002217E
:408B40002046FFF769FD6CE000212046FFF764FD67E004212046FFF75FFD62E003212046FFF75AFD5DE02046FFF736FFC8B394ED170AB5EEC00AF1EE10FA03D194F8270004
:408B800001280BD094F8500058B32046FFF724FF06463146E06ADDF059FE10BB012084F8500000212046FFF737FD94F82700012804D12046FFF710FF20631BE02046FFF7BB
:408BC0000BFF0646E06ADDF031FE864212D92046FFF702FF0646E06ADDF028FE301A206308E0FFE7002084F8510084F850002046FFF7CDFD15E005212046FFF70DFD10E055
:408C000008212046FFF708FD0BE007212046FFF703FD06E000BF00BF06212046FFF7FCFC00BF00BF204637F15EFC002084F8270094F82300062833D194ED190AB8EE400ABE
:408C4000DFED160AB4EEE00AF1EE10FA01DB012000E0002001462A46204637F12BFC94ED180AB8EE400ADFED0D0AB4EEE00AF1EE10FA01DB012000E0002001462A46204625
:408C800037F1F2FB31E000009A99193FCDCC4C3F000020C2BB18170818A010080000484494ED170AB5EEC00AF1EE10FA01DB012000E0002001462A46204637F1FBFBD4EDBE
:408CC000170A40F2DC5000EE100AB8EE400AF4EEC00AF1EE10FA01DB012000E0002001462A46204637F1C0FB00BF00BFBDEC028B70BD10B5044606212046FFF78DFC204609
:408D000037F1F1FB10BD2DE9F04104460D4616460027606DA84206D0656533463A460C21204663F19BFF3846BDE8F08170B52DED028B0446B0EE408A0026A06850B1B0EE3B
:408D4000C80AF0EE408AA5682868016B28468847064600BFE06850B1B0EEC80AF0EE408AE5682868016B28468847064600BF3046BDEC028B70BD70B52DED028B0446B0EEA9
:408D8000408A0025A06830B1A0680268B0EE480A916B88470546E06830B1E0680268B0EE480A916B884705462846BDEC028B70BD2DE9F0412DED028B04460D4616461F4665
:408DC0009DED088A2046DDF049FC04461C4820606760A560E660B8EE480A2046FFF7CBFF9FED180A2046FFF7A1FF2046BDEC028BBDE8F08110B50446114820609FED110A96
:408E00002046FFF793FF00206060A060E0602046DDF027FC0446204610BD70B504462046FFF7E8FF054668F17DFE70BD0146002070470146002070470246002070470000F8
:408E400078A717080000000070B504460D461646204663F15BFE044604F10C0063F138FFA0F10C041F4820604030E06026619FED1E0A84ED050A2576204670BD10B504467D
:408E800004F10C0063F12EFFA0F10C04204663F143FE0446204610BD70B504462046FFF7EDFF054668F13EFE70BD10B504460C3C2046FFF7F1FF10BD10B504460C3C204626
:408EC000FFF7DCFF10BD90ED050A70470146087E704702460020136913B1012013690B6070470000FC9E1708000000000021017141718160C160704700B502462448106016
:408F00001046FFF7F3FF104600BD00B502460B461F4810601046FFF7E9FF5371104600BD704770B504462046FFF7FAFF054668F1F9FD70BD01464879704710B503460A4651
:408F400000241846FFF7F6FF904200D05A71204610BD0146087970470246002013798B4200D0117170470146886870470246002093688B4200D0916070470146C8687047D7
:408F800002460020D3688B4200D0D16070470000E0AE170870B504460D46204663F198FE04460C4820602571204670BD10B50446204663F197FE0446204610BD70B5044639
:408FC0002046FFF7F3FF054668F1ACFD70BD014608797047D4A81008064901607047704770B504462046FFF7FAFF054668F19AFD70BD0000209D1708FFFFFFFFFFFFFFFF78
:409000006BF17AB96BF178B810B50446204639F1AAF9C820E03444F8780C0C20207400206074A0740220E07400206061A061E06120626062A062A085E08520866086A08634
:40904000E08620876087A087E08784F8400084F8410084F8420084F8430084F8440084F8450084F8460084F84700012084F84800002084F8490004F8050CE03C10BDF8B505
:4090800004460F4615461E462B46032239462046009639F1BDF80446FE48206000F58070E060103020610020C4F8EC002046FFF7ABFF23462A46F849204663F15AFD20460D
:4090C000F8BD0246002000230B60D2F8EC301BB10120D2F8EC300B6070472DE9F8430446894615461E46089FB84669464046FFF7E8FF28B3012C06D0032C0BD0042C10D012
:40910000052C1CD114E033462A469B21404663F1A5FD14E033462A469C21404663F19EFD0DE033462A469D21404663F197FD06E033462A469E21404663F190FD00BF00BF78
:40914000BDE8F88370B504460D46D4F8EC0028B1AFF27901D4F8EC0063F154FDC4F8EC50D4F8EC0038B123460022AFF29101D4F8EC0063F1FEFC00231A469A21204663F1AF
:409180006DFD70BD10B50446C248206000F58070E06010302061D4F8EC0020B10021D4F8EC0020F0BAF800212046FFF7CBFF204639F16AF80446204610BD70B504462046EA
:4091C000FFF7E0FF054668F1ADFC70BD10B50446103C2046FFF7F1FF10BD10B504460C3C2046FFF7EAFF10BD10B50446103C2046FFF7C8FF10BD10B504460C3C2046FFF745
:40920000C1FF10BD70B50546012406E0A34B00222146284663F122FD641C7D2CF6D37E2406E09E4B00222146284663F117FD641C9F2CF6D370BD70B504460D461646974BCB
:4092400000224FF6FF71204663F108FD70BD70B504460D461646914B00224FF6FF71204663F1FCFC70BD034600201060704701460020704702460020704710B5044600207F
:40928000186010BD10B504460020186010BD02460020704730B50546039C0020206030BD10B504460020186010BD10B504460020186010BD01460020704702460020704755
:4092C00010B50346002019B1022901D00720002193F8F1408C4201D083F8F11010BD2DE9F04104460D4616460027D4F80001A84207D0C4F8005133463A468821204663F130
:40930000ADFC3846BDE8F0810146D1F8000170472DE9F04104460D4616460027E06CA8420CD0E56433463A465521204663F196FC33463A465721204663F190FC3846BDE8D1
:40934000F081014691F8F00070472DE9F04F2DED028B85B0044600200490E06EDDF066FA80460026002500272068D0F8C410204688470390204639F1D7F908EE100A0020A7
:409380000290019081468246454800688047E06604A92046FFF795FE20B104981FF0F0FF042801D0012000E00020824694F82901012810D1BAF1000F0FD1204639F1F1F839
:4093C00028B1A16901F5D27001F0CFFC28B9002084F8290101E084F829A1A06970B1A06905F06EFD06462046FFF7ABFF8346A16901F13000594618F0DCFF05462046FFF7C5
:40940000A0FF834601AA5946A06903F067FB08B3019839F134F8142818D2DFE800F00A17171714100F0E130D0B121717171717170C1100BF00BF00BF00BF00BF00BF00BFE8
:4094400000BF00BF00BF4FF0000902E04FF0010900BF00BF2A464146204639F1AFFD002E2ED9002D2CD9B8EE481A00EE106AB8EE400AC1EE000A00EE105AB8EE400A9FED37
:40948000091AC1EE001A20EEA10ADFED070A20EE200A0BE000A31708CD311408FF18170818A010088096184B00007A44BCEEC00A10EE10BAFC4A59462046FFF729FF04E065
:4094C000F94A00212046FFF723FF204639F101FE204638F1C9FD012825D100EE105AB8EE400A9FEDF21AC0EE010A00EE106AB8EE400A1FED131AC0EE011A60EEA18A206893
:40950000D0F8C4102046884700EE100AB8EE400A5FED1B0A80EE201A28EE810ABCEEC00A10EE107A13E02046FFF7EEFE074694F8C900012806D1474501D2002707E0A7EBD0
:40954000080704E094F8CA00012800D14744D64A39462046FFF7C3FE204639F122F800B3D34800688047E0B9A06905F02FFDC0B9BFB1B9F1010F14D194F8290188B9022056
:409580000290204638F170FD28B9C74A0121204639F1B2F888E0C44A0D21204639F1ACF882E000200290204638F1FBFF28B9BE4A0021204639F1A0F876E0A16901F5D27090
:4095C00001F0D3FB022803D094F82901012805D1B54A0921204639F18FF865E0B44800688047012805D1B04A1221204639F184F85AE094F8D30050B1A06905F0E7FC02286D
:4096000005D1A94A0721204639F176F84CE094F8D30050B1A06905F0D9FC012805D1A24A0621204639F168F83EE0204638F11CFD01280BD12068D0F8C4102046884728B9D5
:40964000994A0B21204639F157F82DE02DB9964A1421204639F150F826E0204638F104FD70B9B9F1000F05D08F4A0121204639F143F819E08C4A0921204639F13DF813E058
:40968000B9F1010F0BD12068D0F8C4102046884728B9854A0B21204639F12EF804E0824A0921204639F128F87F4A20460299FFF707FE2068016D204688474FF0000B2046FF
:4096C00039F1B0F928B394F8DC00012821D1204639F1C1F900EE100AB8EE400AF0EE408A94ED130AB8EE400AB0EE401A94ED100AB8EE400AF0EE400AB0EE680A39F1F6FBEB
:4097000038B9D4F840B0684A0121204639F175F906E0D4F84CB0644A0021204639F16DF9C4F844B0204639F12BFE002005B0BDEC028BBDE8F08FF8B504460125204638F1F3
:4097400091FE0C2809DA2046FFF7FBFD06466A463146A06903F0C2F900B900252846F8BD014691F8F200704770B5044600252046FFF7F6FF022805D1204638F175FC01283D
:4097800000D10125284670BDF8B50446002500260020009094F82901012801D101262DE0204638F16CFE09280AD00A2807D00B2808D194F8DE00022800D101261DE000BFDF
:4097C00001261AE02046FFF7BCFD07466A463946A06903F083F978B1204638F1E2FE58B1009838F138FF18B9009838F1DAFE08B9012000E00020064600BF00BF94F8CF0035
:40980000B04207D084F8CF60274B2A461921204663F124FA2846F8BD014691F8240170472DE9F04104460D461646002794F82401A84207D084F8245133463A467E21204629
:4098400063F10CFA3846BDE8F0812DE9F04104460D461646002794F8F000A84207D084F8F05033463A467F21204663F1F7F93846BDE8F081014691F9200170472DE9F041D3
:4098800004460D461646002794F92001A84207D084F8205133463A468021204663F1DEF93846BDE8F0810000FF18170800401C46B0000020014691F8F30070472DE9F04104
:4098C00005460C461646002714B1012C00D0072795F8F300A04207D085F8F34033463A468121284663F1BAF93846BDE8F081014691F8260170472DE9F04104460D461646DD
:40990000002794F82601A84207D084F8265133463A468221204663F1A1F93846BDE8F0812DE9F04104460D4616460027D4F80801A84207D0C4F8085133463A468321204600
:4099400063F18CF93846BDE8F081014691F8250170472DE9F04104460D461646002794F82501A84207D084F8255133463A468421204663F173F93846BDE8F0810146B1F8B9
:409980001C0170472DE9F04104460D4616460027B4F81C01A84207D0A4F81C5133463A468521204663F15AF93846BDE8F081014691F8280170472DE9F04104460D461646A9
:4099C000002794F82801A84207D084F8285133463A468621204663F141F93846BDE8F0810246002070470146092070470346072070470146002070470346072070479FED6F
:409A0000FB0A70470146002070470346002070470146002070470346002070479FEDF30A7047024600BF00BF072070479FEDEF0A70470246072070479FEDEC0A7047034626
:409A4000072070470146062070470346072070479FEDE60A70470246072070479FEDE30A70470246072070479FEDE00A704702460720704701460020704703460720704776
:409A80000346072070472DE9F04105460C46164600271CB1022C01D00727002495F8F200A04207D085F8F24033463A468721284663F1D4F83846BDE8F081014691F8F1008F
:409AC000704710B50446204639F1B2F908B9012010BD0020FCE70146D1F8FC0070472DE9F04104460D4616460027D4F8FC00A84207D0C4F8FC5033463A468921204663F19B
:409B0000ADF83846BDE8F081014691F823017047014691F82201704770B5054600242846FFF7F6FF0443284639F10EF844EA80042846FFF7E9FF44EA0014284639F142F8B3
:409B400044EA8014204670BD2DE9F04104460D461646002794F82301A84207D084F8235133463A468A21204663F178F83846BDE8F0812DE9F04104460D461646002794F873
:409B80002201A84207D084F8225133463A468B21204663F163F83846BDE8F0812DE9F04105460C461646002704F0030028B1324601212846FFF7DDFF04E032460021284688
:409BC000FFF7D7FF04F00C0028B132460121284638F1BEFF04E032460021284638F1B8FF04F0300028B1324601212846FFF7ACFF04E0324600212846FFF7A6FF04F0C00027
:409C000028B132460121284638F1E0FF04E032460021284638F1DAFF3846BDE8F08100B502461046FFF757FF00F0C00008B1012000BD0020FCE7014691F8210170472DE912
:409C4000F04104460D461646002794F82101A84207D084F8215133463A468C21204662F1FDFF3846BDE8F08100B502461046FFF732FF00F4403008B1012000BD0020FCE7CF
:409C800000B502461046FFF726FF00F4405008B1012000BD0020FCE700B502461046FFF71AFF00F4400008B1012000BD0020FCE700B502461046FFF70EFF00F4404008B165
:409CC000012000BD0020FCE700B502461046FFF702FF00F0407008B1012000BD0020FCE700B502461046FFF7F6FE00F4402008B1012000BD0020FCE700B502461046FFF78B
:409D0000EAFE00F4401008B1012000BD0020FCE700B502461046FFF7DEFE00F0406008B1012000BD0020FCE700B502461046FFF7D2FE00F0300008B1012000BD0020FCE73B
:409D400000B502461046FFF7C6FE00F4406008B1012000BD0020FCE700B502461046FFF7BAFE00F4407008B1012000BD0020FCE700B502461046FFF7AEFE00F00C0008B1BF
:409D8000012000BD0020FCE70146B1F8180170472DE9F04104460D4616460027B4F81801A84207D0A4F8185133463A468D21204662F154FF3846BDE8F0810146B1F80E01CA
:409DC00070472DE9F04104460D4616460027B4F80E01A84207D0A4F80E5133463A468E21204662F13BFF3846BDE8F081000000000146B1F8100170472DE9F04104460D4603
:409E000016460027B4F81001A84207D0A4F8105133463A468F21204662F120FF3846BDE8F0810146B1F8160170472DE9F04104460D4616460027B4F81601A84207D0A4F8CA
:409E4000165133463A469021204662F107FF3846BDE8F0810146B1F8140170472DE9F04104460D4616460027B4F81401A84207D0A4F8145133463A469121204662F1EEFE88
:409E80003846BDE8F0810146B1F8120170472DE9F04104460D4616460027B4F81201A84207D0A4F8125133463A469221204662F1D5FE3846BDE8F0810146B1F80C017047EE
:409EC0002DE9F04104460D4616460027B4F80C01A84207D0A4F80C5133463A469321204662F1BCFE3846BDE8F0810146B1F81E0170472DE9F04104460D4616460027B4F8FB
:409F00001E01A84207D0A4F81E5133463A469421204662F1A3FE3846BDE8F0810146D1F8040170472DE9F04104460D4616460027D4F80401A84207D0C4F8045133463A46CB
:409F40009521204662F18AFE3846BDE8F081014691F8270170472DE9F04104460D461646002794F82701A84207D084F8275133463A469621204662F171FE3846BDE8F0816B
:409F80000146B1F81A0170472DE9F04104460D4616460027B4F81A01A84207D0A4F81A5133463A469721204662F158FE3846BDE8F0810146D1F8F40070472DE9F041044649
:409FC0000D4616460027D4F8F400A84207D0C4F8F45033463A469821204662F13FFE3846BDE8F0810146D1F8F80070472DE9F04104460D4616460027D4F8F800A84207D023
:40A00000C4F8F85033463A469921204662F126FE3846BDE8F0812DE9F04104460D4616460027A06CA8420DD0A564656533463A465621204662F112FE33463A4659212046D9
:40A0400062F10CFE3846BDE8F0810346072070470346072070470146D1F808017047000010B50446206968B1206902689FEDAF0A91688847206918B1206902685168884753
:40A0800000202061606968B1606902689FEDA70A91688847606918B1606902685168884700206061002020766076206881682046884710BD70B504460D46204662F126FD1A
:40A0C00004469B482060E5600020206160612046FFF7C6FF204670BD10B50446944820600020E060206968B1206902689FED8F0A91688847206918B120690268516888473E
:40A1000000202061606968B1606902689FED870A91688847606918B1606902685168884700206061204662F1F7FC0446204610BD70B504462046FFF7CFFF054667F1F2FC03
:40A1400070BD70B50546012406E07A4B00222146284662F183FD641C052CF6D370BD014600204A7E02F0010202B1012070472DE9F04104460D46164600272046FFF7EFFFA1
:40A18000A84210D0012D04D1607E40F00100607603E0607E20F00100607633463A460121204662F15BFD3846BDE8F0810246002013690B600B6803B10120704701460020D0
:40A1C0004A7E02F0040202B10120704710B52DED028B04462046FFF7F1FF08EE100A206928B120690268B8EE480A91688847606928B160690268B8EE480A91688847BDECAF
:40A20000028B10BD70B504460D46206958B1206902689FED460A91688847206918B1206902685168884725612046FFF7CFFF70BD0246002053690B600B6803B101207047A1
:40A2400070B504460D46606958B1606902689FED370A91688847606918B1606902685168884765612046FFF7B1FF70BD0146087E70472DE9F04104460D4616460027207EAD
:40A28000A84206D0257633463A460321204662F1E5FC3846BDE8F081014600204A7E02F0020202B1012070472DE9F04104460D46164600272046FFF7EFFFA84210D0012D9F
:40A2C00004D1607E40F00200607603E0607E20F00200607633463A460421204662F1BEFC3846BDE8F08170B5044600252046FFF736FF20B12046FFF7CFFF00B10125204678
:40A30000FFF75CFFA84210D0012D04D1607E40F00400607603E0607E20F004006076054B00220221204662F199FC70BD000000008C9D17088F1817082DE9F04704468946E8
:40A3400015461E46089FB846022C06D133462A460521404662F182FC00BF00BFBDE8F08710B50446206938B1206918B1206902685168884700202061606938B1606918B141
:40A380006069026851688847002060610020207760779FEDFD0A84ED080AA08484F8260010BD70B504460D46204662F1AFFB044604F10C0062F18CFCA0F10C04F348206023
:40A3C0001830E060002020616061A5612046FFF7C7FFEF48007884F82600ED4AED492046E4F0A9F84DB1EA480078401E82B22346AFF2BB01284662F1BCFB204670BD10B5E2
:40A400000446E24820601830E060A06920B1AFF2D701A06962F1F6FBDD4ADE49204669F161F92046FFF79CFF04F10C0062F15AFCA0F10C04204662F16FFB0446204610BDB6
:40A4400070B504462046FFF7DAFF054667F16AFB70BD10B504460C3C2046FFF7F1FF10BD10B504460C3C2046FFF7C9FF10BD70B50546012406E0C84B00222146284662F173
:40A48000EDFB641C062CF6D370BD70B504460D46206958B1206902689FEDBB0A91688847206918B12069026851688847256170BD70B504460D46606958B1606902689FEDD9
:40A4C000B20A91688847606918B16069026851688847656170BD10B52DED028B04469FEDAA0AB0EE408AA06928B1A0690268516A8847B0EE408AB0EE480ABDEC028B10BD00
:40A5000070B52DED028B0446B0EE408A0D460026B5EEC08AF1EE10FA05D203269FED9A0AB0EE408A0BE09FED9D0AB4EEC08AF1EE10FA04DD02269FED990AB0EE408A94EDA2
:40A54000080AB4EE480AF1EE10FA07D084ED088A2B4632460321204662F180FB3046BDEC028B70BD2DE9F04104460D4616460027607FA8423AD06577206908B1606908B916
:40A5800006272DE025B1012D0FD0022D27D119E0206902689FED7C0A91688847606902689FED790A9168884719E020690268B7EE000A91688847606902689FED730A9168EF
:40A5C00088470CE0206902689FED6F0A9168884760690268B7EE000A9168884700BF00BF33463A460421204662F138FB3846BDE8F0812DE9F0412DED028B05460C46164633
:40A600000027287FA04216D02C7733463A460121284662F123FB012C0DD1324600212846FFF7A0FF2846FFF756FFB0EE408A31462846FFF765FF3846BDEC028BBDE8F08116
:40A640000146087F70472DE9F04105460C461646002742F21070844201DD02270446A88CA04206D0AC8433463A460221284662F1F5FA3846BDE8F0810146888C704790ED18
:40A68000080A70470146487F7047024690690860086808B1012070470020FCE73C480078704700B50246002300200860FFF7F6FF904207DD3748006850F82200086008683A
:40A6C00000B10123184600BD30B52DED028B81B00446A069002868D0A08C00EE100AB8EE400ADFED2E0A80EE201AF0EE418AA06941F115FA0546C821DCF0A8F828B1264A4E
:40A7000000212046FFF72EFFF0E0A0690268516A8847B0EE408A94ED080A30EE280AB4EEC80AF1EE10FA6FD294F8260030B1012805D0022809D0032863D13DE000BF164A8A
:40A7400002212046FFF70EFF5BE069460020FFF7A8FF48B30098FFF7BEFEDFED110AB4EEE00AF1EE10FA09D32046FFF788FFDFED0D0AB4EEE00AF1EE10FA17DB064A022189
:40A780002046FFF7EFFE16E00000000064A410080C00001008000010C31817080000C842000064420000244200E0A0E0524A00212046FFF7D7FE24E069460120FFF771FF6E
:40A7C000C8B10098FFF787FE5FED0B0AB4EEE00AF1EE10FA09D32046FFF751FF5FED0F0AB4EEE00AF1EE10FA05DB434A02212046FFF7B8FE04E0404A00212046FFF7B2FE58
:40A8000000BF00BF72E0FFE794ED080A30EE680AB4EEC80AF1EE10FA63DD94ED080AB5EEC00AF1EE10FA5CD094F8260030B1012829D002284DD0032851D149E0694602204A
:40A84000FFF72FFFC8B12046FFF719FF5FED2C0AB4EEE00AF1EE10FA09D30098FFF73BFE5FED300AB4EEE00AF1EE10FA05DD224A01212046FFF776FE04E01F4A002120461E
:40A88000FFF770FE2BE069460320FFF70AFFC8B12046FFF7F4FE5FED3E0AB4EEE00AF1EE10FA09D30098FFF716FE5FED420AB4EEE00AF1EE10FA05DD0F4A01212046FFF744
:40A8C00051FE04E00C4A00212046FFF74BFE06E000BF094A01212046FFF744FE00BF00BF04E0054A00212046FFF73CFE00BF01B0BDEC028B30BD0000C3181708014691F88C
:40A900003400704770B503460A460324012A18DB1846FFF7F3FF904213DB1046D51702EB15752E1103F11C0555F826501146D61702EB16763611A2EB06167600F54005F006
:40A940000304204670BD0146C87D70472DE9F04105460C46164698460027012C55DB2846FFF7CCFFA04250DB2846FFF7ECFF20B12846FFF7E8FF032848D121462846FFF7A2
:40A98000C1FFB04242D0E21704EB1272131105F11C0252F823202146E31704EB13731B11A4EB03134FEA430C032303FA0CF39A432046E31704EB13734FEA231C05F11C0312
:40A9C00043F82C20E21704EB1272131105F11C0252F82320E31704EB13731B11A4EB03135B0006FA03F31A43E31704EB13734FEA231C05F11C0343F82C201030C1B24346F2
:40AA00003A46284662F12AF900E007273846BDE8F08170B50446002020756075A075E07502202076032060760020A076072084F83A00002506E0002104F11C0040F825103F
:40AA4000681CC5B220214800C11700EBD161012202EB6111A942EEDC002508E0681CC1B2FC4B03222046FFF771FF681CC5B2202DF4DB002044F8280FA0606060207360731A
:40AA8000E07320746074E07440F6C41060610020A06154F8280D81682046884770BD70B504460D46204662F131F8044604F10C0062F10EF9A0F10C04E74820601830E060AE
:40AAC00025612046FFF7A5FF204670BD10B50446E14820601830E0600020206104F10C0062F100F9A0F10C04204662F115F80446204610BD70B504462046FFF7E7FF05462F
:40AB000067F110F870BD10B504460C3C2046FFF7F1FF10BD10B504460C3C2046FFF7D6FF10BD70B50546012406E0CA4B00222146284662F193F8641C0F2CF6D9002407E0C9
:40AB400004F11101C34B0022284662F187F8641C2846FFF7D3FEA042F2D870BD0146087D70472DE9F04104460D4616460027207DA84206D0257533463A460121204662F11B
:40AB80006DF83846BDE8F0812DE9F04104460D4616460027E07DA84206D0E57533463A460221204662F15AF83846BDE8F0810146887D70470146C86A70472DE9F04104463F
:40ABC0000D4616460027E06AA84206D0E56233463A460821204662F141F83846BDE8F0810146487E70472DE9F04104460D4616460027607EA8420DD06576607E012803D100
:40AC0000964800688047A06233463A460921204662F124F83846BDE8F0810146086C70472DE9F04104460D4616460027206CA84206D0256433463A460A21204662F10EF8E8
:40AC40003846BDE8F0810146487D70472DE9F04105460C4616460027687DA04207D06C7533463A460C21284661F1F8FF06E02CB133463A460C21284661F1F0FF3846BDE8FF
:40AC8000F081014691F8380020B191F83B0008B1012070470020FCE72DE9F04104460D461646002794F83800A84207D084F8385033463A460421204661F1D0FF3846BDE83A
:40ACC000F081014691F8390070472DE9F04104460D461646002794F83900A84207D084F8395033463A460521204661F1B7FF3846BDE8F081014691F83B0070472DE9F04107
:40AD000004460D461646002794F83B00A8420FD094F83B0020B9324601212046FFF7BCFF84F83B5033463A460621204661F196FF3846BDE8F0810146C86B70472DE9F04192
:40AD400004460D4616460027E06BA84206D0E56333463A460721204661F180FF3846BDE8F081014691F83600704700B50246137E1046FFF7F6FF012804D1107E022801D061
:40AD8000012305E01046FFF7ECFF022800D10023184600BD2DE9F04104460D461646002794F818802046FFF7CEFDF8B9207E022803D145B94FF0000805E0012D01D1A84603
:40ADC00001E04FF00008207E40450FD02046FFF7C8FF012802D10220207601E084F8188033463A460D21204661F138FF3846BDE8F0812DE9F04104460D461646002794F8C0
:40AE000018802046FFF79FFD03281FD1207E022803D145B94FF0000805E0012D01D1A84601E04FF00008207E40450FD02046FFF798FF012802D10220207601E084F81880ED
:40AE400033463A460D21204661F108FF3846BDE8F081000095181708DC9D170818A010080146887E70472DE9F04104460D4616460027A07EA84206D0A57633463A460B219B
:40AE8000204661F1EBFE3846BDE8F0812DE9F04105460C4617464FF00008202C03DD20244FF0020803E014B901244FF0030895F83400A0421FD085F834402846FFF743FDD6
:40AEC00020B12846FFF73FFD03280ED1002608E0701CC1B2FC4B01222846FFF737FD701CC6B295F83400B042F2DC3B4642460E21284661F1B3FE4046BDE8F081014691F82E
:40AF000035007047014691F8370070472DE9F04104460D4616460027012D0FD12046FFF724FF012808D1206901F07AFC8046206904F038F8804501D30025022794F8370064
:40AF4000A84201D1012D07D184F8375033463A460F21204661F182FE3846BDE8F081014691F83A00704770B504460D466878C0F3C20694F83A00B04207D084F83A60D24B77
:40AF800000221021204661F169FE70BD70B505460C46A07800F00701CB4A2846FFF756FE70BD2DE9F04705460E464FF00408707800F00709B9F1070F02D04FF0010801E04C
:40AFC0004FF002082846FFF7BEFC40455FD100245BE02046E21704EB92729210121DB25C2146E31704EB93739B10A4EB83035B001A4102F00307601CC1B22846FFF782FC0C
:40B00000B84240D0601CC21700EB1272131105F11C0252F82320611CCB1701EB13731B11A1EB03134FEA430C032303FA0CF39A43C31700EB13734FEA231C05F11C0343F844
:40B040002C20C21700EB1272131105F11C0252F82320CB1701EB13731B11A1EB03135B0007FA03F31A43C31700EB13734FEA231C05F11C0343F82C201030C1B2924B002295
:40B08000284661F1EBFD601CC4B2102CA1DBBDE8F0872DE9F04105460E464FF00408707800F00707072F02D04FF0010801E04FF002082846FFF747FC404512D1022F01D17F
:40B0C000012400E0002495F83700A04201D1012C07D185F837407C4B00220F21284661F1BDFDBDE8F0812DE9FC5F05460E4604200190707800F0070795F818804FF0000BF3
:40B10000072F02D00120019001E0022001902846FFF74DFD28BB0198A8756B4B00220321284661F19BFD002417E0E21704EB92729210121DB25CE31704EB93739B10A4EB17
:40B1400083035B001A4102F00302032A03D00BF1010000F0FF0B601CC4B2102CE5DB85F835B02846FFF723FD02462846FFF7EBFB82426FD12846FFF7E6FB012804D028468B
:40B18000FFF7E1FB022865D1012F05D0022F02D0072F3CD102E000BF01273AE00027002000904FF00109824629E0296901F130006A46514615F081FFE8B100983BF18EFED5
:40B1C0008146B9F1100F16DCA9F10101CA1701EB92729210121DB25C0846C31700EB93739B10A0EB83035B001A4102F00302012A01D101270AE00AF1010000F0FF0A296969
:40B2000001F1300015F055FF5045CEDC01E0002700BF00BFB8F1020F03D147B94FF0000805E0012F01D1B84601E04FF00008287E40450FD02846FFF794FD012802D10220CF
:40B24000287601E085F818801F4B00220D21284661F104FDBDE8FC9F70B504460D461B4800688047206329462046FFF73CFF29462046FFF70EFF29462046FFF792FE294600
:40B280002046FFF783FE29462046FFF76CFE70BD70B504462046FFF7A3FC012818D14EF66021A06ADBF0D2FA20B32046FFF782FC451C054A29462046FFF77FFC0348006817
:40B2C0008047A06216E000009518170818A010082046FFF785FC032805D1216901F5D270FFF7CFFC30B90020A062454A00212046FFF763FC2046FFF726FB012804D020463C
:40B30000FFF721FB022827D140F6C411206BDBF09DFA08B300202076394B00220D21204661F19CFC002084F83700354B00220F21204661F193FC00206075314B00220C21A0
:40B34000204661F18BFC072084F83A002C4B00221021204661F182FC2046FFF728FC012804D02046FFF723FC02280DD14FF4FA61206BDBF06BFA38B10020A075204B0022AD
:40B380000321204661F16AFC207E022824D1206901F090F9092817D0206903F0AEF900281ADD206903F036FA0546206903F0A5F9854211D1206903F00DFE054606212069F5
:40B3C00003F00DFE854207D1002020760C4B00220D21204661F142FC70BD70B504460D46002694F83600A84201D084F83650044B32460D21204661F131FC304670BD00004C
:40B40000951817080021C1600174417481614161704710B50446204661F178FB04463D4820602046FFF7EEFF204610BD10B5044638482060E06838B1E06818B1E068026891
:40B44000516888470020E060204661F165FB0446204610BD70B504462046FFF7E7FF054666F160FB70BD70B50546012406E02A4B00222146284661F1F1FB641C022CF6D3D8
:40B4800070BD70B504460D46E06858B1E06802689FED220A91688847E06818B1E068026851688847E56070BD70B504460D461C4800688047A06165612068416920468847DA
:40B4C00070BD10B50446D4E90510DBF0BFF980F001002074207C617C884219D0207C60740D4B00220121204661F1B8FBE06878B1207C012806D1E0680268B7EE000A9168AC
:40B50000884705E0E06802689FED040A9168884710BD00000CA21008991817080000000018A010080021016101754175C16180F82010704710B50446204661F1E7FA0446EE
:40B5400004F10C0061F1C4FBA0F10C046A4820601830E060694A6A49204667F1CDFE2046FFF7E0FF204610BD10B50446624820601830E060206938B1206918B12069026889
:40B5800051688847002020615C4A5D49204668F1FCF804F10C0061F1A5FBA0F10C04204661F1BAFA0446204610BD70B504462046FFF7DAFF054666F1B5FA70BD10B50446B5
:40B5C0000C3C2046FFF7F1FF10BD10B504460C3C2046FFF7C9FF10BD70B50546012406E0484B00222146284661F138FB641C022CF6D370BD70B504460D46206958B1206997
:40B6000002689FED410A91688847206918B12069026851688847256170BD014691F82000704770B504460D460026207DA8423DD0206988B32046FFF7F0FFE0B1012D13D1AC
:40B64000207D08B9012000E000202075227D0AB1012200E0002200EE902AB8EEE00A206902689168884719E0022D01D1207DA8B10220207512E02575207D30B120690268A0
:40B68000B7EE000A9168884708E0206902689FED1E0A9168884701E0FFE70626207D6075184B00220121204661F1D8FA304670BD0146087D08B1012070470020FCE70246DB
:40B6C000002082F8201070470C480078704700B50246002300200860FFF7F6FF904205DD01230748006850F822000860086808B9002000BD1846FCE730A2170810000020E2
:40B700000C000020CD1817080000000070B504460D46164604212046FDF73CFC044642482060A560E66000202061B7EE000A84ED050A9FED3E0A84ED060A204670BD10B5E8
:40B740000446394820600020A060E06020612046FDF72CFC0446204610BD70B504462046FFF7EDFF054666F1DDF970BD014600208A6812B1CA6802B1012070470146012001
:40B78000704701460020704790ED050A704700B5014691ED060A9FED261AC0EE010A0846FFF7F2FF20EE800A00BD01460869704701460420704770B52DED028B04469FEDA5
:40B7C0001B0AB0EE408A206881682046884701281AD1A0680268D1688847A8B9E06860F197FE054613490968884700EE100AF8EEC00A2046FFF7C8FF20EE800AB0EE408A37
:40B800000D4800688047206184ED068ABDEC028B70BD80ED050A704701460020704770470146002070477047E8AA170800000000286B6E4E44FF0E0818A0100810B504468A
:40B84000204640F1BBF8002084F84300022084F84400002084F84500F8490870F8490860206881682046884710BD70B504460D462A46042120463FF1FFFF0446F148206019
:40B880003C30E060103020612046FFF7D7FF204670BD10B50446204640F130F80446204610BD70B504462046FFF7F3FF054666F139F970BD10B50446103C2046FFF7F1FFA6
:40B8C00010BD10B504460C3C2046FFF7EAFF10BD10B50446103C2046FFF7DBFF10BD10B504460C3C2046FFF7D4FF10BD70B50546012406E0D44B00222146284661F1AEF9D7
:40B90000641C0B2CF6D30D2406E0CF4B00222146284661F1A3F9641C102CF6D370BD9FEDCB0A704702460720704770B504460025E06930B1E069026891688847012800D14E
:40B940000125284670BD10B52DED028B04469FEDBF0AB0EE408AE06928B1E069026851698847B0EE408AB0EE480ABDEC028B10BD10B504462068016A2046884710BD70B5B1
:40B9800005460C46AD480470B14800688047AC490860AD4B00220F21284661F15FF970BD70B504460D46032D10D194F84400042802D0052804D100E000BF94F8445004E027
:40B9C00001212046FFF7DBFF00BF00BF94F84400A8421BD015B1012D0ED100BF94F84400012802D094F8440028B9974B00220C21204661F133F900E000BF00BF84F844503B
:40BA0000914B00220D21204661F128F970BD014691F84400704770B52DED028B0446E5692868C16A2846884794F8430010B101285AD15AE040F6B83181480068DAF006FF70
:40BA4000002851D02868416928468847B0EE408AE06902689169884760637B4B00220E21204661F1FBF8002000EE100AB8EE400AB4EEC08AF1EE10FA04D206212046FFF757
:40BA80008FFF30E042F2107000EE100AB8EE400AB4EEC08AF1EE10FA04DD03212046FFF77FFF20E09FED6B0AB4EEC08AF1EE10FA04DD00212046FFF773FF14E09FED660AF2
:40BAC000B4EEC08AF1EE10FA04D201212046FFF767FF08E02046FFF79AFF022803DB00212046FFF75DFF00BF48E041F2707154480068DAF0ABFE20B100212046FFF73FFFFB
:40BB00003BE02046FFF783FF032804D0042803D0052830D101E000BF00BF40F6B83148480068DAF093FE28B32868416928468847B0EE408AE0690268916988476063424B89
:40BB400000220E21204661F189F84FF47A7000EE100AB8EE400AB4EEC08AF1EE10FA04DD05212046FFF71CFF03E004212046FFF717FF00BF00E000BF00BF00BF00BFBDEC05
:40BB8000028B70BD70B50446E06940B3E069FDF71EFA012823D194F843002849097888421DD02B480068804725490860E56923480078012807D128463EF195FB06460121F1
:40BBC000CFF005FC06E028463EF18DFB06460221CFF0FDFB1948007884F8430000BF70BD70B504462068016920468847204640F10AF8E069002869D0E069FDF7E8F90128B0
:40BC00005BD0032860D1E5692868C16A284688472868416928468847B5EEC00AF1EE10FA2DD02068C16A2046884710B3012815D0022818D0032821D11AE00000400000202B
:40BC400044000020149E1708971817080000000018A010080020004500C0F34401212046FFF79EFE0AE000212046FFF799FE05E004E001212046FFF793FE00BF1CE0206862
:40BC8000C16A2046884788B1012804D0022807D0032810D109E000212046FFF781FE0AE001212046FFF77CFE05E004E000212046FFF776FE00BF00BF07E02046FFF762FF3E
:40BCC0002046FFF7A8FE00E000BF00BF70BD014691F84500704702460320022900D1022082F845107047000010B5044620463FF165FE206881682046884710BD70B50446F2
:40BD00000D462A460B2120463FF1B6FD0446454820603430E060103020612046FFF7E4FF204670BD10B5044620463FF1E7FD0446204610BD70B504462046FFF7F3FF05462F
:40BD400065F1F0FE70BD10B50446103C2046FFF7F1FF10BD10B504460C3C2046FFF7EAFF10BD10B50446103C2046FFF7DBFF10BD10B504460C3C2046FFF7D4FF10BD70B59F
:40BD80000546012406E0284B00222146284660F165FF641C0B2CF6D370BD9FED240A704702460720704710B50446E06930B1E06902689168884708B1012010BD0020FCE76C
:40BDC00010B52DED028B04469FED180AB0EE408AE06928B1E069026851698847B0EE408AB0EE480ABDEC028B10BD10B504462068016A2046884710BD10B5044620680169B9
:40BE00002046884720463FF1FEFEE06940B1E069FDF7DDF8032803D1E0690268D16A884710BD00003CA51008C71817080000000001480068704700001C05002000000000C6
:40BE40000000000000000000000000003037373031373134353500000000000030373730313731343335000000000000526176656E20496E64757374726965732C20496E71
:40BE8000632E000000000000000000005365702D31332D32303138000000000032322E332E312E370000000000000000526176656E205261746520436F6E74726F6C204DA1
:40BEC0006F64756C6500000000000000303737303137313433390000000000000000000000000000000000000000000000000000000000000000000000000000FFFFFFFF26
:40BF0000FFFFFFFFFFFFFFFFFFFFFFFFFFFFFFFFFFFFFFFFFFFFFFFFFFFFFFFFFFFFFFFFFFFFFFFFFFFFFFFFFFFFFFFFFFFFFFFFFFFFFFFFFFFFFFFFFFFFFFFFFFFFFFFF41
:40BF4000FFFFFFFFFFFFFFFFFFFFFFFFFFFFFFFFFFFFFFFFFFFFFFFFFFFFFFFFFFFFFFFFFFFFFFFFFFFFFFFFFFFFFFFFFFFFFFFFFFFFFFFFFFFFFFFFFFFFFFFFFFFFFFFF01
:40BF8000FFFFFFFFFFFFFFFFFFFFFFFFFFFFFFFFFFFFFFFFFFFFFFFFFFFFFFFFFFFFFFFFFFFFFFFFFFFFFFFFFFFFFFFFFFFFFFFFFFFFFFFFFFFFFFFFFFFFFFFFFFFFFFFFC1
:40BFC000FFFFFFFFFFFFFFFFFFFFFFFFFFFFFFFFFFFFFFFF00001408FFFF150800C00008FFFF0F0800900008FBBF000804880008F78F000800800008FF870008DF17EB14BA
:40C0000000487047B88600102DE9F0470446894615461E46DDF820804746092C11D004DC012C15D0072C1CD104E0632C11D0672C17D10FE033462A467A21384660F10EFE47
:40C0400020E033462A467B21384660F107FE19E000BF00BF33462A467C21384660F1FEFD10E0892C01D3C82C05D9B4F5A47F08D9B4F5C47F05D833462A467C21384660F18A
:40C08000EDFD00BF00BFBDE8F0872DE9F0470446894615461E46089FB846A01E0F286BD2DFE800F04039474E555C63161D6A240F082B320033462A468821404660F1CEFDBE
:40C0C00066E033462A468721404660F1C7FD5FE033462A468421404660F1C0FD58E033462A468521404660F1B9FD51E033462A468621404660F1B2FD4AE033462A46892115
:40C10000404660F1ABFD43E033462A468A21404660F1A4FD3CE033462A467E21404660F19DFD35E033462A467D21404660F196FD2EE033462A467F21404660F18FFD27E035
:40C1400033462A468021404660F188FD20E033462A468121404660F181FD19E033462A468221404660F17AFD12E033462A468321404660F173FD0BE0112C08D3502C06D803
:40C1800004F17A0133462A46404660F167FD00BF00BFBDE8F0872DE9F04704460F4690469946089D2E46214606F1180041F197FCBDE8F08770B50446D4F8E80188B1D4F817
:40C1C000E80102689FEDFE0A91688847D4F8E80120B1D4F8E8010268516888470020C4F8E801D4F8EC0188B1D4F8EC0102689FEDF40A91688847D4F8EC0120B1D4F8EC01F4
:40C200000268516888470020C4F8EC01D4F8F00188B1D4F8F00102689FEDE90A91688847D4F8F00120B1D4F8F0010268516888470020C4F8F001D4F8F40188B1D4F8F4011A
:40C2400002689FEDDF0A91688847D4F8F40120B1D4F8F4010268516888470020C4F8F401D4F8F80188B1D4F8F80102689FEDD40A91688847D4F8F80120B1D4F8F8010268DD
:40C28000516888470020C4F8F801D4F8FC0188B1D4F8FC0102689FEDCA0A91688847D4F8FC0120B1D4F8FC010268516888470020C4F8FC01D4F8000250B1D4F8000220B128
:40C2C000D4F800020268516888470020C4F80002D4F8040250B1D4F8040220B1D4F804020268516888470020C4F80402002004F5027420706070A0700120E0700020207163
:40C30000A4F50274002511E0002104F2192041550A3041550C210A304155002004F50E7202EBC50210605060681CC5B20A2DEBDB9FEDA40A04F5227484ED000A9FEDA20A44
:40C3400084ED010A0020A06020646064A0649F4800688047E0609D4800688047206100206061A061E061C82020620020A062974800688047E0620020E06420656065A06538
:40C38000A4F860000F2084F86200002084F86300012084F86400002084F88E0084F88F0084F8900084F8910084F8920084F89500012084F89300002084F8940084F8960095
:40C3C00084F89700012084F89800002084F8990084F89A0084F89C00A4F5227400BF0BE0002204F225310A5404F20D210A5404F231310A54411CC8B20C28F1DB002004F2C8
:40C400002334A076E07620776077A077E0772070A4F2233404F5D270FEF7FBFA04F1300014F0FFFF6A4820F0C1F8206881682046884770BD2DE9F04781460E4617461C461F
:40C440004FF0000800202060002515E0214628463FF1A3FA70B120683FF15DFBB04207D120683FF174FBB84202D14FF0010807E000202060681CC5B23FF18CFAA842E5DCFF
:40C4800000BF4046BDE8F087F8B504460D466946284635F157FF88B3009835F1F0FF0A2810D005DC58B105280ED0092819D10AE00B2805D0132804D0142812D105E000BF6A
:40C4C00000BF00BF00BF00BF00BF009835F1CAFF0646404B3246002104F1300016F021FA0BE0009835F1BEFF06463A4B3246012104F1300016F015FA00BF00BFF8BD2DE9F0
:40C50000FE430446002623E002AA314604F1300014F0D3FDD0B102983AF1E0FC0546012D14DB04F5D270FEF7E9F9A8420EDB294604F5D270FEF7E6F9012800D100E0002044
:40C540000746244A394602983AF1EBFC701CC6B204F1300014F0ADFDB042D5DC01AA002104F1300016F015F8D0B10198FDF77EFE0546012D14DB04F5D270FEF7BFF9A84293
:40C580000EDB294604F5D270FEF7BCF9012800D100E0002007460F4A39460198FDF784FE01AA012104F1300015F0F3FF38B30198FDF75CFE0546012D21DB04F5D2700BE0BA
:40C5C00000000000000070420000044218A01008CC1800109B181708FEF790F9A8420EDB294604F5D270FEF78DF9012800D100E000200746FC4A39460198FDF755FE6A469B
:40C60000012104F1300016F008FDD0B100983BF103FD0546294604F5D270009FFEF772F9012800D100E0002080463868EE4A414643693846984700980068C16900988847B6
:40C6400000BF6A46002104F1300016F0E6FCD0B100983BF1E1FC0546294604F5D270009FFEF750F9012800D100E0002080463868DD4A414643693846984700980068C169E8
:40C680000098884700BFBDE8FE832DE9F04104460D4616460027D4F89002A84207D0C4F8905233463A461021204660F1D7FA3846BDE8F081014691F80A02704770B50446C2
:40C6C000DF2533F152FD00B90025C4F8E452C64B00221A21204660F1C1FA70BD0146D1F8E40270470146D1F89C027047014691F82103704770B5044601252046FFF7F6FF43
:40C7000000B10DE02046FFF7D5FF042807D004F5D270FEF72AFB18B1D4F89C0200B90025284670BD2DE9F04105460C4617460026AE480068804740F2BF11884203DA284684
:40C74000FFF7D8FF18B9002C00D902260024D5F89C02A04200D13EB1C5F89C423B4632461621284660F17AFA3046BDE8F08170B504469E48006880470546D4F8A46220462C
:40C78000FFF7B0FF00281FD940F2BF10854211D34FF47A71D4F8E002DAF058F828B1924A00212046FFF7BEFF13E02046FFF79AFF05460EE08E4800688047C4F8E0022046F9
:40C7C000FFF790FF054604E0894800688047C4F8E002D4F8A402A84207D0C4F8A452824B00221821204660F139FA2046FFF776FFA84204D82046FFF771FFB04209D8204654
:40C80000FFF76CFFA8420AD92046FFF767FFB04205D8754B00221921204660F11FFA70BD0146D1F8A402704738B50546002000902846FFF7F5FF02462846FFF74FFF8242B5
:40C8400014D200240FE06B46062221462846FFF7F1FD30B100980068634A0021036B00989847601CC4B2052CEDDB13E000240FE06B46062221462846FFF7DCFD30B10098B2
:40C880000068594A0121036B00989847601CC4B2052CEDDB38BD70B50446002504F5D270FEF7EFF950B104F5D270FEF70AFA28B904F5D270FEF794F9012816D104F5D270BC
:40C8C000FEF753FA01280FD104F1300016F069F8012805D004F1300016F063F8032801D1022502E0012500E0002594F80902A84207D084F809523C4B00220F21204660F1ED
:40C90000ADF970BD2DE9F84F04464FF0000804F1300014F0CEFB834604F5D270FDF7EEFF83451BDA002512E06A46414604F1300014F0C3FB48B1681CC1B22B4A00983AF145
:40C94000D0FA08F1010000F0FF08681CC5B204F1300014F0AEFBA842E6DC8DE004F1300014F0A7FB834604F5D270FDF7C7FF9BFBF0F000F0FF0904F1300014F09AFB834698
:40C9800004F5D270FDF7BAFF9BFBF0F100FB11B000F0FF0A04F5D270FDF7B0FFA0EB0A0B0BEBDB70C0F34707002518E0002612E06A46414604F1300014F07FFB48B1681C17
:40C9C000C1B2094A00983AF18CFA08F1010000F0FF08701CC6B24E45EADB681CC5B2BD42E4DB3D4621E000009B181708AC00002018A01008002612E06A46414604F13000BC
:40CA000014F05BFB48B1681CC1B2FA4A00983AF168FA08F1010000F0FF08701CC6B209F101008642E8DB681CC5B207EB0A00A842E0DC07EB0A00C5B218E0002612E06A46F8
:40CA4000414604F1300014F038FB48B1681CC1B2E84A00983AF145FA08F1010000F0FF08701CC6B24E45EADB681CC5B204F5D270FDF744FFA842E0DCBDE8F88F38B50446EC
:40CA80000020009004F5D270FDF75DFF28BB04F1300014F00EFB0546D64A294604F5D270FEF7F4F92046FFF72DFF6A46002104F1300015F06EFD20B1CE4A00210098FDF7AB
:40CAC000D8FB6A46012104F1300015F062FD20B1C84A00210098FDF7CCFB38BD2DE9F04180460E4614460027002020600A2E16DA00250FE02146284635F124FC40B120686A
:40CB000035F1B0FCB04201D1012707E000202060681CC5B235F113FCA842EBDC00BF3846BDE8F081024600200A2902DA02F21923585C70472DE9F04104460D461646002703
:40CB4000072E12D2DFE806F004B62944638F120094F80C0248B9002084F80C02A54A294604F1300015F021FF0127B3E094F80C0218B194F80C0206280ED11DB9002084F890
:40CB80000C0202E0062084F80C029A4A294604F1300015F00AFF01279CE094F80C0238B194F80C02022803D094F80C0206280ED11DB9002084F80C0202E0022084F80C02DC
:40CBC0008C4A294604F1300015F0EFFE012781E094F80C0258B194F80C02022807D094F80C02062803D094F80C0203280ED11DB9002084F80C0202E0032084F80C027D4AFD
:40CC0000294604F1300015F0D0FE012762E094F80C0278B194F80C0202280BD094F80C02042807D094F80C02062803D094F80C02032817D165B9022084F80C02002120468B
:40CC4000FFF770FF0F2801D1002504E0022502E0042084F80C02674A294604F1300015F0A4FE012736E094F80C0298B194F80C0202280FD094F80C0204280BD094F80C029B
:40CC8000062807D094F80C02032803D094F80C0205280ED11DB9002084F80C0202E0052084F80C02534A294604F1300015F07DFE01270FE01DB9002084F80C0202E00120D5
:40CCC00084F80C024B4A294604F1300015F06DFE012700BF00BF3846BDE8F081014691F80902704710B5044604F5D270FEF70AF918B3414800688047012808D02046FFF723
:40CD0000EDFF20B104F1300015F032FE58B9394A002104F5D270FEF7F9F8032200212046FFF708FF09E0354800688047C4F89402032201212046FFF7FDFE10BD90EDA30AE1
:40CD40007047F0B52DED028B83B00746002002900190002439E06946204635F1F3FA90B3002529E00098006802AA294683690098984701281ED1029833F13CFA032819D079
:40CD8000029833F137FA042814D0029833F132FA03280FD001A9029833F14DFA50B13846019EFFF7CBFFB0EE408A3068C1683046884700BF681CC5B200980068C169009809
:40CDC0008847A842CEDC601CC4B235F1B8FAA042C1DC03B0BDEC028BF0BD90EDA20A7047F0B52DED028B83B0074600200290019000243FE09B181708B000002018A010084D
:40CE00006946204635F19EFA90B3002529E00098006802AA294683690098984701281ED1029833F1E7F9032809D0029833F1E2F9042804D0029833F1DDF907280FD101A990
:40CE4000029833F1F8F950B13846019EFFF7C5FFB0EE408A3068C1683046884700BF681CC5B200980068C16900988847A842CEDC601CC4B235F163FAA042C1DC03B0BDEC8E
:40CE8000028BF0BD014691F80B027047014691F81C037047014691F81B037047014691F81D03704770B5044600252046FFF7F6FF002866D02046FFF7EDFF18B92046FFF7FA
:40CEC000E5FFA0B32046FFF7DDFF0A2803D02046FFF7DCFF30B10125FE4800688047C4F898022AE02046FFF7CDFF28B9F94800688047C4F8980220E02046FFF7C3FF4EF67A
:40CF0000602100FB01F63146D4F89802D9F09EFC08B9012511E0F049D4F89802D9F096FC58B1EC4800688047C4F8980205E0FFE7E84800688047C4F89802D4F8F80140B174
:40CF4000D4F8F801026800EE105AB8EE400A91688847D4F8FC0140B1D4F8FC01026800EE105AB8EE400A9168884794F81E03A84207D084F81E53D94B0022052120465FF1F8
:40CF80006DFE70BD2DE9FF4106460F46B5B23C460020039028467C2D76D020DC162847D00EDC04282CD006DC012824D0022826D003286AD128E00A2868D00F28F9D12FE07F
:40CFC000222829D006DC192873D01A2872D02128EFD11DE07A286ED07B28EAD1BFE07D380E2852D2DFE800F0A5A4A9AAB2B3D93438392C28686C2046FFF754FF2AE100BF3B
:40D000002046FFF74FFF25E12046FFF74BFF21E12046FFF7E5FE1DE12046FFF792FE19E12046FFF75FFE04F1300014F09CFC11E12046FFF79CFB0DE12046FFF760FA09E188
:40D040002046FFF728FC04F1300014F08CFC01E12046FFF720FCFDE0FCE004F5D270FDF77DFD804603AA41469D48FFF737FDF8B104F5D270FDF7E7FD022808D100220221B6
:40D08000039834F1B7FF13E06DE086E077E004F5D270FDF7D8FD012805D100220121039834F1A8FF04E000220321039834F1A2FFD0E05CE05FE04BE02046FFF713FEC9E058
:40D0C00004F5D270FDF74AFD804603AA41468448FFF704FD58B304F5D270FDF740FF28B900221146039835F160FA20E004F5D270FDF735FF01280AD100221146039835F16E
:40D10000EBF900220121039835F14FFA0FE004F5D270FDF724FF022809D100220121039835F1DAF900220121039835F13EFA91E090E02046FFF7A2FC8CE000BF2046FFF701
:40D14000AAFB04F1300014F00EFC83E082E081E02046FFF793FC2046FFF7D1F97AE02046FFF799FB76E02046FFF7C9F972E02046FFF75AFB6EE02046FFF7F9FA6AE0204692
:40D18000FFF79CFA2046FFF795FA0A2804D1002211462046FFF779FA5CE08B2D05DBCA2D03DC2046FFF7ABF953E04D2D08DB562D06DCA5F14D00C1B22046FFF765F948E0D2
:40D1C00040F2E330854244DBB5F57A7F41DC0020029001900090A5F2E3301FFA80F808F0FF0102AB03222046FFF724F980B308F0FF016B4607222046FFF71CF900B3029830
:40D2000017F0C4FF0B2802D00D2812D10BE00022012100983FF130F801AB032200213048FFF708F90BE00022022100983FF124F805E00022114600983FF11EF800BF00BFB9
:40D240000099029818F0A8FADDE9011018F09AFA00BF00BF00BFBDE8FF8138B5044620465FF154FC044604F10C005FF131FDA0F10C0404F110005FF115FDA0F110041948E8
:40D2800020601830E06010302061AFF20733022240F2265104F11800009440F13BFBA0F11804214604F1300014F0FDFEA0F13004214604F5D270FDF7F2FBA0F5D27400207A
:40D2C00004F5F47420606060A060E06020616061A06109E018A01008C02709009B181708C8060010709E1708C4F8C400C4F8D000C4F8D800C4F8DC00A4F5F4742046FEF7F0
:40D3000059FF23460022F84920465FF132FC23460022F64904F5D2705FF12BFC23460022F34904F130005FF124FC204638BD10B50446F04820601830E06010302061D4F8D6
:40D34000E80188B1D4F8E80102689FEDEB0A91688847D4F8E80120B1D4F8E8010268516888470020C4F8E801D4F8EC0188B1D4F8EC0102689FEDE00A91688847D4F8EC0125
:40D3800020B1D4F8EC010268516888470020C4F8EC01D4F8F00188B1D4F8F00102689FEDD60A91688847D4F8F00120B1D4F8F0010268516888470020C4F8F001D4F8F4010C
:40D3C00088B1D4F8F40102689FEDCB0A91688847D4F8F40120B1D4F8F4010268516888470020C4F8F401D4F8F80188B1D4F8F80102689FEDC10A91688847D4F8F80120B1A8
:40D40000D4F8F8010268516888470020C4F8F801D4F8FC0188B1D4F8FC0102689FEDB60A91688847D4F8FC0120B1D4F8FC010268516888470020C4F8FC01D4F8000250B11A
:40D44000D4F8000220B1D4F800020268516888470020C4F80002D4F8040250B1D4F8040220B1D4F804020268516888470020C4F80402A2481FF09AF804F5D270FDF726FB78
:40D48000A0F5D27404F1300014F049FEA0F1300404F1180040F168FAA0F1180404F110005FF105FCA0F1100404F10C005FF11AFCA0F10C0420465FF12FFB0446204610BDAF
:40D4C00070B504462046FFF732FF054664F12AFB70BD10B50446103C2046FFF7F1FF10BD10B504460C3C2046FFF7EAFF10BD10B50446103C2046FFF71AFF10BD10B50446B5
:40D500000C3C2046FFF713FF10BD7CB50546012406E07B4B0022214628465FF19FFB641C40F226508442F4D9D5F8000220B1D5F8000202689168884705F1300014F0CDFEE9
:40D5400005F5D270FDF7EDFA00240AE0E0B201A934F1F8FE20B101980068816801988847641C34F1ECFEA042F0D800240AE0E0B269463EF112FA20B10098006881680098F7
:40D580008847641C3EF106FAA042F0D87CBDF8B50646012500240EE06946204634F1D2FE38B100980068816C0098884708B9002505E0601CC4B234F1C2FEA042ECDC00BF87
:40D5C0002846F8BD2DE9F04704468A4616461F46DDF82080C146012C06D00C2C20D00D2C26D00E2C34D12BE0002508E005F2E6413B46324648465FF131FB681CC5B2052D65
:40D60000F4DB3B46324640F2E54148465FF126FB3B46324640F2EB4148465FF11FFB23E03B46324640F2E34148465FF117FB1BE03B46324640F2E44148465FF10FFB13E014
:40D640003B46324640F2E54148465FF107FB0BE00F2C08D3132C06D804F2D7413B46324648465FF1FBFA00BF00BFBDE8F0872DE9F04705460C4616461F46DDF82080C146C0
:40D680000F2D10D008DC022D15D00A2D23D00C2D19D00E2D56D135E0102D4BD0112D39D0122D4FD13EE004F2C7413B46324648465FF1D4FA47E004F2BB413B463246484634
:40D6C0005FF1CCFA3FE004F2CB413B46324648465FF1C4FA37E004F2CF413B46324648465FF1BCFA2FE0000097C100088BC0000809C00008709E170800000000CC18001000
:40D700009B18170804F2D3413B46324648465FF1A5FA18E004F2D7413B46324648465FF19DFA10E004F2DB413B46324648465FF195FA08E004F2DF413B46324648465FF1E6
:40D740008DFA00E000BF00BFBDE8F0872DE9F04705460C4616461F46DDF82080C1460E2D1AD004DC022D1FD00D2D2DD104E00F2D0AD0102D28D11FE004F2A9413B4632461E
:40D7800048465FF16BFA20E004F2AF413B46324648465FF163FA18E004F2B5413B46324648465FF15BFA10E004F2A3413B46324648465FF153FA08E004F29D413B46324659
:40D7C00048465FF14BFA00E000BF00BFBDE8F0872DE9F04705460C4616461F46DDF82080C1460E2D1AD004DC022D1FD00D2D2DD104E00F2D0AD0102D28D11FE004F285411F
:40D800003B46324648465FF129FA20E004F28B413B46324648465FF121FA18E004F291413B46324648465FF119FA10E004F27F413B46324648465FF111FA08E004F2974152
:40D840003B46324648465FF109FA00E000BF00BFBDE8F0872DE9F04705460C4616461F46DDF82080C146062C77DAA81E0E2872D2DFE800F0070F171F272F373F47714F573D
:40D880005F6704F231413B46324648465FF1E6F962E004F23D413B46324648465FF1DEF95AE004F243413B46324648465FF1D6F952E004F249413B46324648465FF1CEF976
:40D8C0004AE004F24F413B46324648465FF1C6F942E004F255413B46324648465FF1BEF93AE004F25B413B46324648465FF1B6F932E004F261413B46324648465FF1AEF94C
:40D900002AE004F267413B46324648465FF1A6F922E004F26D413B46324648465FF19EF91AE004F273413B46324648465FF196F912E004F279413B46324648465FF18EF9AB
:40D940000AE004F237413B46324648465FF186F902E002E0FFE700BF00BFBDE8F0872DE9F04705460C4616461F46DDF82080C146052C5FDAA81E11285AD2DFE800F0091128
:40D980005959595959592959313941192149510004F2FF313B46324648465FF15FF948E004F20E413B46324648465FF157F940E004F204413B46324648465FF14FF938E0D5
:40D9C00004F209413B46324648465FF147F930E004F213413B46324648465FF13FF928E004F583613B46324648465FF137F920E004F21D413B46324648465FF12FF918E030
:40DA000004F222413B46324648465FF127F910E004F227413B46324648465FF11FF908E004F22C413B46324648465FF117F900E000BF00BFBDE8F0872DE9F04705460C46C3
:40DA400016461F46DDF82080C146062C77DAA81E0E2872D2DFE800F0070F171F272F373F47714F575F6704F29B313B46324648465FF1F4F862E004F2A7313B463246484697
:40DA80005FF1ECF85AE004F2AD313B46324648465FF1E4F852E004F2B3313B46324648465FF1DCF84AE004F2B9313B46324648465FF1D4F842E004F2BF313B46324648467E
:40DAC0005FF1CCF83AE004F2C5313B46324648465FF1C4F832E004F2CB313B46324648465FF1BCF82AE004F2D1313B46324648465FF1B4F822E004F2D7313B4632464846DE
:40DB00005FF1ACF81AE004F2DD313B46324648465FF1A4F812E004F2E3313B46324648465FF19CF80AE004F2A1313B46324648465FF194F802E002E0FFE700BF00BFBDE837
:40DB4000F0872DE9F04705460C4616461F46DDF82080C146022C64DAA81E0C285FD2DFE800F00E06161E262E363E465E4E5604F2EB313B46324648465FF170F850E004F2EA
:40DB8000E9313B46324648465FF168F848E004F2ED313B46324648465FF160F840E004F2EF313B46324648465FF158F838E004F2F1313B46324648465FF150F830E004F2F7
:40DBC000F3313B46324648465FF148F828E004F2F5313B46324648465FF140F820E004F2F7313B46324648465FF138F818E004F2F9313B46324648465FF130F810E004F295
:40DC0000FB313B46324648465FF128F808E004F2FD313B46324648465FF120F800BF00BF00BFBDE8F0872DE9F04107460C46002C59D020463DF18BFF064620463DF16BFFCA
:40DC400005460F2E4ED2DFE806F0081211131B101C242C343C4D4D444C003B462A46AFF21D1120465EF185FF3CE000BF00BF39E03B462A46AFF23F2120465EF17AFF31E0F3
:40DC800030E03B462A46AFF2293120465EF171FF28E03B462A46AFF2434120465EF169FF20E03B462A46AFF2D74120465EF161FF18E03B462A46AFF26B5120465EF159FFF6
:40DCC00010E03B462A46AFF2596120465EF151FF08E03B462A46AFF2137120465EF149FF00BF00BF00BFBDE8F0812DE9F04704460D4616461F46DDF82080C146012C07D169
:40DD000005F211513B46324648465EF1A7FF00BF00BFBDE8F08770B504460D46164623463246AFF2390128465EF123FF70BD2DE9F0470446894615461E46089FB84600BF05
:40DD40004CB1F02C07D804F1CA0133462A4640465EF184FF19E0F12C0AD3B4F5F07F07D804F1CA0133462A4640465EF177FF0CE0B4F5F07F09D9B4F5347F06D804F1CA01EC
:40DD800033462A4640465EF169FF00BF00BFBDE8F08770B504460025D4F80402A8B91420DFF070FB061E04D030463CF1FCFA064600E00020C4F8040223460022AFF2910111
:40DDC000D4F804025EF1D5FE00BF284670BD2DE9F0470446894615461E46089FB846012C04D0022C09D0032C15D10DE033462A46612140465EF132FF25E033462A4662211F
:40DE000040465EF12BFF1EE033462A46632140465EF124FF17E0042C09D30E2C07D804F1600133462A4640465EF118FF0AE00F2C08D3192C06D804F1600133462A46404651
:40DE40005EF10CFF00BF00BFBDE8F08702460020D2F800320B600B6803B1012070472DE9FC4705460C4616461F46DDF82880C1460020019000900A2C4BDA7D2D1BD2192D2C
:40DE800004D01A2D0AD0532D14D10FE004F143013B46324648465EF1E1FE0BE004F14D013B46324648465EF1D9FE03E04846FEF705FC00BF00BFE1B201AA4846FEF70EFE9E
:40DEC00038B3019834F1CAFA062821D2DFE800F00304051D1E1F1BE01AE0B42D13D169464846FFF7B3FF68B1E1B2009835F176FD40B1019807F03BFC20B9FE4A0021009869
:40DF000035F156FD00BF00BF02E001E000E000BF00BFBDE8FC872DE9FE4F044600264FF00C08002001900090002510E1012702AA29462046FEF7D2FD90B1029834F187FA36
:40DF4000814629462046FEF7EDFD814501D1002706E0029820B102980068416802988847012F6FD129462046FEF7DCFD1B280FD2DFE800F00E120F10131435365473747593
:40DF8000769977B77879B8B91115167AD7177B00C7E000BF00BF00BF00BF00BF00BF00BF00BF4FF43A70DFF06DFAB0F100090CD029462046FEF7B6FD824623462A465146A6
:40DFC000484607F07DFE814600E00020029023462A46AFF2751102985EF1CBFDA1E000BF4FF4EC70DFF04EFAB0F100090CD029462046FEF797FD824623462A465146484677
:40E000000CF0E9FB814600E00020029023462A46AFF2B51102985EF1ACFD82E04FF49670DFF030FAB0F100090DD029462046FEF779FD824623462A4651464846FBF71FF89B
:40E04000814601E06EE00020029023462A46AFF2F11102985EF18DFD63E000BF00BF00BF00BF00BF00BF00BF00BF4FF42270DFF009FAB0F100090CD029462046FEF752FD88
:40E08000824623462A465146484601F0DDFE814600E00020029023462A46AFF23D2102985EF167FD3DE04FF4AA70DFF0EBF9B0F100090CD029462046FEF734FD8246234671
:40E0C0002A465146484636F133FA814600E00020029023462A46AFF2792102985EF149FD1FE000BF00BF4FF4BE70DFF0CBF9B0F100090CD029462046FEF714FD8246234688
:40E100002A46514648460FF000FF814600E00020029023462A46AFF2B92102985EF129FD00BF00BF29462046FEF7FCFC022804D0032803D0142806D101E000BF00BF0EB91B
:40E140000126A84600E000BF00BF681CC5B20A2DFFF6ECAE674A314604F1300014F0B2FE01A9654813F048FC38B3624A4146019839F1EAFA41462046FEF7D4FC022805D155
:40E180005C4A0121019839F1AEFB16E041462046FEF7C8FC032805D1564A0221019839F1A2FB0AE041462046FEF7BCFC142804D1504A0321019839F196FBD4F8000238B10D
:40E1C000D4F8000220B1D4F800020268516888472046FEF76FFA072804D02046FEF76AFA06281CD13C20DFF04DF9B0F1000905D02146484635F122F9814600E00020C4F876
:40E20000000269463C483038FFF720FE30B123460022AFF2454100985EF1ABFC00BFBDE8FE8F30B503460A460025284629460A2A04DA03F50E7404EBC20403CC30BD2DE988
:40E24000F047074614461D46DDE908694FF000080A2E17DA07F50E7000EBC60006C884EA010085EA020108430ED007F50E7000EBC60030C006F157014B46424638465EF163
:40E28000EDFC01E04FF007084046BDE8F0872DE9F04104460D461646002794F80B02A84207D084F80B5233463A46012120465EF1D5FC3846BDE8F08102460020D2F8F8317A
:40E2C0000B600B6803B10120704770B504460D46D4F8F80138B1D4F8F80120B1D4F8F801026851688847C4F8F8512046FEF7DAFD70BD00009B181708F8060010024600204B
:40E30000D2F8FC310B600B6803B10120704770B504460D46D4F8FC0138B1D4F8FC0120B1D4F8FC01026851688847C4F8FC512046FEF7B8FD70BD014691F81E03704701467E
:40E3400091F81F0370472DE9F04104460D461646002794F81F03A84207D084F81F5333463A46062120465EF179FC3846BDE8F0810146D1F8A80270470146D1F8AC027047B3
:40E380002DE9F04104460D4616460027D4F8AC02A84207D0C4F8AC5233463A461C2120465EF15CFC3846BDE8F081014691F8200370472DE9F04104460D461646002794F88D
:40E3C0002003A84207D084F8205333463A46072120465EF143FC3846BDE8F08102460020D2F8E8310B600B6803B101207047014691F81603704770B5044600252046FFF75C
:40E40000F6FF48B304F1300013F0ACFF00B90125D4F8E80140B1D4F8E801026800EE105AB8EE400A91688847D4F8EC0140B1D4F8EC01026800EE105AB8EE400A9168884788
:40E4400094F81703A84207D084F81753FA4B0022092120465EF102FC70BD70B504460D46D4F8E80138B1D4F8E80120B1D4F8E801026851688847C4F8E8512046FFF7BBFF46
:40E4800070BD02460020D2F8EC310B600B6803B10120704770B504460D46D4F8EC0138B1D4F8EC0120B1D4F8EC01026851688847C4F8EC512046FFF79EFF70BD014691F8EE
:40E4C000170370472DE9F04104460D461646002794F81B03A84207D084F81B5333463A46022120465EF1BAFB3846BDE8F0812DE9F04104460D461646002794F81C03A84279
:40E5000007D084F81C5333463A46042120465EF1A5FB3846BDE8F0812DE9F04104460D461646002794F81D03A84207D084F81D5333463A46032120465EF190FB3846BDE8D2
:40E54000F0812DE9F04104460D461646002794F81603A84207D084F8165333463A46082120465EF17BFB3846BDE8F081014691F8180370472DE9F04104460D46164600278E
:40E5800094F81803A84207D084F8185333463A460B2120465EF162FB3846BDE8F0812DE9F04104460D461646002794F80A02A84207D084F80A5233463A460A2120465EF1D0
:40E5C0004DFB3846BDE8F08102460020D2F8F0310B600B6803B101207047F8B5044600252046FFF7C3FF002847D094F81A03012800D11EE0002617E06946304633F1A2FE62
:40E6000080B1009833F12AFF02280BD1009833F129FF0746394604F1300013F0CAFE08B1012505E0701CC6B233F189FEB042E3DC00BFD4F8F00140B1D4F8F001026800EE78
:40E64000105AB8EE400A91688847D4F8F40140B1D4F8F401026800EE105AB8EE400A9168884794F81903A84207D084F81953724B00220C2120465EF1F1FAF8BD70B504466A
:40E680000D46D4F8F00138B1D4F8F00120B1D4F8F001026851688847C4F8F0512046FFF79CFF70BD02460020D2F8F4310B600B6803B10120704770B504460D46D4F8F401BF
:40E6C00038B1D4F8F40120B1D4F8F401026851688847C4F8F4512046FFF77FFF70BD70B504460D46164684F81A532046FFF775FF70BD014691F819037047F8B5064600251F
:40E7000000240FE06946204633F11CFE40B100980068816C00988847012801D1681CC5B2601CC4B233F10BFEA042EBDC2846F8BDF8B507460D460026002414E069462046AD
:40E7400033F100FE68B100980068816C00988847012806D1009833F181FEA84201D1701CC6B2601CC4B233F1EAFDA042E6DC3046F8BD024600200A2902DA02F22323585CDE
:40E78000704770B50646002500240FE021463046FFF7EFFF10B1072802D100E000BF02E0681CC5B200BF00BF601CC4B20A2CEDDB284670BDF0B507460D460026002409E078
:40E7C00021463846FFF7D5FFA84201D1701CC6B2601CC4B20A2CF3DB3046F0BD70B506460025002412E021463046FFF7C2FF28B1052802D0072803D101E000BF00BF02E035
:40E80000681CC5B200BF00BF601CC4B20A2CEADB284670BD70B506460025002418E021463046FFF7A6FF58B1042807D0052806D0072807D105E000009B18170800BF00BF62
:40E8400000BF02E0681CC5B200BF00BF601CC4B20A2CE4DB284670BD014691F8EA0270472DE9F04104460D461646002794F8EA02A84207D084F8EA5233463A460D212046A4
:40E880005EF1ECF93846BDE8F08170B5044694F80C0203281DD12046FFF7DEFF4FF47A7110FB01F63146D4F89402D7F0CFFF08B100250FE02046FFF7CFFF0646D4F89402F2
:40E8C000D7F0B4FF4FF47A71B0FBF1F0301AC5B200E00025284670BD02460020D2F804320B600B6803B1012070472DE9F04781460E4617461C464FF00008002020600A2E6B
:40E900001CDA002515E02146284633F11BFD70B1206833F1A7FDB04207D1206833F19EFDB84202D14FF0010807E000202060681CC5B233F104FDA842E5DC00BF4046BDE8E3
:40E94000F087F8B505460E46144600276B46002231462846FFF7C9FF10B10098206001273846F8BDF8B505460E46144600276B46032231462846FFF7B8FF10B1009820609B
:40E9800001273846F8BDF8B505460E46144600276B46022231462846FFF7A7FF10B10098206001273846F8BDF8B505460E46144600276B46012231462846FFF796FF10B1D3
:40E9C0000098206001273846F8BDF8B505460E46144600276B46042231462846FFF785FF10B10098206001273846F8BDF8B505460E46144600276B46052231462846FFF7ED
:40EA000074FF10B10098206001273846F8BD70B506460C4615462946204633F193FC70BD2DE9F04782460E4617461C464FF00009C84600202060002517E02146284633F129
:40EA400081FC70B1206833F109FDB8420BD1464502D14FF001090CE008F1010000F0FF0801E000202060681CC5B233F168FCA842E3DC00BF4846BDE8F08770B506460C4613
:40EA80001546294620463CF188FF70BD2DE9F04782460E4617461C464FF00009C84600202060002519E0214628463CF176FF80B120683DF14CF8B8420DD1B04502D14FF088
:40EAC00001090EE00020206008F1010000F0FF0801E000202060681CC5B23CF15BFFA842E1DC00BF4846BDE8F0872DE9F04107460C46154600260020286031F136FBA04236
:40EB000004DD2946204631F133FB06463046BDE8F0812DE9F04107460C461546002600202860FCF7D1FDA04204DD29462046FCF7CEFD06463046BDE8F08110B502460B469B
:40EB40000020002108E002F21924645C9C4201D1441CE0B24C1CE1B20A29F4DB10BD2DE9F04105460E461446984600270A2C0FDA05F21920005DB0420BD005F219200655C6
:40EB800004F12F0143463A4628465EF167F800E007273846BDE8F08102460C200A2902DA02F22D23585C704710B502460B460020002108E002F22324645C9C4201D1441CA5
:40EBC000E0B24C1CE1B20A29F4DB10BD2DE9F04705460E4617461C46DDF820904FF000080A2C16DA05F22D20005DB84204D105F22320005DB0420ED005F22D2007550A3863
:40EC0000065504F139014B46424628465EF126F801E04FF007084046BDE8F08710B502460C23002007E002F22D24245C8C4200D10346441CE0B20A28F5DB184610BD70B551
:40EC40002DED028B0446B0EE408A0D46002694EDA20AB4EE480AF1EE10FA07D084EDA28A2B463246212120465DF1F8FF3046BDEC028B70BD70B52DED028B0446B0EE408A17
:40EC80000D46002694EDA30AB4EE480AF1EE10FA07D084EDA38A2B463246222120465DF1DDFF3046BDEC028B70BD014691F8EB0270472DE9F04104460D461646002794F85F
:40ECC000EB02A84207D084F8EB5233463A46252120465DF1C3FF3846BDE8F081014691F8EC0270472DE9F04104460D461646002794F8EC02A84207D084F8EC5233463A469A
:40ED0000262120465DF1AAFF3846BDE8F0810146D1F8A00270472DE9F04105460C46164600275CB1D5F8A002A04207D0C5F8A04233463A46172128465DF190FF3846BDE858
:40ED4000F081014691F8220370472DE9F04104460D461646002794F82203A84207D084F8225333463A46272120465DF177FF3846BDE8F081014691F8230370472DE9F041B9
:40ED800004460D461646002794F82303A84208D084F8235333463A4640F2255120465DF15DFF3846BDE8F081014691F8240370472DE9F04104460F461546002684F8247360
:40EDC0002B46324640F2EC4120465DF147FF3046BDE8F081024602F22530405C70472DE9F04105460C461646984600270C2C03DA05F22530065500E0072704F2ED414346A5
:40EE00003A4628465DF12AFF3846BDE8F081024602F23130405C70472DE9F04105460C461646984600270C2C03DA05F23130065500E0072704F2F94143463A4628465DF1D9
:40EE40000DFF3846BDE8F08130B504460B4600252046FFF7A9FF48B119462046FFF7BAFF20B10C2B02DA04F20D20C55C284630BD2DE9F04106460C461546984600270C2CDC
:40EE800005DA102D03DA06F20D20055500E0072704F2055143463A4630465DF1DFFE3846BDE8F08110B50346002093F821438C4201D083F8211310BD014691F80C02704775
:40EEC00070B52DED028B04462046FDF7A9FC05462846E0F072FB41EC180B9FEDF90B53EC102B65F1CDF90BD22046FDF7F7FE022806D12046FFF7E0FF032801D140F23D5568
:40EF00002846BDEC028B70BDF8B5064600250020009000243FE0002000902146EA48FDF701FE1B2834D2DFE800F0320E10110F1A1B1C301317181931141D15161E1F12206B
:40EF400021222523240000BF00BF00BF00BF00BF00BF00BF00BF00BF00BF00BF00BF00BF00BF00BF00BF00BF00BF00BF00BF00BF00BF00BF6A4621463046FDF7AFFD18B1C3
:40EF8000009833F10EFB054302E000BF00BF00BF00BF601CC4B23046FFF7AFFBA042BADC2846F8BD10B503464AF6DD441846FDF781FB0246042A05D0052A03D0092A01D035
:40EFC000032A01D141F63124204610BD014691F80802704710B5044631F1C7F810BDF8B507460D46002600240DE06946204631F1BFF830B1009831F1FDF8A84201D1701CBB
:40F00000C6B2601CC4B231F1B0F8A042EDDC3046F8BD10B5044633F192F910BDF8B507460D46002600240DE06946204633F18AF930B1009833F112FAA84201D1701CC6B292
:40F04000601CC4B233F17BF9A042EDDC3046F8BD10B504463CF19EFC10BDF8B507460D46002600240DE0694620463CF196FC30B100983CF16CFDA84201D1701CC6B2601CEA
:40F08000C4B23CF187FCA042EDDC3046F8BD0146D1F8C00270472DE9F04104460D4616460027D4F8C002A84207D0C4F8C05233463A461F2120465DF1D1FD3846BDE8F081F8
:40F0C0000146D1F8C40270472DE9F04104460D4616460027D4F8C402A84207D0C4F8C45233463A46202120465DF1B8FD3846BDE8F0810146D1F8B80270472DE9F0410446AE
:40F100000D4616460027D4F8B802A84207D0C4F8B85233463A461D2120465DF19FFD3846BDE8F0810146D1F8BC0270472DE9F04104460D4616460027D4F8BC02A84207D09A
:40F14000C4F8BC5233463A461E2120465DF186FD3846BDE8F0810146D1F8900270470146D1F8C80270472DE9F04104460D4616460027D4F8C802A84207D0C4F8C8523346CB
:40F180003A46112120465DF169FD3846BDE8F0810146D1F8CC0270472DE9F04104460D4616460027D4F8CC02A84207D0C4F8CC5233463A46122120465DF150FD3846BDE86E
:40F1C000F0810146D1F8D00270472DE9F04104460D4616460027D4F8D002A84207D0C4F8D05233463A46132120465DF137FD3846BDE8F081014691F83D0370472DE9F041AA
:40F2000004460D461646002794F83D03A84207D084F83D5333463A46142120465DF11EFD3846BDE8F081014691F83E0370472DE9F04104460D461646002794F83E03A8429E
:40F2400007D084F83E5333463A46152120465DF105FD3846BDE8F081F8B5064600250020009000240AE06B46062221463046FDF7E1F808B1681CC5B2601CC4B2052CF2DB2E
:40F280002846F8BDF8B50546002600200090002412E06B46062221462846FDF7CBF848B100980068D0F8801000988847012801D1012603E0601CC4B2052CEADB3046F8BD12
:40F2C0000000000000F06B40C80600100146D1F8F40270470146D1F8F80270470146D1F8FC0270470146D1F8000370470146D1F8040370470146D1F80803704700B50246EB
:40F3000041F288331046FDF7D5F9092801D143F69823184600BD034683F8421300207047014691F83F0370472DE9F04104460D461646002794F83F03A84208D084F83F53F7
:40F3400033463A4640F21D5120465DF187FC3846BDE8F081014691F8400370472DE9F04104460D461646002794F84003A84208D084F8405333463A4640F21E5120465DF10A
:40F380006DFC3846BDE8F08170B506460C460625032C00D1072529460C20CCF018F870BD014691F8410370472DE9F04104460D461646002794F84103A84208D084F84153CE
:40F3C00033463A4640F21F5120465DF147FC3846BDE8F0810146B1F80C0370470146B1F80E0370470146B1F8100370470146B1F8120370470146B1F81403704710B5044636
:40F4000004F5D270FBF7B1FC022801D1012010BD0020FCE72DE9F0410446002600270AE0394604F1300012F0C4FF0546B54200D92E46781CC7B20A2FF2DBFE4800688047BD
:40F440008046D4F8B412D7F020FAB4F8E8120844A4F8E80294F8420330BBF648006880478046D4F8B412D7F010FA02462046FDF7D7F9424300EE102AB8EE400A9FEDEE1AE6
:40F48000C0EE010A6420B6FBF0F000EE100AB8EE400A20EE800ABCEEC00A10EE100AD4F8B0120844C4F8B002E449D4F8B002884216D904F52B746068B0FBF1F021680844F5
:40F4C0002060DE496068B0FBF1F201FB12006060A4F52B74DA4B00221C2120465DF1BEFBB4F8E802B0F57A7F51DDB4F8E8024FF47A7190FBF1F0D4F8C0120844C4F8C0021E
:40F50000CF4B00221F2120465DF1A8FBB4F8E8024FF47A7190FBF1F0D4F8C4120844C4F8C402C74B0022202120465DF197FBB4F8E8024FF47A7190FBF1F0D4F8BC12084487
:40F54000C4F8BC02BE4B00221E2120465DF186FB9EB194F8420380B9B4F8E8024FF47A7190FBF1F0D4F8B8120844C4F8B802B44B00221D2120465DF171FBB4F8E8024FF439
:40F580007A7190FBF1F201FB1200A4F8E802A94800688047C4F8B402BDE8F0812DE9F04704464FF0000AD04618E0414604F1300013F04BFB70B1414604F1300013F0A3FB65
:40F5C00028B1414604F1300013F0D8FB10B14FF0010A06E008F1010000F0FF08B8F1060FE3DBBAF1000F07D02046FDF777FB18B12046FFF789FC08B9012000E0002007461C
:40F600002046FFF759FC032801D1012000E00020814617B9B9F1000F09D0864800688047C4F8DC02834800688047C4F8D4022046FFF746FC0546002694F84103F8B92046B9
:40F64000FDF74CF8A8421BD92046FEF7AEFEB8B12046FFF753FE80464146D4F8D402D7F0F5F838B142F21071D4F8DC02D7F0EEF800B101266F4800688047C4F8D8021EE06D
:40F680006C4800688047C4F8D4022046FFF78AFCA84204D3674800688047C4F8D8022046FFF780FCA8420AD22046FFF727FE80464146D4F8D802D7F0C9F800B1022694F8BF
:40F6C000080210B99FB1002611E067B9B9F1000F01D0022E07D1022E07D000212046FDF721FA0F2801D1002601E094F8086294F80802B04207D084F80862514B00221B213C
:40F7000020465DF1ABFABDE8F08770B504464D4800688047012805D1012202212046FDF709FA08E094F80C02012804D1012200212046FDF7FFF92046FFF748FC60B9424826
:40F74000FCF7CCFF05462046FFF7BAFB85420FD92046FEF72AFE58B100212046FDF7E2F90F280ED0022211462046FDF7E3F908E094F80C02022804D1022200212046FDF7F8
:40F78000D9F92046FFF722FC022814D12046FFF797FB05462046FFF705FC85420BD300212046FDF7BFF90F2805D0042202212046FDF7C0F908E094F80C02042804D104226F
:40F7C00000212046FDF7B6F92046FCF78BFF28B1062201212046FDF7ADF908E094F80C02062804D1062200212046FDF7A3F994F80C02032833D12046FFF72EF84FF47A719C
:40F8000010FB01F52946D4F89402D7F01FF840B92046FDF763FA20B104F1300013F0A8F8B8B9074A002104F5D270FBF76FFB032200210BE018A0100800007A4440420F0005
:40F840009B181708B0000020C80600102046FDF771F9FD4B00220E2120465DF1FFF970BD2DE9F8438046002500240BE0694620461AF059FA20B1F44AFF2100981AF0C1FF84
:40F88000601CC4B21AF04CFAA042EFDC00241CE021464046FEF7C5FC002358405940084311D021464046FEF7BCFC06466A461AF083FA28B1E44A294600981AF0A2FF00E060
:40F8C00005E0681CC5B2601CC4B20A2CE0DB00BFBDE8F88338B50446002000906946DB481CF03AFFB0B1009800680169009888474FF47A71B0FBF1F085B2B4F80C03A842A0
:40F9000008D0A4F80C53D04B00224FF4A46120465DF1A4F96946CD481CF0FEFEB0B1009800680169009888474FF47A71B0FBF1F085B2B4F80E03A84208D0A4F80E53C24BA6
:40F94000002240F2215120465DF188F96946BF481CF0EAFEB0B1009800680169009888474FF47A71B0FBF1F085B2B4F81003A84208D0A4F81053B44B002240F22251204613
:40F980005DF16CF96946B1481CF0D6FEB0B1009800680169009888474FF47A71B0FBF1F085B2B4F81203A84208D0A4F81253A64B002240F2235120465DF150F96946A34815
:40F9C0001CF0C2FEB0B1009800680169009888474FF47A71B0FBF1F085B2B4F81403A84208D0A4F81453984B002240F2245120465DF134F938BD2DE9F84F04469448006823
:40FA000080478346934800688047DFED930A20EE200ABDEEC00A10EE105A904800688047DFED8D0A20EE200ABDEEC00A10EE106A8B4800688047DFED880A20EE200ABDEEDC
:40FA4000C00A10EE107A874800688047DFED820A20EE200ABDEEC00A10EE108A824800688047DFED7D0A20EE200ABDEEC00A10EE109A7E4800688047DFED770A20EE200A7E
:40FA8000BDEEC00A10EE10AA00200090D4F8F002584507D0C4F8F0B26B4B0022282120465DF1DCF8D4F8F402A84215D044F25060854203DD05460220009005E06C488542B5
:40FAC00002DA054603200090C4F8F4525E4B29212046009A5DF1C2F800200090D4F80003B04215D0B6F5FA5F04DD4FF4FA560220009005E016F5FA5F02DA5E4E032000902B
:40FB0000C4F80063504B2A212046009A5DF1A6F800200090D4F8F802B84215D044F25060874203DD07460220009005E05048874202DA074603200090C4F8F872424B2B21D0
:40FB40002046009A5DF18AF800200090D4F80403404516D0B8F5FA5F04DD4FF4FA580220009006E018F5FA5F03DADFF8088103200090C4F80483344B2C212046009A5DF100
:40FB80006DF800200090D4F8FC02484515D044F25060814503DD81460220009005E03448814502DA814603200090C4F8FC92264B2D212046009A5DF151F800200090D4F856
:40FBC0000803504516D0BAF5FA5F04DD4FF4FA5A0220009006E01AF5FA5F03DADFF894A003200090C4F808A3174B2E212046009A5DF134F8BDE8F88F38B504462046FFF713
:40FC000084FD2046FFF7CAFC2046FFF703FC2046FEF7F1FB2046FEF7E0FC2046FDF742F904F5D270FBF734FB2046FFF7E4FE2046FFF750FE69462046FEF708F910B100980B
:40FC400034F1FDFB38BD00009B181708CC18001044060010480600100000C8424C06001050060010540600105C06001060060010B0B9FFFFC0E0FFFF10B50448FDF7EDFADF
:40FC80000446034A0349DCF0D4FF10BDC8060010008000082FD3000810B50446204632F162FB002004F58874E07001202071FE4800688047A0600020E060FB480068804732
:40FCC0006061F94800688047A0610020E06120629FEDF60A84ED130A9FEDF40A84ED150A6062A062E06220639FEDF00A84ED0D0A9FEDEE0A84ED0F0A84F84000B7EE000AAB
:40FD000084ED140A9FEDE90A84ED110A9FEDE70A84ED120A84F8580084F859002066E0656066A066E06684F8700060670021A167E167C4F88000C4F88400A4F5887404F56B
:40FD4000C0708161C161016241622821283061F12BFB142104F5E87061F104FB002004F5F27420602071A071E0712072E06084F83400A4F5F274042084F819022068CC4A8D
:40FD800000210369204698479FEDC80A04F50E7404ED040A002044F80C0C20746074A074E07420756075A07520836083207760770220A077A4F50E74204632F148FB0C288E
:40FDC00009D0204632F143FB102804D0204632F13EFB1A2801D1012000E0002004F2572420700A2060700020A070E070207120726072A072E071A4F2572400BF05E00022B6
:40FE000004F517710A54411CC8B20228F7DB002004F51974607120602071A0719FEDA30A84ED020A9FEDA10A84ED030A9FED9F0A84ED040A9FED9D0A84ED050AA061E06163
:40FE40002062A4F5197410BDF8B504460F4615461E462B46022239462046009632F1D8F904469448F43444F8F40C00F58E7044F8E80C103044F8E40C002044F8080C44F839
:40FE8000040C20606060A060E0602061606120766076A076E07620776077A077C4F83C01C4F84001C4F84401C4F84801C4F84C01C4F85001F43C00BF06E00021D4F8F4202B
:40FEC00042F82010411CC8B20228F6DB002006E00021D4F8002142F82010411CC8B20128F6DB2046FFF7D8FE23462A46724920465CF13FFE2046F8BD70B504466D48206002
:40FF000000F58E70E06010302061002513E0D4F8F00050F8250068B1D4F8F00050F8250040B1D4F8F02052F8250052F825201268516888476D1C94F80C01A842E7D800258D
:40FF400013E0D4F8F40050F8250068B1D4F8F40050F8250040B1D4F8F42052F8250052F825201268516888476D1C94F80E01A842E7D8002513E0D4F8F80050F8250068B11B
:40FF8000D4F8F80050F8250040B1D4F8F82052F8250052F825201268516888476D1C94F80D01A842E7D800250BE0D4F8FC0038B1D4F8FC0020B1D4F8FC000268516888475B
:40FFC0006D1C94F80F01A842EFD8D4F8EC0038B1D4F8EC0020B1D4F8EC00026851688847002513E0D4F8080150F8250068B1D4F8080150F8250040B1D4F8082152F825004D
:020000040801F1
:4000000052F825201268516888476D1C94F81001A842E7D8002513E0D4F8000150F8250068B1D4F8000150F8250040B1D4F8002152F8250052F825201268516888476D1C54
:4000400094F81101A842E7D8002513E0D4F8040150F8250068B1D4F8040150F8250040B1D4F8042152F8250052F825201268516888476D1C94F81201A842E7D8D4F8F0001D
:4000800018B1D4F8F00061F149FDD4F8F40018B1D4F8F40061F142FDD4F8F80018B1D4F8F80061F13BFD09E018A0100800000000F718170828A71008CD311408D4F80001B9
:4000C00018B1D4F8000161F129FDD4F8080118B1D4F8080161F122FDD4F8300218B1D4F8300261F11BFDD4F8340218B1D4F8340261F114FDD4F8380218B1D4F8380261F188
:400100000DFDD4F83C0218B1D4F83C0261F106FDD4F8400218B1D4F8400261F1FFFCD4F8440218B1D4F8440261F1F8FCD4F8040118B1D4F8040161F1F1FC204632F1A4F84F
:400140000446204670BD70B504462046FFF7D4FE054661F1E7FC70BD10B50446103C2046FFF7F1FF10BD10B504460C3C2046FFF7EAFF10BD10B50446103C2046FFF7BCFE0A
:4001800010BD10B504460C3C2046FFF7B5FE10BD70B50546012406E0F84B0022214628465CF15CFD641C7D2CF6D38F2406E0F34B0022214628465CF151FD641CB4F5A07F41
:4001C000F5D370BD70B504460D461646002D7CD120683246036F20469847206832460021836F2046984794F8190205286ED2DFE800F0512A037B7C0020683146B0EE080A74
:40020000D0F8802020469047206831469FEDDC0AD0F8A8202046904720683146B0EE080AD0F8A02020469047206831461FED610AD0F8B02020469047206832462946436901
:400240002046984779E020683146B0EE080AD0F8802020469047206831469FEDC90AD0F8A8202046904720683146B0EE080AD0F8A02020469047206831461FED740AD0F89C
:40028000B0202046904720683246294643692046984752E020683146B0EE080AD0F8802020469047206831469FEDB50AD0F8A82020469047206831469FEDB20AD0F8A02065
:4002C000204690472068314601E03EE034E01FED890AD0F8B0202046904720683246294643692046984728E000BF20683146B0EE000AD0F8802020469047206831469FED3D
:40030000A00AD0F8A8202046904720683146B7EE000AD0F8A02020469047206831461FED9D0AD0F8B0202046904720683246294643692046984700E000BF00BF8F4B002292
:400340004FF6FF7120465CF189FC70BD70B504460D461646002D74D1002084F8180294F8190205286ED2DFE800F06E3703A2A300206831469FED840AD0F88820204690479F
:40038000206832460021B2EE0E0AD0F89030204698472068324601219FED7B0AD0F89030204698472068324602211FEDC00AD0F8903020469847206832460321B2EE040AFF
:4003C000D0F8903020469847206832460021D0F8B83020469847A0E0206831469FED6A0AD0F8882020469047206832460021B2EE0E0AD0F890302046984720683246012126
:400400009FED610AD0F89030204698472068324602211FEDDA0AD0F8903020469847206832460321B2EE040AD0F8903020469847206832464FF4C871D0F8B8302046984708
:400440006BE072E068E0206831469FED4F0AD0F88820204690472068324600219FED4A0AD0F8903020469847206832460121B3EE040AD0F890302046984720683246022177
:400480009FED410AD0F8903020469847206832460321B1EE040AD0F8903020469847206832460021D0F8B8302046984735E000BF206831469FED340AD0F88820204690479A
:4004C0002068324600219FED300AD0F8903020469847206832460121B2EE040AD0F89030204698472068324602219FED280AD0F89030204698472068324603219FED240A1F
:40050000D0F8903020469847206832460021D0F8B8302046984700E000BF00BF174B00224FF6FF7120465CF199FB70BD70B504460E46002507E0206832462946436920467D
:400540009847681CC5B22068C16920468847A842F1DC70BD10B50346002093F80C418C420ADDD3F8F04054F821402CB1D3F8F04054F821401460012010BD0000F71817085E
:400580000000C84200000C420000484200000000CDCCCC3E014691F80C0170472DE9F04105460E460027002410E0D5F8F00050F8240048B1D5F8F01051F824002FF11AFE6D
:4005C000B04201D1781CC7B2601CC4B2102CECDB3846BDE8F08130B504460020052A1AD004DC012A07D0042A46D120E0062A2ED00A2A41D13BE094F80D518D420ADDD4F817
:40060000F85055F821502DB1D4F8F85055F821501D60012031E094F80F518D4206DDD4F8FC501DB1D4F8FC501D60012025E094F80E518D420ADDD4F8F45055F821502DB1C9
:40064000D4F8F45055F821501D60012015E094F811518D420ADDD4F8005155F821502DB1D4F8005155F821501D60012005E0D4F8EC501D60012000BF00BF00BF30BD30B5A9
:400680000446002000251D607AB994F80D518D420ADDD4F8F85055F821502DB1D4F8F85055F821501D60012000E000BF00BF30BD02460020012906D0042907D0052908D07E
:4006C00006290CD108E092F80D0109E092F80E0106E092F80F0103E092F8110100E000BF00BF70472DE9F84304460D4690461E46089F4FF00009B8F1010F09D0B8F1040F73
:4007000038D0B8F1050F1ED0B8F10A0F60D14CE094F80D01A84215DDD4F8F80050F8250080B1D4F8F81051F8250069463BF1FAF940B10098F8F74BFCB04203D1009838604A
:400740004FF0010945E094F80F01A84211DDD4F8FC0070B16946D4F8FC003BF1E3F940B10098F8F734FCB04203D1009838604FF001092EE094F80E01A84215DDD4F8F40003
:4007800050F8250080B1D4F8F41051F8250069463BF1C8F940B10098F8F719FCB04203D1009838604FF0010913E0D4F8EC0070B16946D4F8EC003BF1B5F940B10098F8F770
:4007C00006FCB04203D1009838604FF0010900BF00BF00BF4846BDE8F8832DE9F84304460D4616461F464FF00008CEB994F80D01A84214DDD4F8F80050F8250078B1D4F8B5
:40080000F81051F8250069463BF18CF938B10098F8F7DDFB18B9009838604FF0010800E000BF00BF4046BDE8F88330B504460020012A0AD194F810518D4205DDD4F8085135
:4008400055F821501D60012000E000BF00BF30BD014691F81001704702460020012902D192F8100100E000BF00BF704710B5034600200024146093F812418C4207DDD3F803
:40088000044154F821401460146804B1012010BD2DE9F04104460D460026002D5DD094F80C01102859DA04F5867204F1F0012846DDF0B1FD002850D0D4ED870AB0EE600AE9
:4008C0002068FD49D0F8A02020469047D4ED880AB0EE600A2068F849D0F8A8202046904794F819122068F44AD0F8983020469847D4ED800AB0EE600A2068EF49D0F888209F
:4009000020469047D4ED890AB0EE600A2068EA49D0F8B02020469047D4F814122068E64AD0F8B8302046984794F80C01401EC1B228462FF174FC204631F194FD07463946A2
:4009400028462FF15FFC94F80C01401E82B22346DA4928465CF10DF90126012E05D1D64B0022532120465CF179F93046BDE8F081014691F85E027047014691F856027047BC
:40098000014691F85F0270472DE9F05F06460C461F46DDF828904D460C2E13D00D2E09D00E2E3BD104F1FB013B46002228465CF155F933E004F1F9013B46002228465CF151
:4009C0004DF92BE0012C28D12846FFF7D9FF20B32846FFF7CDFF00281FDD284632F127F900281AD92846FFF7C7FF042815D0A8462846FFF7BDFF8346284632F118F90BFB97
:400A000000FB6420BBFBF0FAD8F800003A465146D0F8EC304046984700BF00BF00BFBDE8F09F2DE9F0412DED028B04460D464FF00008002D7ED028463BF189F805287AD017
:400A400004DC012807D0042876D1B4E0062874D00A28F9D1D3E094F80D0110286EDA04F20D1204F1F801284662F1B6FB8046002615E0D4F8F80050F8260078B1D4F8F800DF
:400A800050F826702068816E20468847B0EE408A3868894982693846904700BF761C94F80D01B042E5D8D4F8300218B1D4F8300261F134F8D4F8340218B1D4F8340261F196
:400AC0002DF8D4F8380218B1D4F8380261F126F8D4F83C0218B1D4F83C0261F11FF8D4F8400218B1D4F8400261F118F8D4F8440218B1D4F8440261F111F804F20D14217807
:400B00008800DCF0BBFCC4F8230121788800DCF0B5FCC4F8270121788800DCF0AFFCC4F82B0121788800DCF0A9FCC4F82F012178880004E06AE031E066E053E02DE0DCF098
:400B40009DFCC4F8330121788800DCF097FCC4F83701A4F20D1400201BE00021D4F8302242F82010D4F8342242F82010D4F8382242F82010D4F83C2242F82010D4F840221F
:400B8000216C42F820100021D4F8442242F82010401C94F80D118142DFD836E094F80F01012807DAFC34E07C401CE07444F8FC594FF0010829E094F80E01022811DA04F57E
:400BC000877204F1F401284662F106FB804694F80E01401E82B22346AFF2532128465BF1C8FF12E094F81101012807DA04F2111204F58071284662F1EFFA804605E0C4F8B0
:400C0000EC504FF0010800E000BF00BF4046BDEC028BBDE8F08170B504460D460026002D47D094F81001102843DA04F5887204F58471284662F100FB00283AD02846F8F7B6
:400C400045F9A8BBD4ED810AB0EE600A20681A4A0021D0F8903020469847D4ED820AB0EE600A2068144A0121D0F8903020469847D4ED830AB0EE600A20680F4A0221D0F859
:400C8000903020469847D4ED840AB0EE600A2068094A0321D0F8903020469847D4ED7F0AB0EE600A20680449D0F88020204690470126304670BD0000F718170853311408A8
:400CC0002DE9F04704460D4616461F46DDF82080C146062C17D2DFE804F01614130B150305F59A713B46324648465BF1B7FF0AE005F59C713B46324648465BF1AFFF02E0B5
:400D000000BF00BF00BF00BFBDE8F08770B504460D4600269DB194F8120104280FDA94F812212346AFF2670128465BF122FF04F5897204F582712846DDF0FDFB06463046D0
:400D400070BD2DE9F0412DED028B04469FEDFE0AB0EE408A9FEDFD0AF0EE408A0027FF262068D0F8941020468847032806D02068D0F8941020468847042840D1002530E0C6
:400D8000D4F8F01051F825002FF155FB38B3D4F8F01051F825002FF183FAB4EEE80AF1EE10FA08DBD4F8F01051F825002FF178FAF0EE408A2E46D4F8F01051F825002FF125
:400DC0006FFAB4EEC80AF1EE10FA08D2D4F8F01051F825002FF164FAB0EE408A2F46681CC5B294F80C01A842CADCFF2E07D194F80C01002803DD94F80C01401EC6B294F8F9
:400E00004A02B84208D084F84A72D14B002240F2091120465BF122FF94F84B02B04208D084F84B62CA4B00224FF4857120465BF115FFBDEC028BBDE8F0812DE9FC5F0446F6
:400E40000D460027204631F10DFB0646A16901F13000314611F0E3FC8046A16901F13000414611F0CDFB8146BA460020019020680121C26A20469047834620680121C26A2D
:400E800020469047A84227DD204631F1E0FA0C2801D14FF0010B05FB09F090FBFBF000F0FF0A99FBFBF05044C0B20190564610E000200090A16901F130006B4642463146BE
:400EC00011F062FC18B1009835F150FF0744701CC6B201988642EBDB3846BDE8FC9F2DE9F04704464FF0FF384FF000090027FF2600251DE029462046FFF79FFF002815D947
:400F0000D4F8440250F82500484504D3D4F8440250F825902E46D4F8440250F82500404504D2D4F8440250F825802F46681CC5B294F80D01A842DDDCFF2E07D194F80D0126
:400F4000002803DD94F80D01401EC6B294F84802B84208D084F848727D4B00224FF4867120465BF17BFE94F84902B04208D084F84962774B002240F20D1120465BF16EFEB2
:400F8000BDE8F08702460020022903DA02F5CC7353F82100704770B50546002428E034B1012C05D0022C11D0032C1ED10FE000BF00212846FFF7E6FF86B2D5F8041151F821
:400FC0002400634A3146F9F73EFB0EE000BF01212846FFF7D7FF86B2D5F8041151F824005B4A3146F9F72FFB00BF00BF601CC4B295F81201A042D2DC70BD014691F86102BA
:40100000704730B503460020022909DA052A07DA01EB810503F5E87404EB450434F8120030BD70B52DED028B82B006460C46B0EE408A154624B1012C1BD0022C41D131E0C7
:4010400001AA00213046FFF711FC28B12946B0EE480A0198F9F754FA01AA01213046FFF705FC28B12946B0EE480A0198F9F748FA27E001AA02213046FFF7F8FB28B1294663
:40108000B0EE480A0198F9F73BFA01AA03213046FFF7ECFB28B12946B0EE480A0198F9F72FFA0EE02A46B0EE480A00213046FFF7B8FF2A46B0EE480A01213046FFF7B1FF46
:4010C00000BF00BF002002B0BDEC028B70BD02460020022903DA02F5D07353F82100704730B503460020022909DA052A07DA01EB810503F5D47404EB850454F8220030BD7F
:401100000246002092F80D318B4203DDD2F83C3253F8210070472DE9F04F2DED088B85B00446204631F19EF900287DD194F8DB0000287AD02046FFF760FF0028F9D0204676
:4011400031F190F9054605E000007A4400000000F7181708A16901F13000294611F029F90028E6D04FF0000A1FE12046FFF745FF002871D00026B146204631F112FA98B1C0
:40118000204630F171FF01280ED1002506E029462046FFF7B5FF0644681CC5B22068C16920468847A842F2DC04AA0121A069FDF7EAFBC0B1049831F1F4F9A0B1049830F1E6
:4011C00053FF01280FD1002506E029460498FFF797FF0644681CC5B204980068C16904988847A842F1DC002511E0A16901F1300003AA29460FF061FF38B1039835F166FE92
:4012000018B109F1010000F0FF09681CC5B2A16901F130000FF04DFFA842E6DCA16901F130000FF046FF01E015E1E6E0484511D0B9F1000F0EDDA16901F130000FF039FF52
:40124000002807DDA16901F130000FF032FF7043B0FBF9F600279DE0A3E03A4651462046FFF73EFF0546042F1CD1042251462046FFF736FFB0B1042251462046FFF7C1FEF0
:4012800000EE100AB8EE400ADFEDF70A80EE201AB0EE418AF54AB0EE480A51462046FFF7C0FE75E0781CC2B251462046FFF718FF8046A8EB0500DEF080F941EC190B514684
:4012C0002046FFF704FF40080190DEF076F941EC1B0B9FEDE70B53EC102BDDF07DFF41EC1A0B53EC192BDEF07BF941EC180BDEF037F98346A8EB050005EB5000A0EB0B0049
:401300000390A8EB050005EB5000584402900398A84200D803950298404501D3CDF808800398864216D83A4651462046FFF769FE00EE100AB8EE400ADFEDCB0A80EE201A73
:40134000B0EE418AC94AB0EE480A51462046FFF768FE22E00298864219D9464517D2781CC2B251462046FFF74CFE00EE100AB8EE400ADFEDBD0A80EE201AB0EE418ABB4AF8
:40138000B0EE480A51462046FFF74BFE05E000BF781CC7B2052FFFF660AF2046FFF7FBFD00BF0AF1010000F0FF0ABAF1020FFFF6DCAE00251CE02046FFF71FFE40B1D4F87E
:4013C000041151F82500A94A0021F9F712F907E0D4F8041151F82500A44A0121F9F709F9D4F8041151F82500F9F76EF9681CC5B294F81201A842DEDC3DE094F8DB00A0B16A
:401400002046FFF7FAFD80B1002509E0D4F8041151F82500954A0021F9F7A4F8681CC5B294F81201A842F1DC25E02046FFF7E5FD08BB2046FFF7AFFD002507E0D4F80411F3
:4014400051F82500F9F740F9681CC5B294F81201A842F3DC0FE0002509E0D4F8041151F82500824A0021F9F77DF8681CC5B294F81201A842F1DC05B0BDEC088BBDE8F08F7E
:4014800070B52DED028B04461FEDD00AB0EE408A1FEDD20AF0EE408A2068D0F8941020468847032806D02068D0F8941020468847042827D1002518E0D4F8F01051F825006A
:4014C0002EF1B9FF78B1D4F8F01051F825002EF1E7FE30EE080AB0EE408AB7EE000A38EE800AF0EE408A681CC5B294F80C01A842E2DCF5EEC08AF1EE10FA03DD88EE280A35
:40150000B0EE408A94ED8A0AB4EE480AF1EE10FA08D084ED8A8A554B00224FF4847120465BF19CFBBDEC028B70BD70B52DED028B04461FEDFA0AB0EE408A1FEDFC0AF0EED0
:40154000408A002519E029462046FFF776FC002811D9D4F8440250F8250000EE100AB8EE400A30EE080AB0EE408AB7EE000A38EE800AF0EE408A681CC5B294F80D01A8429F
:40158000E1DCF5EEC08AF1EE10FA03DD88EE280AB0EE408ABCEEC80A10EE100AD4F82C1281420AD0BCEEC80A84ED8B0A2F4B002240F20B1120465BF151FBBDEC028B70BD60
:4015C000F8B504460E460020009000250EE020686A462946836920469847012804D1234A314600982EF12BFF681CC5B294F80C01A842ECDCF8BD2DE9F04104460E46154607
:40160000002794F80C01A8420DDDD4F8F00050F8250040B1D4F8F01051F82500134A31462EF12BFE01273846BDE8F08170B52DED028B04460E46002529E0D4F8F00050F84E
:40164000250010B3C6B1D4F8F01051F825002EF127FEB0EE408AD4F8F01051F8250003492EF124FE11E000000000C842F7181708000000000088C340D4F8F01051F8250070
:4016800000219FEDF70A2EF111FE681CC5B294F80C01A842D1DCBDEC028B70BD0146D1F8840270472DE9F04104460D461646002794F86A02A84208D084F86A5233463A4621
:4016C00040F23D1120465BF1C9FA3846BDE8F081014691F8680270470146D1F8640270472DE9F04104460D461646002794F85602A84207D084F8565233463A46B8212046DB
:401700005BF1ACFA3846BDE8F0810246002092F80D318B4203DDD2F8343253F8210070472DE9F0472DED028B04468846914600272068C16C20468847002871D0D4ED131AA8
:40174000F8EE611AB0EE611AD4ED101AF8EE611AF0EE610A94F8390001EE900AF8EE611AB0EE610A31F1C2FB07462FB1226CE06C904201D9012000E0002001462068B94A1D
:40178000D0F8F430204698472FB1226CE06C904201D2012000E0002001462068B14AD0F8F03020469847002572E029462046FFF744FB00285AD029462046FFF7A6FF00EE50
:4017C000100AB8EE400AB0EE408A20682946D0F8FC202046904700EE100AB8EE400AF0EE408A94F8390000EE900AF8EE600AB0EE600AB0EE481AF0EE680A31F177FB0746E9
:401800007FB129462046FFF780FF824620682946D0F8FC2020469047824502D9012001E03EE00020064620688E4B2A463146D0F810C12046E04777B129462046FFF765FF5B
:40184000824620682946D0F8FC2020469047824501D2012000E0002006462068814B2A463146D0F80CC12046E0470FE020687D4B2A460021D0F810612046B0472068794B72
:401880002A460021D0F80C612046B047681CC5B220680121C26A20469047A84285DC28E02068704A0021D0F8F4302046984720686C4A0021D0F8F03020469847002511E06E
:4018C0002068684B2A460021D0F810612046B0472068644B2A460021D0F80C612046B047681CC5B220680121C26A20469047A842E6DC94F8570200287DD0B8F1000F7AD016
:4019000094F8DC00012803D094F8DC00002872D12068D0F8E8102046884700286BD1204630F195FD0C2826D1D4F8E411D4F8B800884220D154F8F82F506822685268126862
:40194000516A8847B0EE408A226810680268516A8847F0EE408A94F86001F83C00EE900AF8EE600AB0EE600AB0EE481AF0EE680A31F1BCFAE0BB204630F169FD10283AD1E3
:4019800000212046FFF759FAA0B301212046FFF754FA78B300212046FFF7B7FE054601212046FFF7B2FE854225D001212046FFF7ACFE00EE100AB8EE400AB0EE408A0021FD
:4019C0002046FFF7A2FE00EE100AB8EE400AF0EE408A94F8580200EE900AF8EE600AB0EE600AB0EE481AF0EE680A31F17FFA08B1012001E0FFE7002084F8590200260FE0ED
:401A0000D4F8F40050F8260040B1D4F8F42052F8260052F826201268916A8847701CC6B294F80E01B042EBDC022594F85402012852D194F80E0100284EDD94F80E01012804
:401A400017DBD4F8F4100868F9F7E1FF30B1012802D004280AD107E0002509E0012507E000000000F7181708022501E0032500BF00BF94F80E0102282ED1D4F8F41048685F
:401A8000F9F7C5FF70B1012802D004281FD118E0012D01D0002504E02046FEF771FF00B1042518E02046FEF76BFF40B1D4F8F4100868F9F7ACFF012801D1002500E00125E6
:401AC00009E0032D01D0022D00D1022503E0032D00D100BF00BF00BFD4F8B80018B1012D01D1012000E0002084F85502002229462046FFF7F5FD94F80F01002805DD4B465D
:401B00000022232120465BF1A9F894F85A0238B3D4F8FC0018B9012084F85B0223E0D4F8F81008683AF16BF818B1002084F85B0219E020680021426D2046904700280BD955
:401B4000D4F8FC000268116A8847B5EEC00AF1EE10FA01D1012000E0002084F85B0202E0002084F85B02204631F162F9E16B884203D8012084F8D80002E0002084F8D8004D
:401B80001FED490AB0EE408A94F86902012830D120680621C26A2046904750B3D4F80011086812F0D5FD20B3D4F8B80010B3D4F8BC00F8B9204631F1FDF800EE100AB8EE83
:401BC000400A84ED9D0A1FED5A0A84ED9E0A2046FFF764FD00EE100AB8EEC00A84ED9B0A1FED610A84ED9C0AFA4A00212046FFF759FD77E0D4F8B800E8B32046FFF74EFDED
:401C000000EE900AF8EEE00A94ED9B1A30EEC10AF0EEC00AC4ED9C0A204631F1CBF800EE100AB8EE400AD4ED9D0A30EE600A84ED9E0A94ED9C0AB5EEC00AF1EE10FA16D07F
:401C400094ED9E0AB5EEC00AF1EE10FA0FD094ED9E0AD4ED9C0A70EE600A94ED9E1A80EE810ADFEDDD0A20EE200AB0EE408A2046FFF732FD00E035E000EE100AB8EE400AB1
:401C8000D4ED9E0AB4EEE00AF1EE10FA2AD82046FFF71EFD00EE100AB8EE400AB4EEC80AF1EE10FA04D2CB4A01212046FFF7FAFC204631F17FF800EE100AB8EE400A84EDB1
:401CC0009D0A1FED990A84ED9E0A2046FFF7E6FC00EE100AB8EEC00A84ED9B0A1FEDA00A84ED9C0ABDEC028BBDE8F0872DE9F04104460D4616460027D4F87401A84208D020
:401D0000C4F8745133463A4640F2031120465AF1A5FF3846BDE8F0812DE9F04104460D4616460027D4F87801A84208D0C4F8785133463A464FF4827120465AF18FFF38461B
:401D4000BDE8F0810146D1F8740170470146D1F83001704770B52DED028B04460D461FEDC00AB0EE408A94F80D01A8423CDDD4F82C01002838D9D4F8300250F82500002810
:401D800032D9A069FAF796FC062802D0072815D100BFD4F8300250F8250000EE100AF8EE400A94ED4D0AB8EE401A81EE200ADFED8B0A20EE200AB0EE408A14E0D4F83002B1
:401DC00050F8250000EE100AB8EE400ADFED820A60EE200A94ED4B0AB8EE400A80EE801AB0EE418A00BF00BFB0EE480ABDEC028B70BD0246002092F80D318B4203DDD2F8FF
:401E0000303253F8210070472DE9F0472DED028B04460E4615461F464FF0000894F80D01A84228DD29462046FFF7E3FFB04222D0D4F8300240F8256005F17E013B46424631
:401E400020465AF10BFFD4F8F80050F8259029462046FFF77FFFB0EE408AD9F800003946826948469047D4F8E80018B1D4F8E8002FF1B0FC00BF4046BDEC028BBDE8F08701
:401E8000014691F84C0270472DE9F04704460D4617464FF000082046FFF758FFA84207D0C4F830513B464246902120465AF1D6FE2046FFF7E5FF88B900260BE02046FFF7E1
:401EC00045FF81463B46324649462046FFF79CFF701CC6B294F80D01B042EFDC4046BDE8F0870146D1F8340170472DE9F0472DED028B04460E4617464FF000082046FFF7CD
:401F0000F0FFB0422CD0C4F834613B464246912120465AF1A3FE002517E0D4F8F80050F8250080B1D4F8F80050F8259029462046FFF710FFB0EE408AD9F8000039468269AA
:401F40004846904700BF681CC5B294F80D01A842E3DCD4F8E80018B1D4F8E8002FF13AFC4046BDEC028BBDE8F087014691F8800170470146D1F87C01704770B504460025C0
:401F80002FF0C5FF062811D02FF0C1FF07280DD020680621C26A20469047C8B1D4F8002110680268916F8847032811D194F8690101280DD12046FFF7DCFF48B12046FFF77F
:401FC000D4FF28B1204630F133FF002800D90125284670BDF71817080000C84200401C4670B52DED048B04460D462046FFF7C5FF002826D020680621C26A2046904708B364
:40200000D4F8002110680268916F8847032819D1204630F10DFF02462046FFF7AAFF400082420FD80021C4F88811C4F88C110020C4F88401204630F1FBFE002104F5C8721E
:4020400003C20AE100210846D4F890315940D4F894215040014306D1204630F1E9FE002104F5C87203C2D4F884012844C4F88401204630F1DDFE0146D4F89031D4F89401D3
:40208000591A60F10000C4F88811C4F88C012046FFF76FFFD4F88831D4F88C11181A71F10001CEDBA069FAF705FB052804D0A069FAF700FB082860D120680621C26A204636
:4020C0009047E0B3D4F8002110680268916F8847032852D19FEDF90AB0EE409AD4F8300290ED000AB8EE400ADFEDF40A80EE201AB0EE418AD4F888211046D4F88C1162F1AC
:4021000004F900EE100A60EE080A6421D4F82C01B0FBF1F000EE100AB8EE401A94ED610AB8EE400A60EE081A81EE810A80EE801AF0EE418AB0EE000A28EE000A00E01CE08D
:40214000B4EEE80AF1EE10FA05D2B0EE000A28EE000AF0EE408AF5EEC08AF1EE10FA0BDD9FEDD60A28EE800ABCEEC00A10EE101AD34A2046FFF788FE60E0D4F888211046EB
:40218000D4F88C1162F1C1F800EE100AD4F83002D0ED000AF8EE600AF2EE041A80EEA11AD4ED610AF8EE601AC1EE810A80EE201AB0EE418A2046FFF794FE00EE100AB8EEF3
:4021C000400A2046FFF78DFE00EE900AF8EE600A38EE601A2046FFF7C8FE00EE900AF8EE601A1FED832AC1EE820A01EE200AB0EE408A2046FFF775FE400000EE100AB8EEFA
:40220000400AB4EEC80AF1EE10FA09D22046FFF768FE400000EE100AB8EE400AB0EE408AB5EEC08AF1EE10FA07DDA54ABCEEC80A10EE101A2046FFF758FE00BF0021C4F81F
:402240008811C4F88C110020C4F88401204630F1EFFD002104F5C87203C2BDEC048B70BD0146D1F86C0170470146D1F8700170470146D1F878017047014691F8680170477E
:4022800070B504460025204630F1E1F8172815D12046FFF7F1FF88B12046FFF7E5FF68B12046FFF7DDFF48B1204630F1C1FD002804D994F8DB00012800D00125284670BD8B
:4022C0000246002092F80D318B4203DDD2F8383253F8210070472DE9FF4F2DED0C8B83B004468946164620680121C26A204690478246D4F8B80000287DD0B9F1010F7AD114
:40230000204630F1A4F80C2804D1BAF1000F01DD4FF0010A4FF00008FDE100200190204630F195F80C2828D194F8E80190B1D4F8F80000680190D4F8F800406810B3D4F80A
:40234000F810486802A939F1EDFBD8B1029839F15AF817E0D4F8F80040680190D4F8F800006878B1D4F8F810086802A939F1DAFB40B1029839F147F804E0D4F8F80050F82E
:402380002800019002A9019839F1CCFB00287CD002980068016902988847054641462046FEF74BFD0746204630F15CF88346A16901F13000594610F0BDFE08EE100A029850
:4023C00039F121F8204630F142F80A2804D0204630F13DF811283FD1002F3CD9D4F8F810086839F10CFCE8B141462046FFF768FF00EE100A00E0E9E1B8EE400A9FED2F1ABA
:40240000C0EE010A00EE106AB8EE400A20EE800ABCEEC00A10EE100AD4F87C120844C4F87C0214E041462046FFF794FCF0EE400A00EE105AB8EE400A20EE800ABCEEC00AA4
:4024400010EE100AD4F87C120844C4F87C0229462046FFF7C5FD4DE1D4F8F810086839F1CEFB50B341462046FFF72AFF00EE100AB8EE400A9FED111AC0EE010A00EE106A93
:40248000B8EE400A20EE800A00E034E1BCEEC00AF8EE400A00EE107AB8EE400AF8EE481A80EE211A94ED9F0AB8EE400A00EE810ABCEEC00A84ED9F0A23E003E000007A44DD
:4024C000F718170841462046FFF744FCF0EE400A00EE107AB8EE400AB8EE481AC0EE011A60EEA10A00EE105AB8EE400A20EE800ABCEEC00A10EE100AD4F87C120844C4F863
:402500007C022046FFF7BCFE00287DD0FA48006820B9FA4800688047F7490860204630F187FC02462046FFF79BFE82426DD242F21071F1480068D4F089F900287AD001207D
:4025400084F860022046FFF793FE2844EC4A014600902046FFF7E0FB2046FFF7F3FB40B92046FFF7F3FBE64A014600902046FFF7BDFB2046FFF77CFE00EE100AF8EE409A9A
:402580002068016E2046884700EE100AF8EE400A9FEDDC1A80EE810AC9EE808A2046FFF763FE00EE100AB8EE400AF2EE040A80EE209A2046FFF7C6FB0246C8EE890A20469C
:4025C000FFF7C0FB00EE100AB8EE400A20EE800AF1EE000A20EE200ABCEEC00A10EE100A02EB000BF4EEC98AF1EE10FA04DC2046FFF7A8FB584517D92046FFF7A3FB00EE83
:40260000100AB8EE400A01E070E013E0F1EE040A20EE200ABCEEC00A8DED000AB84A20460099FFF731FC04E0B54A59462046FFF72BFC5FE0002084F860022046FFF782FB10
:40264000F0B32046FFF70CFE8346DCF0B6FF41EC1D0B9FEDAD0B53EC102BDCF0C1FF41EC1B0B2046FFF7FCFD8346DCF0A6FF41EC1C0B53EC1B2B61F137FD41EC190B204670
:4026800030F1D6FB8346DCF098FF41EC1A0B53EC192BDDF09DF818D82046FFF753FB8346974A59462046FFF7EFFB954A00212046FFF732FB924A00212046FFF717FB00E0C8
:4026C00003E000208C4908600BE0204630F1B0FB02462046FFF7C4FD824202D300208649086029462046FFF77BFC03E029462046FFF776FC00BFD4F8FC0040B102A9D4F8D7
:40270000FC0039F10FFA10B1029838F17CFE08F1010000F0FF08D045FFF6FFADD4F87C02B0F57A7F51D300BF4FF47A71D4F87C02B0FBF1F520680621C26A2046904760B9C0
:40274000D4F8A400A84205D9D4F8A400401BC4F8A40002E00020C4F8A40054F8A80F2844206054F8A8096A49884204D3D4F8A800401AC4F8A80054F8AC0F2844206054F8E3
:40278000AC096349884204D3D4F8AC00401AC4F8AC0054F89C0F2844206060692844606160699C3C5A49884204D3D4F8B000401AC4F8B00005EB4501C1EBC511D4F87C02DB
:4027C000A0EBC100C4F87C0200BF5DE0B9F1000F48D000250CE0D4F8F81051F8250002A939F1A0F910B1029838F10DFE681CC5B294F80D01A842EEDCD4F8FC0040B102A989
:40280000D4F8FC0039F18EF910B1029838F1FBFD2046FFF797FA90B12046FFF793FA0546374A29462046FFF72FFB354A00212046FFF772FA324A00212046FFF757FA0021F8
:40284000C4F88811C4F88C110020C4F88401204630F1EEFA002104F5C87203C2002084F8600211E00021C4F88811C4F88C110020C4F88401204630F1DBFA002104F5C872F2
:4028800003C2002084F8600220680621C26A2046904738B3D4F8002110680268516A8847D4EDA10AF8EEE00AB4EE600AF1EE10FA1CD0D4F8002110680268516A8847BDEED8
:4028C000C00A84EDA10A002240F20F112046129B5AF1C4F9D4F88402002804DDD4F88402C4F8A40002E00020C4F8A40003B0BDEC0C8BBDE8FF8F00000000002018A01008DE
:40290000F71817080000C842000000000000E03FFA592E872DE9F04105460C4616469846072795F80D01A0420BDD0027D5F8340240F8246004F1C90143463A4628465AF120
:402940008DF93846BDE8F0812DE9F04105460C4616469846072795F80D01A04211DD0027D5F8440250F82400B0420AD0D5F8440240F8246004F1920143463A4628465AF1FB
:402980006DF93846BDE8F0812DE9F04105460C4616469846072795F80D01A0420BDD0027D5F8380240F8246004F1B90143463A4628465AF153F93846BDE8F0812DE9FF5FBD
:4029C00004460D460020039002900190834620462FF148FD0090A16901F1300000990FF01EFF0746A16901F1300039460FF008FE8046D946002620680121C26A2046904744
:402A0000824620680121C26A20469047A84235DD20462FF11CFD0C2801D14FF0010A05FB08F090FBFAF000F0FF0998FBFAF04844C6B2002E01DD701EC6B2A16901F13000AC
:402A400003AB3A4649460FF09FFE18B1039834F1D9FA0190A16901F1300003AB3A4631460FF092FE18B1039834F1CCFA8346019901EB0B0000EBD07149100291029804B0A1
:402A8000BDE8F09F2DE9F74F2DED108B84B004468B469FEDFE0AF0EE408A9FEDFC0AB0EE409A9FEDFA0AB0EE408A9FEDF80AF0EE409A9FEDF60AB0EE40FA9FEDF40AF0EE32
:402AC00040FA0020029000250027804620680121C26A204690478146BBF1000F19D1002614E0002231462046169BFFF74DFF002231462046169BFFF70DFF06F1220100225F
:402B00002046169B5AF1AAF8701CC6B24E45E8DB41E220462FF19BFC0C280DD1B9F1000F0ADDB9F1010F05DD002223212046169B5AF194F84FF00109002607E24FF0000AB4
:402B400031462046FFF706F9F0EE408A9FEDCF0AB0EE409A002002909FEDCC0AB0EE408A31462046FEF769F9054620462FF17AFC0190A16901F13000019910F0DBFA07468E
:402B8000A069FCF7DEF8E8B3A069FCF7B3FB00EE100AB8EEC00A5FEDA50A80EE201A9FEDBC0A21EE000AF0EE40FA31462046FFF705FF00EE100AB8EEC00A20EE2F0A1FEDBE
:402BC000AF1AC0EE010A94ED7E0AB8EE400A30EE600ABDEEC00A10EE108A404661F138FB41EC1A0B9FEDAB0B53EC102B61F148FB15D2A069F9F714FE0190DCF0DEFC41ECC1
:402C00001A0B00E009E09FEDA30B53EC102BDCF0DFFD04D84FF0DF0801E0D4F8F88120462FF115FC0C280CD194F8E80120B1D4F8F800D0F800A008E0D4F8F800D0F804A0F0
:402C400003E0D4F8F80050F826A0BAF1000F7DD0504638F1D4FF012802D0022862D126E0504639F12EF800EE100AB8EE400AB0EE408A20462FF1EBFB0A2804D020462FF16A
:402C8000E6FB112804D1002D10D9B0EE489A0DE000EE105AB8EE400A68EE000A00EE107AB8EE400A80EE801AB0EE419A61E0F5EEC08AF1EE10FA17DD94ED100AF8EE400AFB
:402CC00094ED7E0AB8EE401A00EE105AB8EE400A21EE000A20EE800ADFED700A68EEA00A80EE201AB0EE419A002D1AD920462FF1AEFB0A2804D020462FF1A9FB112802D1E0
:402D0000B0EE498A0DE000EE107AB8EE400A69EE000A00EE105AB8EE400A80EE801AB0EE418A26E0DAF80000016A50468847B0EE408A20462FF18BFB0A2804D020462FF10B
:402D400086FB112806D1002D12D900E012E0B0EE489A0DE000EE105AB8EE400A68EE000A00EE107AB8EE400A80EE801AB0EE419A00BF00BF29EE280ABCEEC00A10EE102A67
:402D8000474B31462046FFF7FFFDB0EE690A09EE280AF0EE409A2068016E2046884700EE100AB8EE400ADFED3F0A68EE200A9FED3E1A60EE810A80EE801ABCEEC10A8DED53
:402DC000010A374B31462046019AFFF7BDFD002D22D9B8F1000F1FDDD4F8380250F8260000EE100AB8EE400ADFED300A20EE200ADFED2F0A60EE200A00EE108AB8EEC01A13
:402E000000EE105AB8EE400A21EE000A80EE801ABCEEC10A8DED020A214B31462046029AFFF778FD2DB90020D4F83C1241F8260083E020462FF10BFB0A2804D020462FF1E4
:402E400006FB112849D12846DCF0B7FB41EC1B0B404661F1FDF941EC1D0BD4F8401251F82600DCF0AAFB41EC1E0B53EC1D2BDCF0B7FB41EC1C0B53EC1B2BDCF0B1FB41ECC5
:402E80001A0B9FED0C0B53EC102B17E00000000039FA8E3C0000000000F06B4020BCBE4CF71817080000704200007A440000C842002474490000000084D79741DCF08CF94E
:402EC000CDE900019DED000B51EC100BDCF048FBD4F83C1241F826002FE03846DCF06DFB41EC1A0B404661F1B3F941EC1C0BD4F8401251F82600DCF060FB53EC1C2BCDE9CB
:402F000000019DED000B51EC100BDCF069FB41EC1B0B53EC1A2BDCF063FB41EC1D0B1FED1B0B53EC102BDCF057F941EC1E0BDCF017FBD4F83C1241F8260006F1220100226C
:402F40002046169B59F18AFE701CC6B24E45FFF6F5ADD4F8B80000281DD9D4F8F801002819D994ED7E0AF8EE400A94ED2E0AB8EE400A20EE800A5FED330A69EEA00A1FEDA9
:402F8000341A60EE810A80EE801ABCEEC10AB8EE400AB0EE40FA94ED120AB8EE400AB4EE690AF1EE10FA09D0BCEEE90A84ED120A002256212046169B59F150FE94ED130A31
:402FC000B8EE400AB4EE4F0AF1EE10FA0FD0BCEECF0A84ED130A002255212046169B59F13DFE002254212046169B59F137FE04B0BDEC108BBDE8FE8F014691F850017047AA
:4030000090ED580A704790ED550A704790ED560A704770B52DED028B04461FED640AB0EE408AD4F8EC0060B154F8EC0F22681268916A884754F8EC090268516A8847B0EE2A
:40304000408A94ED530AB4EE480AF1EE10FA23D0002516E0D4F8F80050F8250078B1D4F8F80050F8256029462046FEF773FEF0EE408A3068FE4982693046904700BF681C95
:40308000C5B294F80D01A842E4DCD4F8E80018B1D4F8E8002EF19EFBB0EE480ABDEC028B70BD10B52DED028B044694ED510AB0EE408A94F8500120B12046FFF7AAFFB0EECE
:4030C000408AB0EE480ABDEC028B10BD2DE9F0472DED028B04460D4617464FF000082046FFF7DFFFF0EE400A00EE105AB8EE400AF4EE400AF1EE10FA30D000EE105AB8EE21
:40310000400A84ED510A3B464246FF21204659F1A5FD002617E0D4F8F80050F8260080B1D4F8F80050F8269031462046FEF712FEB0EE408AD9F800003946826948469047D2
:4031400000BF701CC6B294F80D01B042E3DCD4F8E80018B1D4F8E8002EF13CFB4046BDEC028BBDE8F08711B52DED028B8FB000200E9001200D900C900B900A900020099030
:4031800008901198C06E0690D3F050FB0790B948006880471199C8661198D0F8B810C0F8BC1011982FF15EF90690119880693030059006990FF0FDF81199C1F8B80011980C
:4031C0002FF150F90690119880693030059006990FF0B0FF1199C1F8E401119880690690FBF76EFE1199C1F8F80111982FF12FF90C2804D1119890F8EA1180F8EB11002117
:40320000119880F8E81111982FF12CF9069011988069303009AB05900021069A0FF081FA80B108AA0021099833F130FC50B1089833F125F9119981F8E801119890F8E8116C
:4032400080F8EA1111982FF102F90C284FD1119890F8E91180F8EC110021119880F8E91111982FF1FFF8069011988069303009AB05900121069A0FF054FA58B108AA00216B
:40328000099833F103FC28B1089833F1F8F8119981F8E901119890F8EB0180B9119890F8EA0101280BD1119890F8EC01012806D17048006880471199C1F8F00117E0119840
:4032C00090F8E801012812D1119890F8E90101280DD11198D0F8F0010690D3F0A7FA40F2DC51884203D20021119880F8E811002006902CE01198D0F8F810069851F8200058
:4033000020B900200A9003200E900DE01198D0F8F810069851F82000059038F1EEFB18B900200A9001200E9006991198FEF712FDB5EEC00AF1EE10FA01DD012000E000203A
:403340000A9908400A900698401CC0B20690119890F80D1106988142CCDC11982FF182F806901198806905900699FBF702FA082805D11198D0F83C0108B900200A90119809
:4033800090F81802012803D139491198FDF7CEF811982FF19EFE119890F8600288B11198FFF72AFE00280BD01198FFF77AFEBCEEC00A8DED060A2E4A06991198FFF786FE3F
:4033C00016E1119880690690F9F774F9001F052871D2DFE800F004037172050000BF00BF1198D0F83411D0F8380181425DD01198D0F83401002858D91198D0F83801002826
:4034000053D900200690119890ED4C0AF8EE400A90ED4D0AB8EE400A60EE800A90ED4E0AB8EE400A80EE801ABCEEC10A8DED060A0F4A06991198FEF727FD1198FEF720FD21
:4034400090B30020059029E01198D0F83012059851F8200000EE100AF8EE400A119890ED4D0AB8EE400A60EE800A90ED4E0A03E0F718170818A01008B8EE400A80EE801A67
:40348000BCEEC10A8DED060AF74BDDE905211198FEF7BAFC0598401CC0B20590119890F80D1105988142CFDC00BF1198D0F83411C0F838119BE099E000BF1198FFF7F1FD7B
:4034C0008DED060A1198FFF7A1FD8DED050A1198FFF799FD8DED040A1198FFF791FD8DED030A9DED060AB5EEC00AF1EE10FA77DD1198FFF781FD30B39DED040AB5EEC00AC2
:40350000F1EE10FA1FDD9DED040ADDED060A80EE201A119890ED590A21EE000ABCEEC00A8DED020A9DED050ADDED060AB4EEE00AF1EE10FA01DD00200290CB4A029911981F
:40354000FEF7A2FC1FE01198FFF756FDD8B99DED030AB5EEC00AF1EE10FA14DD9DED030ADDED060A80EE201A119890ED570A21EE000ABCEEC00A8DED020ABB4A029911985C
:40358000FEF782FC00BF1198FEF77AFC40B3002002901FE0119890ED531A9DED060AC1EE000AD0F83012029851F8200000EE100AB8EE400A20EE800ABCEEC00A8DED010AA5
:4035C000A94BDDE901121198FEF71EFC0298401CC0B20290119890F80D1102988142D9DC9DED060A119880ED530A00E000BF00BF9D4A0A991198FFF745FA9B4911982FF16B
:403600001DFE994911982FF145FE11982FF1B8FE119890F84D0270B9934B079A0A991198FEF759FE1198D0F8B80002460690079911982FF1C3FC1198D0F824014FF4FA71CF
:403640000690D3F003F900286DD01198FDF798F988B3119890F85E0200282CDD11982FF1E6FA002827D911982FF1E1FA119991F85E1248431199D1F8A41001EBC10202EBFF
:403680000111B0EB810F16D31198D0F8F40040680690F8F7BCF901280DD11198FDF76CF9042808D01198D0F8800220B11198D0F88012C0F8A4101198D0F8A4000690119809
:4036C0000068D0F8EC00684A0590DDE90531119898471198D0F8A800634A0146069011982FF16CFB1198D0F8AC005F4A0146069011982FF11DFB1198D0F8B0005A4A014680
:40370000069011982FF179FB1198D0F89C00564A0146069011982FF138FB5448006880471199C1F82401504A0A991198FDF7F8FF119890F8D30040B1119880690690FBF7FD
:4037400045FC012801D1012100E00021119880F8F411119890F8D30040B1119880690690FBF734FC022801D1012100E00021119880F8F51111982FF1B7F80D901198006C15
:4037800008B9012000E000200B900A9808B10B9808B1012000E000200C9011982EF157FE0C282CD10020069022E01198D0F80811069851F8200004901198D0F808110698C5
:4037C00051F820000068406903901198D0F83C0290ED000AB8EE400A8DED050A22499DED050ADDE9032090470698401CC0B20690119890F8101106988142D6DC2EE00020B4
:40380000069025E01198D0F83C12069851F8200000EE100AB8EE400A8DED050A1198D0F80811069851F8200004901198D0F80811069851F82000006840690B4903909DED6E
:40384000050ADDE9032090470698401CC0B20690119890F8101106988142D3DC119890F8DB00132874D203E0F718170818A01008DFE810F013006F006E006E006E006E00A6
:403880001F02AC0196023303AD03F7033904B3046E006E0010066E000603119890F81401B0B100211198C0F8181111980068D0F894000690069911988847032804D10921CF
:4038C0001198FDF77DFE03E000211198FDF778FE11982EF166FE00B3FE4800688047012804D11221119880F8DB1025E0119890F8CB00012804D10921119880F8DB101BE0D8
:403900001198806900F5D2700690F7F72EFA022804D10921119880F8DB100DE0119890F8DC00012804D10C21119880F8DB1003E00121119880F8DB10119890F8DB1090F8F7
:403940001301814203D00021119880F8CB1026E2EFE300200690119890F8140118B100211198C0F8181111982EF11BFE20B90021119880F8DB1024E0D648006880470128D5
:4039800004D11221119880F8DB101AE0119890F8DC00012804D10C21119880F8DB1010E0119890F8F40120B10621119880F8DB1007E0119890F8F50118B10721119880F87B
:4039C000DB10119890F8DB1090F81301814270D11198D0F8E80028B11198D0F8E80005902EF19AFA00200590B7E011980068806906AA0490DDE904311198984701287DD1C9
:403A000006982CF118FD049005991198FDF715FA68B306982CF1EEFB042828D106982CF13FFCB5EEC00AF1EE10FA20D8119890F8CD00E0B90498052819D00498082816D0B5
:403A40000498072813D006982CF14BFCB5EEC00AF1EE10FA05DDA04A082106982CF1EFFC76E09D4A072106982CF1E9FC70E005991198FDF7E2F9E8B906982CF1BBFB0428FC
:403A800004D006982CF1B6FB012813D1049850B106982CF105FC8DED030A8F499DED030A06982CF103FC8C4A002106982CF1C7FC4EE05EE005991198FDF7BFF9F8B906988D
:403AC0002CF198FB03281AD10498052817D00498082814D00498012811D0049802280ED006982CF1FEFBB5EEC00AF1EE10FA06DD794A082106982CF1A2FC29E029E0119869
:403B000090F8CA00012805D1734A012106982CF196FC1DE0119890F8C900012805D16E4A022106982CF18BFC12E0049805280AD006982CF1B5FB8DED030A67499DED030A27
:403B400006982CF1B3FB644A052106982CF177FC00BF0598401CC0B2059011980068C0690490049911988847059988423FF73DAF2BE0002005901EE011980068806906AA46
:403B80000490DDE904311198984701280FD105991198FDF752F950B106982CF181FB8DED040A4D499DED040A06982CF17FFB0598401CC0B2059011980068C06904900499D1
:403BC0001198884705998842D6DCC0E6119890F8140118B100211198C0F8181111982EF1E0FC20B90021119880F8DB1021E0394800688047012804D11221119880F8DB103B
:403C000017E0119890F8DC0001280AD1119890F8F50108B10C9860B10C21119880F8DB1007E0119890F8F50118B90121119880F8DB10119890F8DB1090F81301814233D122
:403C40001198D0F8F000006806902CF1D3FA032825D11198D0F8F000006806902CF141FBB5EEC00AF1EE10FA19D01198D0F8F000006806902CF135FBB0EE408A1198D0F85E
:403C8000F000006806902CF10BFBB4EEC08AF1EE10FA04D208211198FDF792FC08E000211198FDF78DFC03E000211198FDF7BEFC4DE6119890F8140118B100211198C0F8A6
:403CC000181111982EF16DFC40B90021119880F8DB1025E0B0000020F7181708F84800688047012804D11221119880F8DB1017E0119890F8DC0001280AD1119890F8F40167
:403D000008B10C9860B10C21119880F8DB1007E0119890F8F40118B90121119880F8DB10119890F8DB1090F81301814233D11198D0F8F000006806902CF15CFA032825D15E
:403D40001198D0F8F000006806902CF1CAFAB5EEC00AF1EE10FA19D01198D0F8F000006806902CF1BEFAB0EE408A1198D0F8F000006806902CF194FAB4EEC08AF1EE10FA49
:403D800004D208211198FDF71BFC08E000211198FDF716FC03E000211198FDF747FCFBE3119890F8140118B100211198FDF708FC11982EF1F6FB20B90021119880F8DB1046
:403DC00023E0BF4800688047012804D11221119880F8DB1019E0119890F8DC00012810D10D9848B10C9838B9119890F8F40118B9119890F8F50140B10C21119880F8DB10C2
:403E000003E00121119880F8DB10119890F8DB1090F81301814232D11198D0F8F000006806902CF1E7F9032825D11198D0F8F000006806902CF155FAB5EEC00AF1EE10FA55
:403E400019D01198D0F8F000006806902CF149FAB0EE408A1198D0F8F000006806902CF11FFAB4EEC08AF1EE10FA04D208211198FDF7A6FB03E000211198FDF7A1FB8BE3E0
:403E8000119890F81401B0B100211198C0F8181111980068D0F894000690069911988847032804D109211198FDF78AFB03E000211198FDF785FB11982EF173FB20B90021F9
:403EC000119880F8DB1007E07D480068804718B90921119880F8DB105EE3119890F81401D8B100211198C0F8181111980068D0F894000690069911988847032804D10921D5
:403F00001198FDF75DFB03E000211198FDF758FB0021119880F8CC1015E01198806900F5D2700690F6F721FF08B9012000E00020119991F8CC10084308B1012100E0002101
:403F4000119880F8CC1011982EF12BFB20B90021119880F8DB102EE01198806900F5D2700690F6F702FF022825D0554800688047012804D11221119880F8DB101BE0119829
:403F8000806900F5D2700690F6F7EFFE012812D1119890F8CC0001280DD1119890F8DC00012804D10C21119880F8DB1003E00121119880F8DB10119890F8DB1090F8130154
:403FC000814203D000211198FDF730FBE4E2119890F81401B0B100211198C0F8181111980068D0F894000690069911988847032804D109211198FDF7E3FA03E000211198BF
:40400000FDF7DEFA11982EF1CCFA20B90021119880F8DB1019E02A4800688047012804D11221119880F8DB100FE0119890F8DC00012806D10A9840B10C21119880F8DB1081
:4040400003E00121119880F8DB10119890F8DB1090F81301814203D000211198FDF7E6FA9AE2119890F81401B0B100211198C0F8181111980068D0F894000690069911982A
:404080008847032804D109211198FDF799FA03E000211198FDF794FA11982EF182FA20B90021119880F8DB101CE0054800688047012807D11221119880F8DB1012E00000B4
:4040C000B0000020119890F8DC00012806D10B9840B90C21119880F8DB1003E00121119880F8DB1058E211982EF15BFA20B90021119880F8DB1043E0FE48006880470128DF
:4041000004D11221119880F8DB1039E0119890F8DC0001282CD10A9820B90A21119880F8DB102DE00B9828B10B21119880F8DB1026E020E2119890F8F40120B106211198DD
:4041400080F8DB101CE0119890F8F50120B10721119880F8DB1013E00D9820B10821119880F8DB100CE01021119880F8DB1007E0119890F8DC0018B90121119880F8DB10FA
:40418000119890F8DB00102826D100200690059017E011980068806906AA0490DDE9043111989847012808D1119890F84E0220B9D14A072106982CF142F90598401CC0B2C1
:4041C000059011980068C069049004991198884705998842DDDC00BFDEE100200690119890F8140118B100211198C0F8181111982EF1D7F920B90021119880F8DB1028E092
:40420000BC4800688047012804D11221119880F8DB101EE0119890F8DC00012815D1119890F8F40128B9119890F8F50108B90C9820B10C21119880F8DB100AE00D9840B1D7
:404240000C21119880F8DB1003E00121119880F8DB10119890F8DB1090F8130181427DD11198D0F8E80028B11198D0F8E80005902DF152FE00200590CDE011980068806941
:4042800006AA0490DDE9043111989847012836D1119890F84E0290BB06982CF1CCF8049005991198FCF7C9FD50B306982BF1A2FF042826D106982BF1F3FFB5EEC00AF1EEAF
:4042C00010FA1ED8049806281BD00498082818D00498072815D006982CF103F8B5EEC00AF1EE10FA05DD844A082106982CF1A7F88CE0814A072106982CF1A1F886E086E0E7
:40430000FFE705991198FCF798FD90B9049850B106982BF1C5FF8DED030A77499DED030A06982BF1C3FF744A002106982CF187F86CE000200390029011982EF188F80C28E4
:4043400028D1119890F8E801012812D111980068806B03AB01220021019000E067E0019C1198A047012825D102A90398F4F7B1FD20E011980068806B03AB01221146019098
:40438000019C1198A047012814D102A90398F4F7A0FD0FE011980068806B03AB01220190019C05991198A047012803D102A90398F4F78FFD039818B3029808B3059A03992C
:4043C0001198FDF718F9D8B14B4A062106982CF136F803980068C06A01900199039888470446029837F19BFB84420ED20598401D414B072201460190119858F12FFC04E04F
:404400003D4A002106982CF11AF800BF00BF0598401CC0B2059011980068C0690490049911988847059988423FF727AF31E0002005901EE011980068806906AA0490DDE96A
:4044400004311198984701280FD106982BF1F3FF06280AD106982BF123FF8DED040A26499DED040A06982BF121FF0598401CC0B2059011980068C069049004991198884799
:4044800005998842D6DC1D48006880471199C1F8180181E0119890F8140128B11748006880471199C1F81C0111982EF17AF820B90021119880F8DB104DE00E480068804752
:4044C000012804D11221119880F8DB1043E0119890F8DC0001283AD1119890F8F40138B9119890F8F50118B90C9808B90D9858B10C2105E0B0000020F718170818A0100819
:40450000119880F8DB1026E01198D0F82001C8B11198D0F820016421484306901198D0F81C0105900699D2F091F958B91198D0F8180138B11198D0F81801FE490690D2F06B
:4045400085F940B10D21119880F8DB1003E00121119880F8DB10119890F8DB1090F81301814204D105211198FDF72AF802E000211198816610E00022114611982EF115F87B
:4045800000211198FDF71CF800211198C0F81811119880F8DB1000BF00BF0021119880F81411119890F8DB1090F81301814215D011980068006D06900699119888470121E0
:4045C000119880F81411119890F8DB1080F81311D94B07221A21119858F140FB1198FCF7A4FF1198FCF74CFF1198FCF794FD1198D0F8280140F6B8310690D2F027F958B17B
:40460000CE48006880471199C1F828011198FCF766FC1198FCF795FB0E980FB0BDEC028B18BD2DE9F04104460D461646002794F84C02A84207D084F84C5233463A468F214A
:40464000204658F10BFB3846BDE8F0810146D1F83C0170472DE9F04105460C46164600272846FFF7F3FFA04208D0C5F83C4133463A464FF48871284658F1F0FA3846BDE843
:40468000F08190ED530A704790ED510A70472DE9F04104460D461646002794F85001A84208D084F8505133463A4640F21111204658F1D4FABDE8F0812DE9F04104460D4682
:4046C0001646002794F86801A84208D084F8685133463A464FF48071204658F1BFFA3846BDE8F0812DE9F04104460D4616460027D4F87001A84208D0C4F8705133463A4646
:404700004FF48171204658F1A9FA3846BDE8F0812DE9F04104460D4616460027D4F86C01A84208D0C4F86C5133463A4640F20111204658F193FA3846BDE8F081014691F8A6
:40474000690170472DE9F04104460D461646002794F86901A84208D084F8695133463A4640F20511204658F179FA3846BDE8F0812DE9F04104460D4616460027D4F87C011C
:40478000A84208D0C4F87C5133463A464FF48371204658F163FA3846BDE8F0812DE9F04104460D461646002794F88001A84208D084F8805133463A4640F20711204658F169
:4047C0004DFA3846BDE8F08190ED570A704770B52DED028B0446B0EE408A0D4600262046FEF70EFCB4EE480AF1EE10FA08D084ED588A2B4632464FF48A71204658F12EFAE7
:404800003046BDEC028B70BD2DE9F0412DED028B0446B0EE408A0D46164600272046FFF7D3FFB4EE480AF1EE10FA19D084ED578A3EB1D4ED510AB0EE600A29462046FFF705
:40484000C6FF2B463A4640F21511204658F106FA2A46BCEEC80A10EE101A2046FDF714FB3846BDEC028BBDE8F08190ED590A704770B52DED028B0446B0EE408A0D460026A6
:4048800094ED590AB4EE480AF1EE10FA08D084ED598A2B4632464FF48B71204658F1DEF93046BDEC028B70BD30B52DED048B81B004460020009020462DF1D4FD05466B467A
:4048C0000A222946A069F7F7B5FDE8B1009836F15BFAF0EE408A009836F150FAB0EE408A2046FEF790FBB0EE409A38EEC80AC0EE090AF0EE609A0021F0EE690AB0EE480A5D
:40490000009836F1A3FA00BF01B0BDEC048B30BD70B52DED028B0446B0EE408A0D46002694ED560AB4EE480AF1EE10FA0FD084ED568A05E0C0D40100F718170818A0100829
:404940002B4632464FF48971204658F187F92046FFF7AAFF3046BDEC028B70BD70B52DED028B0446B0EE408A0D46002694ED550AB4EE480AF1EE10FA19D094ED550AB5EEE4
:40498000C00AF1EE10FA09D1DFEDFC0A68EE200AB0EE600A29462046FFF7BAFF84ED558A2B46324640F21311204658F157F92046FFF77AFF3046BDEC028B70BD30B52DED51
:4049C000048B81B004460020009020462DF14AFD05466B460A222946A069F7F72BFDE8B1009836F1D1F9B0EE408A009836F1C6F9F0EE408A00980068416900988847B0EE1D
:404A0000409A38EE680AC0EE090AF0EE609A0021B0EE690A2046FFF7A1FF00BF01B0BDEC048B30BD014691F8690270472DE9F04104460D461646002794F86902A84208D096
:404A400084F8695233463A464FF49E71204658F105F93846BDE8F081014691F86A0270472DE9F04104460D4616460027D4F86402A84208D0C4F8645233463A464FF49F7167
:404A8000204658F1EBF83846BDE8F0812DE9F04104460D461646002794F86802A84208D084F8685233463A4640F23F11204658F1D5F83846BDE8F08190ED9B0A70470246CF
:404AC0000020D2ED9B0AF4EE400AF1EE10FA01D082ED9B0A704790ED9C0A704702460020D2ED9C0AF4EE400AF1EE10FA01D082ED9B0A704790ED9D0A704702460020D2ED27
:404B00009D0AF4EE400AF1EE10FA01D082ED9D0A704790ED9E0A704702460020D2ED9E0AF4EE400AF1EE10FA01D082ED9E0A70472DE9F04706460D4614461F46DDF820908C
:404B40004FF00008022D23DA052C21DA05EB850106F5D47000EB810050F82400B84217D005EB850106F5D47000EB810040F824703DB904F217114B464246304658F16EF8E9
:404B800006E004F21D114B464246304658F166F84046BDE8F0872DE9F04706460D4614461F46DDF820904FF00008022D23DA052C21DA05EB850106F5E87000EB410030F827
:404BC0001400B84217D005EB850106F5E87000EB410020F814703DB904F223114B464246304658F13BF806E004F229114B464246304658F133F84046BDE8F0872DE9F04102
:404C000005460C46164698460027022C10DA05F5CC7050F82400B0420AD005F5CC7040F8246004F22F1143463A46284658F116F83846BDE8F0812DE9F04105460C46164626
:404C400098460027022C10DA05F5D07050F82400B0420AD005F5D07040F8246004F2311143463A46284657F1F9FF3846BDE8F08170B504460D46164694F86102A84208D05D
:404C800084F8615233463A4640F23311204657F1E5FF384670BD70B504460D46002694F80D01A8420DDDD4F8F82052F8250052F825201268116A8847BCEEC00A10EE106A31
:404CC0000FE094F80D0194F80F110844A84208DDD4F8FC000268116A8847BCEEC00A10EE106A304670BD0146092070470346072070470146D1F82C0170472DE9F0472DEDB0
:404D0000028B04460E4617464FF000082068016E20468847B0422CD0C4F82C613B4642462021204657F19AFF002517E0D4F8F80050F8250080B1D4F8F80050F82590294602
:404D40002046FDF707F8B0EE408AD9F80000394682694846904700BF681CC5B294F80D01A842E3DCD4F8E80018B1D4F8E8002CF131FD4046BDEC028BBDE8F087CDCC4C3D5F
:404D800010B52DED028B04469FEDFE0AB0EE408AD4F82C0100282ED9D4F8300100282AD9A069F7F787FC062802D0072811D100BF94ED4D0AF8EE400A94ED4C0AB8EE400AD8
:404DC00080EE801A9FEDF00A21EE000AB0EE408A10E094ED4C0AB8EE400ADFEDEC0A60EE200A94ED4B0AB8EE400A80EE801AB0EE418A00BF00BFB0EE480ABDEC028B10BD0B
:404E00000146002070470346072070470146D1F8200170472DE9F04104460D4616460027D4F82001A84207D0C4F8205133463A464321204657F112FF3846BDE8F08190EDD6
:404E40007F0A70472DE9F0412DED028B0446B0EE408A0E4600279FEDCD0AB4EEC08AF1EE10FA04DD02279FEDC90AB0EE408A002511E0D4F8080150F8250058B1D4F8081188
:404E800051F8250051F825100968CA693146B0EE480A90476D1C94F81001A842E9D894ED7F0AB4EE480AF1EE10FA07D084ED7F8A33463A464821204657F1D0FE3846BDEC16
:404EC000028BBDE8F08190ED800A70472DE9F0412DED028B0446B0EE408A0E4600279FEDAC0AB4EEC08AF1EE10FA04DD02279FEDA80AB0EE408AB5EEC08AF1EE10FA04D2C3
:404F000003279FEDA00AB0EE408A00250EE0D4F8F00050F8250040B1D4F8F01051F825003146B0EE480A2BF16BFA6D1C94F80C01A842ECD894ED800AB4EE480AF1EE10FAA2
:404F400007D084ED808A33463A465121204657F185FE3846BDEC028BBDE8F08131B1012907D0022908D003290CD108E090ED810A08E090ED820A05E090ED830A02E090ED5B
:404F8000840A00BF00BF70472DE9F0412DED028B0446B0EE408A0F4616464FF000089FED7C0AB4EEC08AF1EE10FA05DD4FF002089FED770AB0EE408AB5EEC08AF1EE10FA39
:404FC00005D24FF003089FED6F0AB0EE408A37B1012F30D0022F5AD0032F7CD185E0002515E0D4F8080150F8250078B1D4F8081151F82500F3F76AFF40B9D4F8081151F87A
:4050000025003146B0EE480A2CF165FB6D1C94F81001A842E5D894ED810AB4EE480AF1EE10FA07D084ED818A334642464421204657F114FE86E0002515E0D4F8080150F89B
:40504000250078B1D4F8081151F82500F3F73EFF40B9D4F8081151F825003146B0EE480A2CF157FB6D1C94F81001A842E5D894ED820AB4EE480AF1EE10FA07D084ED828A3B
:40508000334642464521204657F1E8FD5AE0002515E0D4F8080150F8250078B1D4F8081151F82500F3F712FF40B9D4F8081151F825003146B0EE480A2CF149FB6D1C94F8C0
:4050C0001001A842E5D894ED830AB4EE480AF1EE10FA09D000E034E084ED838A334642464621204657F1BAFD2CE0002515E0D4F8080150F8250078B1D4F8081151F8250011
:40510000F3F7E4FE40B9D4F8081151F825003146B0EE480A2CF139FB6D1C94F81001A842E5D894ED840AB4EE480AF1EE10FA07D084ED848A334642464721204657F18EFDEE
:4051400000E000BF00BF4046BDEC028BBDE8F081014691F8190270472DE9F04104460D461646002794F81902A84207D084F8195233463A464B21204657F170FD3846BDE804
:40518000F08100000000000000401C460000C84200007A4490ED870A70472DE9F0412DED028B0446B0EE408A0E46002794ED870AB4EE480AF1EE10FA16D0F74890ED000A99
:4051C000B4EEC80AF1EE10FA02D884ED878A05E0F14890ED000A84ED870A032733463A464F21204657F13AFD002511E0D4F8F00050F8250050B1D4F8F01051F82500D4ED9C
:40520000870AB0EE600A31462BF1C3F8681CC5B294F80C01A842E9DC3846BDEC028BBDE8F08190ED880A70472DE9F0412DED028B0446B0EE408A0E46002794ED880AB4EEE4
:40524000480AF1EE10FA07D084ED888A33463A464E21204657F102FD00250FE0D4F8F00050F8250040B1D4F8F01051F825003146B0EE480A2BF156F8681CC5B294F80C01B7
:40528000A842EBDC3846BDEC028BBDE8F08190ED890A70472DE9F0412DED028B0446B0EE408A0E46002794ED890AB4EE480AF1EE10FA07D084ED898A33463A465021204675
:4052C00057F1CCFC00250FE0D4F8F00050F8250040B1D4F8F01051F825003146B0EE480A2BF102F8681CC5B294F80C01A842EBDC3846BDEC028BBDE8F0810146D1F8140284
:4053000070472DE9F04104460E4617464FF0070894F81902012802D0022834D100BF4FF0000800251EE0D4F8F00050F82500B8B1D4F8F01051F825002AF15CFF022807D0E9
:40534000D4F8F01051F825002AF154FF012807D1D4F8F01051F825003A463146F3F7D3FC681CC5B294F80C01A842DCDCD4F81402B04207D0C4F814623B46424652212046A5
:4053800057F16CFC0AE0D4F81402B04205D03B4642465221204657F161FC00BF00BF4046BDE8F08110B50346072021B9012483F81842002000BF00BF10BD10B50346002067
:4053C000C3F8801210BD2DE9F04104460D4616460027D4F89000A8425FD02046FBF7D0FAF0B32046FBF7C4FA002841DD20462DF11EFC00283CD920462DF119FC94F85E1226
:40540000484305EBC50101EB0511B0EB810F06D2D4F8F4104868F6F7FAFA01281DD020462DF105FC94F85E12484305EBC50101EB0511B0EB810F05D9D4F8F4104868F6F775
:40544000E6FA50B120462DF1F2FB94F85E1248436421B0FBF1F0A84212D13246204600E006E0D4F89010FFF7A8FFC4F8905007E032462046D4F89010FFF79FFFC4F89050CB
:4054800033463A467A21204657F1E8FB33463A464FF48771204657F1E1FBD4F8A400A84245D02046FBF76CFAF0B32046FBF760FA00283ADD20462DF1BAFB002835D9204673
:4054C0002DF1B5FB94F85E12484305EBC50101EB0511B0EB810F06D2D4F8F4104868F6F796FA01281DD020462DF1A1FB94F85E12484305EBC50101EB0511B0EB810F05D921
:40550000D4F8F4104868F6F782FA50B120462DF18EFB94F85E1248436421B0FBF1F0A84205D1C4F8A45002E0FFE7C4F8A4503846BDE8F0810146D1F88002704702460020AF
:4055400092F80D318B4203DDD2F8443253F82100704770B504460125D4F8F400006830B1D4F8F4100868F6F752FA00B10025284670BD10B5044620462DF1E2F810BD2DE97B
:40558000F04704460F4616463246394620462DF1EFF88046002511E0004417082068D0F8C410204688478146206833462A464946D0F800C12046E047681CC5B294F80D014D
:4055C000A842EBDC4046BDE8F0870246002092F80D318B4203DDD2F8403253F8210070472DE9F04105460E4614469846002795F80D01A04212DD28682146D0F8FC20284622
:405600009047B0420AD0D5F8400240F8246004F1A20143463A46284657F120FB3846BDE8F08190ED8A0A7047014691F84A027047014691F84B0270470146D1F82C02704792
:40564000014691F848027047014691F84902704710B50346002093F84D428C4201D083F84D1210BD10B50346002093F84E428C4201D083F84E1210BD014691F85A02704786
:405680002DE9F04104460D461646002794F85A02A84207D084F85A5233463A46B521204657F1DCFA3846BDE8F081014691F85B027047014691F8570270472DE9F041044676
:4056C0000D461646002794F85702A84207D084F8575233463A46B321204657F1BFFA3846BDE8F081014691F8580270472DE9F04105460C4616460027642C01DD02276424DA
:4057000095F85802A04207D085F8584233463A46B221284657F1A2FA3846BDE8F081014691F85902704710B5044620462DF142FA10BD0246002092F80D318B4204DDB2F8FA
:4057400050320B4103F00100704710B5044620462DF134FA10BD0246002092F80D318B4204DDB2F852320B4103F001007047014691F8540270472DE9F04104460D46164602
:40578000002794F85402A84207D084F8545233463A46B421204657F161FA3846BDE8F081014691F85502704702460020022902DA02F51773585C70472DE9F04105460C4675
:4057C00016461F464FF00008022C09DA05F51770065504F1FD013B460022284657F13EFA4046BDE8F0812DE9F04104460D461646002794F85F02A84207D084F85F523346D9
:405800003A46B621204657F129FA3846BDE8F0812DE9F04105460C4616460027642C08DC85F85E4233463A46B721284657F116FA00E002273846BDE8F0812DE9F0410446EF
:40584000002720680121C26A204690478046002600251CE020462CF1FAFD0C280AD194F8E80118B1D4F8F800066807E0D4F8F800466803E0D4F8F80050F825602EB13046C6
:4058800036F1BDF908B1012703E0681CC5B24545E0DB3846BDE8F08170B52DED048B04460D46002620462CF17CFE98B394F81201A8422FDDD4F8041151F82500F4F7DFFEEE
:4058C000B0EE408AD4F8041151F82500F4F703FEF0EE408AD4F8041151F82500F4F7CCFE00EE100AB8EE400ADFED6B0A80EE201AB0EE419A38EE090AB4EEE80AF1EE10FA49
:4059000006D338EE490AB4EEE80AF1EE10FA00DD012600BF3046BDEC048B70BD2DE9FC5F04460D46002720462CF19CFD0646A16901F1300031460CF072FF8046A16901F18B
:40594000300041460CF05CFE8146BA460020019020680121C26A20469047834620680121C26A20469047A84227DD20462CF16FFD0C2801D14FF0010B05FB09F090FBFBF016
:4059800000F0FF0A99FBFBF05044C0B20190564610E000200090A16901F130006B46424631460CF0F1FE18B1009831F1EBFA0744701CC6B201988642EBDB3846BDE8FC9F39
:4059C00070B504460D4616463246294620462DF163FA70BD2DE9F04104460E4615469846002794F80D01A8421DDDB4F85002284100F00100B04216D0012E06D1B4F850029D
:405A0000A9400843A4F8500206E0B4F850020121A9408843A4F8500205F1D90143463A46204657F11BF93846BDE8F08170B504460D4616463246294620462DF142FA70BD7B
:405A40002DE9F04104460E4615469846002794F80D01A8421DDDB4F85202284100F00100B04216D0012E06D1B4F85202A9400843A4F8520206E0B4F852020121A94088434B
:405A8000A4F8520205F1E90143463A46204657F1E5F83846BDE8F0810000C84270B5044620462CF160FC002004F5987404F8010C207001206070FE48006880476060002092
:405AC000A060FB48006880476061A4F5987400202CE09FEDF80A04F5A47101EB800181ED000A002204F5AE7141F82020143141F82020143141F82020143141F820201431EF
:405B000041F82020143141F8202000210AE0002300EB400504F5EA7202EB850242F821304A1CD1B20329F2DB411CC8B20528D0DB9FEDE00A84ED840A0020C4F81402C4F8C8
:405B4000180220462CF183FC05280CD10020C4F81C02062084F820020020C4F82402062084F828020BE00020C4F81C02032084F820020020C4F82402032084F828020020E2
:405B8000C4F82C0200214FF40C7001519FEDC90A84ED8D0A9FEDC70A84ED8E0A002084F8400284F84102C4F844029FEDC20A84ED8F0A84F86C0284F86D022068BE4A03692A
:405BC000204698479FEDBB0A84ED9F0A002009E09FEDB80A04F5207101EB800181ED000A411CC8B20528F3DB00214FF425700155401C01550020C4F89802C4F89C02AC4898
:405C000000688047C4F8A0020020C4F8A4026065C4F8A802C4F8AC02A54800688047C4F8B402A34800688047C4F8B002002084F8B8029FEDA00A84ED920A4FF47A70C4F828
:405C40004C02002084F8CA0284F8CB0284F8C90284F8CC0284F8CD0284F8CE0284F8CF0284F8D00284F8C002C4F8C40284F8C802C4F8BC02012084F8D10284F8D202002002
:405C8000C4F8D402C4F8D80284F8DC0284F8DD02072084F8DE029FED870A84ED3B0A9FED850A84ED3C0A9FED830A84ED3D0A0020C4F8E0027E4800688047C4F8E40270BD8C
:405CC000F8B504460F4615461E462B4600223946204600962CF19CFA04467848A43444F8A40C00F5807044F8980C103044F8940C00206065A065E06520666066A066E06662
:405D000020676067A067E06784F8800084F8810084F8820084F8830084F8840084F8850084F8860084F8870084F8880084F8890084F88A00A43C2046FFF7B0FE23462A46F9
:405D40005F49204656F115FF2046F8BD10B504465A48206000F58070E0601030206194F82401002810DDD4F8F80068B1002084F82401D4F8F80020B1D4F8F80002685168A8
:405D800088470020C4F8F80094F82501002810DDD4F8FC0068B1002084F82501D4F8FC0020B1D4F8FC000268516888470020C4F8FC0094F82601002810DDD4F8000168B1FD
:405DC000002084F82601D4F8000120B1D4F800010268516888470020C4F8000194F82901002810DDD4F8180168B1002084F82901D4F8180120B1D4F818010268516888478A
:405E00000020C4F8180194F82A01002810DDD4F81C0168B1002084F82A01D4F81C0120B1D4F81C010268516888470020C4F81C0194F82B01002810DDD4F8200168B1002057
:405E400084F82B01D4F8200120B1D4F820010268516888470020C4F8200194F82C01002810DDD4F80C0168B1002084F82C01D4F80C0120B1D4F80C010268516888470020C2
:405E8000C4F80C0194F82D01002810DDD4F8100168B1002084F82D01D4F8100120B1D4F810010268516888470020C4F8100109E018A0100800000000BF18170844A3100872
:405EC000CD31140894F82E01002810DDD4F8140168B1002084F82E01D4F8140120B1D4F814010268516888470020C4F8140120462CF1CAF90446204610BD70B504462046E5
:405F0000FFF724FF05465BF10DFE70BD10B50446103C2046FFF7F1FF10BD10B504460C3C2046FFF7EAFF10BD10B50446103C2046FFF70CFF10BD10B504460C3C2046FFF75A
:405F400005FF10BD70B50546012406E0F74B00222146284656F182FE641C7D2CF6D37E2406E0F24B00222146284656F177FE641CB62CF6D370BD70B504460D461646002DC8
:405F80007BD120683246036F20469847206832460021836F2046984794F86D0205286DD2DFE800F05B2F03908A0020683146B0EE080AD0F88020204690473246002120466E
:405FC0002CF1E9FC206831469FEDD90AD0F8A8202046904720683146B0EE080AD0F8A02020469047206831461FED4E0AD0F8B0202046904720683246294643692046984758
:4060000088E020683146B0EE080AD0F88020204690473246002120462CF1BDFC206831469FEDC30AD0F8A8202046904720683146B0EE080AD0F8A020204690472068314637
:406040001FED640AD0F8B020204690472068324629464369204698475CE020683146B0EE080AD0F88020204690473246002120462CF191FC2068314601E053E049E09FED70
:40608000AC0AD0F8A82020469047206831469FEDA90AD0F8A02020469047206831461FED7B0AD0F8B020204690472068324629464369204698472DE03246002120462CF16C
:4060C0006AFC00BF20683146B0EE000AD0F8802020469047206831469FED950AD0F8A8202046904720683146B7EE000AD0F8A02020469047206831461FED920AD0F8B02086
:406100002046904720683246294643692046984700E000BF00BF854B00224FF6FF71204656F19CFD70BD70B504460D461646002D74D1002084F86C0294F86D0205286ED248
:40614000DFE800F06E3703A2A300206831469FED7A0AD0F8882020469047206832460021B2EE0E0AD0F89030204698472068324601219FED710AD0F890302046984720689B
:40618000324602211FEDB50AD0F89030204698472068324603219FED690AD0F8903020469847206832460021D0F8B83020469847A0E0206831469FED600AD0F8882020465B
:4061C0009047206832460021B2EE0E0AD0F89030204698472068324601219FED570AD0F89030204698472068324602211FEDCF0AD0F89030204698472068324603219FEDC1
:406200004F0AD0F8903020469847206832464FF4C871D0F8B830204698476BE072E068E0206831469FED440AD0F88820204690472068324600219FED400AD0F89030204677
:406240009847206832460121B3EE040AD0F89030204698472068324602219FED370AD0F89030204698472068324603219FED320AD0F8903020469847206832460021D0F842
:40628000B8302046984735E000BF206831469FED2A0AD0F88820204690472068324600219FED250AD0F8903020469847206832460121B2EE040AD0F89030204698472068A3
:4062C000324602219FED1E0AD0F8903020469847206832460321B7EE080AD0F8903020469847206832460021D0F8B8302046984700E000BF00BF0D4B00224FF6FF712046D1
:4063000056F1ACFC70BD10B50346002093F824418C4206DDD3F8F8401CB1D3F8F8401460012010BD014691F824017047BF1817080000C84200000C42000048420000204257
:406340000000000070B504460D460026D4F8F80038B1D4F8F80029F14DFFA84201D1701CC6B2304670BD30B5044600200E2A47D2DFE802F019071022464646462B3446464D
:40638000463D94F82551012D03D1D4F8FC501D60012036E094F82651012D03D1D4F800511D6001202DE094F82851012D03D1D4F808511D60012024E094F82751012D03D1E9
:4063C000D4F804511D6001201BE094F82C51012D03D1D4F80C511D60012012E094F82D51012D03D1D4F810511D60012009E094F82E51012D03D1D4F814511D60012000E0A3
:4064000000BF00BF30BD30B50446002000251D602AB919B9D4F8FC501D60012000E000BF00BF30BD024600200E291DD2DFE801F010070A0D1C1C1C1C13161C1C1C1992F846
:40644000250112E092F826010FE092F827010CE092F8280109E092F82C0106E092F82D0103E092F82E0100E000BF00BF70472DE9F8430446884617461D46089E4FF000090D
:406480000A2F7DD2DFE807F02D05194182828282586C94F8250101280ED16946D4F8FC0035F140FB40B10098F2F791FDA84203D1009830604FF0010969E094F82601012858
:4064C0000ED16946D4F8000135F12CFB40B10098F2F77DFDA84203D1009830604FF0010955E094F8280101280ED16946D4F8080135F118FB40B10098F2F769FDA84203D194
:40650000009830604FF0010941E0B8F1000F12D194F8270101280EDB6946D4F8040135F101FB40B10098F2F752FDA84203D1009830604FF001092AE094F82C0101280ED10B
:406540006946D4F80C0135F1EDFA40B10098F2F73EFDA84203D1009830604FF0010916E094F82D01012810D16946D4F8100135F1D9FA50B10098F2F72AFDA84205D100E022
:4065800004E0009830604FF0010900E000BF00BF4846BDE8F8832DE9F84304460D4617461E464FF0000817B1012F29D113E08DB994F8250101280DD16946D4F8FC0035F103
:4065C000B1FA38B10098F2F702FD18B9009830604FF0010815E095B994F8270101280EDB6946D4F8040135F19DFA40B10098F2F7EEFC012803D1009830604FF0010800E057
:4066000000BF00BF4046BDE8F88330B50446002022B1012A14D0032A1BD108E094F82B51012D03D1D4F820511D60012012E094F82A51012D03D1D4F81C511D60012009E064
:4066400094F82951012D03D1D4F818511D60012000E000BF00BF30BD014691F82A0191F82B21104491F829211044C0B270470246002031B1012907D0032908D192F82A017B
:4066800006E092F82B0103E092F8290100E000BF00BF70472DE9F04104460D460026002D5ED094F8240101285ADAC4F8F85094F82401401C84F82401D4ED9C0AB0EE600AFE
:4066C0002068FA49D0F8A02020469047D4ED9D0AB0EE600A2068F549D0F8A8202046904794F86D122068F14AD0F8983020469847D4ED950AB0EE600A2068EC49D0F88820CF
:4067000020469047D4ED9E0AB0EE600A2068E749D0F8B02020469047D4F868122068E34AD0F8B8302046984794F82421521ED1B2D4F8F80029F173FD20462BF193FE0746BC
:406740003946D4F8F80029F15DFD94F82411491E8AB22346D649D4F8F80056F10AFA0126012E05D1D14B00225321204656F176FA3046BDE8F081DFEDCF0AB0EE600A092901
:4067800033D2DFE801F0050A0F14191E23282D00DFEDC90AB0EE600A28E0DFEDC80AB0EE600A23E0DFEDC60AB0EE600A1EE0DFEDC50AB0EE600A19E0DFEDC30AB0EE600A04
:4067C00014E0DFEDC20AB0EE600A0FE0DFEDC00AB0EE600A0AE0DFEDBF0AB0EE600A05E0DFEDBD0AB0EE600A00E000BF00BF704700B503469FEDAF0AB0EE401AD3F81C0238
:4068000068B193F820121846FFF7B5FFD3ED870AF8EE600AC0EE201AB0EE611A03E09FEDA50AB0EE401AB0EE410A00BD2DE9F0412DED028B04460D464FF00008002D74D0D9
:40684000284635F184F90E2870D2DFE800F052072D609A9A9A9A707E9A9A9A8C94F82501012820DA94F82501401C84F82501C4F8FC50002611E0D4F8FC0068B1D4F8FC7085
:406880002068816E20468847B0EE408A3868874982693846904700BF761C94F82501B042E9D84FF001086DE094F8260101281FDA94F82601401C84F82601C4F8005100260F
:4068C00010E0D4F8000160B12046D4F80071FFF78FFFB0EE408A3868744982693846904700BF761C94F82601B042EAD84FF0010848E094F82801012808DA94F82801401CA5
:4069000084F82801C4F808514FF001083AE094F82701012808DA94F82701401C84F82701C4F804514FF001082CE02CE029E094F82C01012808DA94F82C01401C84F82C01CC
:40694000C4F80C514FF001081CE094F82D01012808DA94F82D01401C84F82D01C4F810514FF001080EE094F82E01012808DA94F82E01401C84F82E01C4F814514FF00108F1
:4069800000E000BF00BF4046BDEC028BBDE8F081F8B504460D46002600200090002D37D069462846F2F795FA78B3009835F1CFF820B101281CD0032828D10CE094F82B0160
:4069C000012807DAC4F8205194F82B01401C84F82B0101261BE094F82A01012807DAC4F81C5194F82A01401C84F82A0101260EE094F82901012807DAC4F8185194F829012E
:406A0000401C84F82901012601E001E000BF00BFCDB32846F2F75AFAA8BBD4ED960AB0EE600A2068214A0021D0F8903020469847D4ED970AB0EE600A20681C4A0121D0F8D3
:406A4000903020469847D4ED980AB0EE600A2068164A0221D0F8903020469847D4ED990AB0EE600A2068114A0321D0F8903020469847D4ED940AB0EE600A20680B49D0F883
:406A80008020204690473046F8BD70B504460D4694F82401012808D1D4F8F80028B100222946D4F8F80029F1CAFC70BDBF1817085331140800000000002474498096184B6A
:406AC0000F0B674AE966104C58BC8A4A00007A440F0BE74626FADD46E76C8A4A70B52DED028B04460D4694F82401012816D1D4F8F80098B15DB1D4F8F80029F1D1FBB0EE3C
:406B0000408A0021D4F8F80029F1D0FB06E000211FED180AD4F8F80029F1C8FBBDEC028B70BD2DE9F04104460E461546002794F8240158B1D4F8F80040B1012D06D100228B
:406B40003146D4F8F80029F198FB01273846BDE8F0812DE9F04104460F462068C16C20468847E8B3D4ED131AF8EE611AB0EE611AD4ED101AF8EE611AF0EE610A94F8390044
:406B800001EE900AF8EE611AB0EE610A2CF1AEF928B1216CE06C884201D9012000E0002005462068FE4A2946D0F8F43020469847D4ED131AF8EE611AB0EE611AD4ED101A99
:406BC000F8EE611AF0EE610A94F8390001EE900AF8EE611AB0EE610A2CF188F938B100E00FE0216CE06C884201D2012000E0002005462068EA4A2946D0F8F03020469847A3
:406C00000DE02068E64A0021D0F8F430204698472068E34A0021D0F8F03020469847D4F8D452012620680321C26A20469047002808DD94F8DD0228B9D4F804010EF0A6FA64
:406C400000B100262068C16C2046884748B3012E17D120462BF1FBFB04280BD0D4ED8D0A00EE105AB8EE400A20EE800ABCEEC00A10EE105AD4F8D802A84204D9D4F8D8524B
:406C800001E0D4F8D852D4F8A402A84205D2012084F8DC02C4F8A45206E0002084F8DC0202E0002084F8DC0294F8270128B3D4F8040134F122FF00B3D4F8040134F1A4FEF0
:406CC000D8B1D4F8040134F1B8FEB5EEC00AF1EE10FA12DDD4F8040134F1CDFE68B1D4F8040134F18BFE05464FF47A71CFF0AEFD18B1012084F8CD0202E0002084F8CD025C
:406D000094F8270128B3D4F8040134F1F6FE00B3D4F8040134F1B3FED8B1D4F8040134F1C7FEB5EEC00AF1EE10FA12DDD4F8040134F1DCFE68B1D4F8040134F162FE05466D
:406D40004FF47A71CFF082FD18B1012084F8CE0202E0002084F8CE0294F8280128B3D4F8080134F1CAFE00B3D4F8080134F14CFED8B1D4F8080134F160FEB5EEC00AF1EEAD
:406D800010FA12DDD4F8080134F175FE68B1D4F8080134F133FE05464FF47A71CFF056FD18B1012084F8CC0202E0002084F8CC0220462CF13DF8E16B884203D8012084F8D8
:406DC000D80002E0002084F8D800BDE8F0812DE9F04104460D4616460027D4F81402A84207D0C4F8145233463A468421204655F135FFD4F81802A84201D0C4F81852384660
:406E0000BDE8F0812DE9F04105460C46164698460727052C1BDA002705F5D67050F82400B0420AD005F5D67040F8246004F1A80143463A46284655F111FF05F5E07050F832
:406E40002400B04203D005F5E07040F824603846BDE8F081014691F8D00270472DE9F0412DED028B0446B0EE408A1FEDEE0AF0EE408A002620462BF1EAFA162804D02046E6
:406E80002BF1E5FA15287CD120680D21C26A20469047002875DDD4F81401002871D0D4F81471012577E0384634F1FBF8042803D0384634F1A4FE70B12946384634F163F933
:406EC00000EE100AB8EE400ADFED360A80EE201AF0EE418A03E09FED340AF0EE408A04F5A47000EB850090ED000A08EE280A04F5A47000EB850080ED000A04F5A47000EBD0
:406F0000850090ED000ADFED290AB4EEE00AF1EE10FA3EDB00BF04F5A47000EB850090ED000ADFED220A80EE201ABCEEC10A10EE106A04F5E07050F82500811904F5E070CF
:406F400040F8251050F825001949884208D304F5E07050F82500411A04F5E07040F8251004F5A47000EB8500D0ED000A4FF47A7106FB01F000EE100AB8EE400A30EEC00A25
:406F800000E06AE004F5A47000EB850080ED000A00BF681CC5B2052D85DB38460AE00000BF1817080050C3470000000000007A44FA592E8734F175F8042803D0384634F1B5
:406FC0001EFE68B1384634F15EF900EE100AB8EE400A5FED0C0A80EE201AF0EE418A03E01FED0F0AF0EE408A94ED840A08EE280A84ED840A94ED840A5FED140AB4EEE00ACC
:40700000F1EE10FA28DB00BF94ED840A5FED190A80EE201ABCEEC10A10EE106AD4F818023044C4F81802F549D4F81802884204D3D4F81802401AC4F81802D4ED840A4FF4F5
:407040007A7106FB01F000EE100AB8EE400A30EEC00A84ED840A00BF00BFBDEC028BBDE8F0812DE9F0472DED028B82B004460F4616469846DDF830A000252068816E2046E4
:407080008847B0EE408AA94620462BF1E0F9152806D120462BF185FA40B14FF0010905E0D4F8B800002801D94FF00109B9F1010F7ED1002F7CD000200190D4F8FC0078B126
:4070C00001A9D4F8FC0034F12DFD48B1019800680169019888470546019834F194F900E00025D4F8FC0034F18AFDE8B320462BF11BFB00EE100AB8EE400A1FED541AC0EEA1
:40710000010A00EE106AB8EE400A20EE800ABCEEC00AB8EE400AD4ED3B0A30EE200A84ED3B0A20462BF100FB00EE100AB8EE400A1FED621AC0EE010A00EE106AB8EE400ADE
:4071400020EE800ABCEEC00AB8EE400AD4ED3C0A30EE200A84ED3C0A20462BF1E5FA00EE100AB8EE400A00E00FE01FED701AC0EE010A00EE106AB8EE400A20EE800AF0EEC8
:40718000408A2046FFF76AFE2CE0D4ED3B0A00EE105AB8EE400A28EE000A94ED8E1A40EE010AC4ED3B0AD4ED3C0A00EE105A00E097E0B8EE400A28EE000A94ED8E1A40EE52
:4071C000010AC4ED3C0A00EE905AF8EE600A68EE200A94ED8E1A60EE810AB0EE600A2046FFF73CFE94ED3B0A5FED900AB4EEE00AF1EE10FA28DB9C3494ED140A5FED950AC7
:4072000080EE201ABCEEC10A10EE105A206828442060A0689C3CA84205D9D4F8A400401BC4F8A40002E00020C4F8A400D4ED3B0A4FF47A7105FB01F000EE100AB8EE400A03
:4072400030EEC00A84ED3B0A94ED3C0A5FEDAB0AB4EEE00AF1EE10FA42DB00BFA83494ED120A5FEDB00A80EE201ABCEEC10A10EE105A20682844206054F8A809604988426F
:4072800004D3D4F8A800401AC4F8A80054F8AC0F2844206054F8AC095949884204D3D4F8AC00401AC4F8AC0054F8B00F2844206054F8B0095249884204D3D4F8B000401A46
:4072C000C4F8B000D4ED3C0A4E4905FB01F000EE100AB8EE400A30EEC00A84ED3C0A00BF15E0A7B100200190D4F8FC0070B101A9D4F8FC0034F116FC40B101980068016951
:40730000019888470546019834F17DF800BF94F8B802002871D0002001902046FFF79AFD002871D0012852D0022802D003284DD16DE0D4F8000178B101A9D4F8000134F17D
:40734000F1FB48B1019800680169019888470546019834F158F800E000252046FFF748FAF0EE400A94ED3D1A00EE105AB8EE400A00EE201A84ED3D1A94ED3D0A5FEDF50A0E
:40738000B4EEE00AF1EE10FA20DD94ED3D0A5FEDF90A80EE201ABCEEC10A10EE105AD4F8E0022844C4F8E002D4F8A4002844C4F8A400D4ED3D0A4FF47A70684300EE100AE3
:4073C000B8EE400A30EEC00A84ED3D0A38E0D4F80C01D0B1A434A06E0268516A8847BCEEC00A10EE105A2168691AD4F83C020844C4F83C0244F8A45908E02EE0FA592E8742
:407400006466D070A086010019E0002518E0D4F8100190B1A434E06E0268516A8847BCEEC00A10EE105A2168691AD4F83C020844C4F83C0244F8A45900E0002500E000BFB8
:4074400000BFF74800688047C4F8B402F54B0722B521204655F102FC24E0D4F8E00200280EDDF149D4F8B402CFF0F0F940B10020C4F8E002EB4B0722B521204655F1EEFBE2
:40748000B8F1000F0ED000200190D4F8000140B101A9D4F8000134F145FB10B1019833F1B2FF00BF02B0BDEC028BBDE8F0872DE9F0412DED028B044688469FEDDC0AF0EEA3
:4074C000408A0127D4E92E10884206D000BFD44800688047C4F8A00209E0012F07D140F2DC51D4F8A002CFF0B1F900B1002720680321C26A20469047002879D0D4F8040141
:4075000034F1FBFA002873D0D4F804010DF03EFE04286DD0D4F8B800002869D9D4F84402002865D994F8DD02002861D1D4F804010268516A8847BCEEC00A10EE105A5DB377
:40754000A06C48B394ED8D0AB5EEC00AF1EE10FA2CDD94ED120AB8EE400AD4ED8E0A80EE208A022600EE106AF8EEC00AB0EE480A5AF1A8FB00EE905AF8EE600A80EE201AA1
:40758000F0EE418A4FB10121B0EE680A04F520702BF1CEFC84ED9F0A08E00021B0EE680A04F520702BF1C4FC84ED9F0AD4F8040134F143FAD4ED9F0A20EE200AB0EE408A92
:4075C0005AF1A0FABCEEC00A84EDA70AD4F8040134F16EFAD4ED9F0A20EE200AB0EE408A5AF190FABCEEC00A84EDA60A05E0FFE70020C4F89802C4F89C0294F8270100B33C
:40760000D4F8040134F179FAD8B1D4F8040134F136FAB0B1D4F8040134F14AFAB5EEC00AF1EE10FA0DDDD4F89802002809D9D4F89812D4F8A402884203D2D4F89802C4F83E
:40764000A40294F8270100B3D4F8040134F155FAD8B1D4F8040134F1D7F9B0B1D4F8040134F1EBF9B5EEC00AF1EE10FA0DDDD4F89C02002809D9D4F89C12D4F8A4028842C4
:4076800003D9D4F89C02C4F8A402BDEC028BBDE8F08170B504460E46D4F8AC5294EDAA0AB8EE400AB0EE401A94EDAB0AB8EE400AF0EE400AB7EE000A2BF118FC18B1D4F86A
:4076C000A802C4F8AC02D4F8AC02A84205D0554B00227E21204655F1C1FA70BD2DE9F04104460D46164620680121C26A20469047074620680221C26A204690473844A8422E
:407700000ADD04F50B7040F8256005F12201454B0022204655F1A2FABDE8F0812DE9F0432DED028B81B004460E4617461D469FED3F0AB0EE408A4FF4B3792046FFF758F831
:40774000B0EE408A46B1D4F80001A8B9D4F80C0190B9D4F8100178B9002201212046FFF7BDFF0020C4F8A80284F8B8022C4800688047C4F8B00240E1002F7DD1A16901F585
:40778000D270F3F7F2FA012876D0B5F5B37F73D894F8B80240B9B5F5B37F05D9204800688047C4F8B002F3E094F8B802002876D141F28831D4F8B002CFF048F800286ED0C6
:4077C0002046FFF747FB012802D0032868D157E094ED920AB5EEC00AF1EE10FA07D1D4F80C010268116A884784ED920A47E0D4F80C010268116A8847D4ED920A9FED0C1AAD
:4078000070EE810AB4EEE00AF1EE10FA12DD012084F8B802024800688047C4F8B0022EE018A01008BF181708C0D40100000000000000C842D4F80C010268D16A8847F0B954
:40784000206800221146D0F8EC3020469847D4F80C0101680A6B01219047012084F8B802002001230246014600902046FFF7F9FB002084F8B80200E080E0C4F8E00256E0BA
:4078800094ED920AB5EEC00AF1EE10FA09D1D4F810010268116A884784ED920A3DE047E03CE0D4F810010268116A8847D4ED920A1FED211A70EE810AB4EEE00AF1EE10FAEA
:4078C00008DD012084F8B802FE4800688047C4F8B00222E0D4F810010268D16A8847E0B9206800221146D0F8EC3020469847D4F8100101680A6B01219047012084F8B80248
:40790000002001230246014600902046FFF7A9FB002084F8B802C4F8E00208E0012084F8B802E84800688047C4F8B00200BF2FE094F8B802B0B1B5F5B37F13D94FF47A7179
:40794000D4F8B002CEF082FF60B1002084F8B802DC4800688047C4F8B002B7EE000A84ED920A15E094F8B80290B1B5F5B37F0FD2D44800688047C4F8B00209E00020C4F8AF
:40798000E00284F8B802CF4800688047C4F8B002D4F8000168B1D4F800010268116A8847BCEEC00A10EE108A424601212046FFF795FE94F8B802E8B12046FFF74BFAB8B106
:4079C000012813D0022802D0032812D10FE0D4F8000150B1D4F800010268116A884720EE080ABCEEC00A84EDAA0A02E000BF00BF00BF02E00020C4F8A80201B0BDEC028B0C
:407A0000BDE8F0830146D1F84C0270472DE9F0472DED028B044688464FF4FA67A16901F5D270F3F71DFA05460026022D01D0012D12D120462AF1B5FD70B194F8C00210B141
:407A400094F8C80240B9012084F8CA029D4800688047C4F8C40205E01DB120462AF1A1FD00B9012694F8CA0201286ED120462AF1F9FC8146A16901F1300049460AF099FCBF
:407A800000287CD1A069F4F7CBFE8146A069F4F725FE814573D2002E71D12068D0F8A41020468847DFED880AC0EE208A854800688047D4F8C412401A00EE100AF8EE400A1C
:407AC000824890ED000A08EEA00AB0EE408A2046FFF798FF0A21B0FBF1F000EE100AB8EE400AB4EEC80AF1EE10FA0BD22046FFF789FF0A21B0FBF1F000EE100AB8EE400ABE
:407B0000B0EE408AD4F8080133F1F7FFC0B3D4F808010268516A8847F0EE408AD4F8080133F18BFFF4EEC08AF1EE10FA0EDDD4F8F80028F1B5FBDFED660A30EE600AB0EE98
:407B4000408A012084F8CB0226E03DE094F8CB02012821D154F8F80F28F1A2FBB0EE408A20690268516A8847F0EE408A2069F83C33F163FFDFED570A20EE200A01E015E026
:407B80000AE0F4EEC08AF1EE10FA05D29FED520A38EE000AB0EE408AD4F8F80001684F4A0B690121B0EE480A98470DE0002084F8CA0284F8CB02D4F8F8000168474A0B6974
:407BC00000211FEDE60A984784F8C05220462AF1E8FC84F8C802BDEC028BBDE8F087014691F82F01704702460020052903DA02F5C27353F82100704702460020052903DA12
:407C000002F5AE7353F8210070472DE9F04705460F469046002628680D21C26A28469047002870DDD5F8140100286CD0D5F8149100247EE0484633F134FA042803D04846D5
:407C400033F1DDFFC8B134F020FDB0B92146484633F199FA00EE100AB8EE400A9FED201AC0EE010A00EE107AB8EE400A20EE800ABCEEC00A10EE106A00E0002605F5AE70B4
:407C800050F82400B0420AD005F5AE7040F8246004F18501114B0022284654F1DFFF484633F1FFF9042803D0484633F1A8FF58B334F0EBFC40BB2146484633F164FA00EEB6
:407CC000100A0FE018A010080000FA4400441708CDCCCC3D3333733FCDCC4C3DBF1817080050C347B8EE400A1FED031AC0EE010A00EE108AB8EE400A20EE800ABCEEC00A88
:407D000010EE106A02E018E0FFE7002605F5B87050F82400B0420AD005F5B87040F8246004F18A01F94B0022284654F197FF601CC4B2052CFFF67EAF00BFBDE8F0872DE948
:407D4000F0412DED108B82B004460D46B0EE408A16469FEDEF0AF0EE408A9FEDED0A8DED010A2068816E20468847F0EE408A94F8250110B1D4F8FC0048B99FEDE50A8DEDD0
:407D8000010A002211462046FFF7A8FC5FE0D4F8FC0033F134FFB0B3012802D0022842D113E0002D0CD9D4F8FC0033F18AFF00EE100AB8EE400A20EE080A8DED010A03E04C
:407DC0009FEDD30A8DED010A32E0F5EEC08AF1EE10FA19DD94ED100AF8EE400A00EE106AB8EE401A00EE105AB8EE400A21EE000A20EE800ADFEDC70A28EEA01AC0EE010A25
:407E0000CDED010A04E004E09FEDC10A8DED010A0EE0D4F8FC000268116A884720EE080A8DED010A04E09FEDBA0A8DED010A00BF00BFD4F8FC000268116A8847BCEEC00AA3
:407E400010EE107A3A4600212046FFF747FC9DED010A20EE280ABCEEC00A84ED120A002E1ED9002D1CD994ED120AB8EE400ADFEDAA0A20EE200ADFEDA90A60EE200A00EEF3
:407E8000106AB8EE401A00EE105AB8EE400A21EE000A80EE801ABCEEC10A84ED130A01E00020E064A069F6F765FF002876D020680D21C26A2046904700286FDDD4F814015B
:407EC00000286BD02046D4E91221FFF79EFE2068D0F8C4102046884707462046FFF77FFE062852D2DFE800F04F030405065000BF00BF00BF2046FFF772FE80464146204642
:407F0000FFF77AFE00282CD920462AF107FC002827D920462AF102FC00EE100AF8EE400A2046FFF75CFE804641462046FFF75BFE00EE100AB8EE401A2046FFF750FE804613
:407F400041462046FFF758FE00EE100AB8EE400AC1EE001A20EEA10ABCEEC00A10EE107A10E02046FFF73BFE804641462046FFF73AFE002805D9002120462AF154F80746AB
:407F800000E0002701E000BF00BF00BF20685F4A3946D0F8C8302046984700BFB5EEC08AF1EE10FA3BD018EE100AD7F03DFD41EC1D0B9FED5B0B53EC102BD7F011FB41EC65
:407FC0001C0B9FED590B53EC102BD7F009FB41EC1A0B2846D7F0F1FA41EC1C0B3046D7F0ECFA41EC1E0B206CD7F0E7FA41EC1F0B53EC1E2BD7F0F4FA41EC1D0B53EC1C2B43
:40800000D7F0EEFA41EC1B0B53EC1A2BD7F0E4F841EC190BD7F0A4FAC4F8A40202E00020C4F8A40202B0BDEC108BBDE8F0812DE9F04104460E46174620462BF1DAF884ED88
:408040008D0ADEB90020E064A064002511E0D4F8FC0068B1D4F8FC000268116A8847BCEEC00A10EE108AE9B242462046FFF736FB6D1C94F82501A842E9D86FE020462AF185
:40808000E6F9042802D0152857D10FE094ED8D0A84ED8E0AD4F84422D4ED8E0AB0EE600A2046D4F8B810FFF74AFE56E094ED8D0A84ED8E0AD4F84422D4ED8E0AB0EE600AB9
:4080C0002046D4F8B810FFF73AFE206CE8B1D4F8B800D0B194ED120AB8EE400ADFED0E0A20EE200ADFED0D0A20EE201A94ED100AB8EE400AC1EE000A94ED2E0AB8EE400A6D
:4081000080EE801A84ED8F1A16E011E0BF1817080000000020BCBE4C0000C8420024744900000000000059400000000080842E411FED090A84ED8F0A0FE0B7EE000A84ED2B
:408140008E0AD4F84422D4ED8E0AB0EE600A2046D4F8B810FFF7F3FD00BF00BF3B4600225521204654F17AFD3B4600225621204654F174FDBDE8F081014691F8CF02704797
:4081800011B52DED028B8BB000200A9001200990089000200790069001200590002004900D98C06E0290CEF041FB0390FE48006880470D99C8660D98D0F8B810C0F8BC1060
:4081C0000D982AF14FF902900D9880693030019002990AF0EEF80D99C1F8B8000D9880690290F6F76DFE0D99C1F84402002007900D9890F82501002812DD0D98D0F8FC002D
:4082000010B903200A900BE00D98D0F8FC00029033F173FC10B901200A9001E001200790002006900D9890F8250100281EDD0D98FFF7A2FFD0B10D98D0F8000148B10D982D
:40824000D0F80001029033F158FC78B1012006900CE00D98D0F80C0110B10120069005E00D98D0F8100108B1012006900D9890F86C02012808D10D9800684069CB4A002111
:408280000290029B0D9898470D982AF122FF079868B10D980068806E029002990D988847B5EEC00AF1EE10FA01DD012000E000200490BE4A04990D98FFF7B9FEBB490D984D
:4082C000FFF7A4FB0D98D0F8440202900D98D0F8B80001900246029B06990D98FFF71EFA0D982AF1B4F8022804D0032803D0142822D101E000BF00BF002002900D98806981
:40830000303002A9019009F077FBA0B10D9890F8DC00012808D10D98D0F8A4020146019002982FF165FD06E00D98806C0146019002982FF15DFD00E000BF00BF9B490D9889
:408340002AF17CFF99490D98FFF7A3F997490D982AF1A0FF0D982BF113F894490D98FFF7A6F80D980068C06A03210290029A0D989047002810DD0D98D0F8040160B10D98EB
:40838000D0F8040102900CF001FF042804D1874A00210D982AF1FFFA84480090069BDDE903210D98FEF75DFE0D98D0F8B8000246029003990D982AF101FE0D98D0F84401CE
:4083C0004FF4FA710290CEF041FA00286ED00D98D0F8A40002900D980068D0F8EC00734A0190DDE901310D9898470D98D0F8A8006E4A014602900D982AF1E0FC0D98D0F801
:40840000AC006A4A014602900D982AF191FC0D98D0F8B000654A014602900D982AF1EDFC0D98D0F89C00614A014602900D982AF1ACFC0D982AF10BF8162804D00D982AF1DE
:4084400006F815282CD10D980068C06A0D210290029A0D989047002822DD0D98D0F81401F0B1012002900FE00D9800F5E070029950F821004D4B024601900D98FEF7C2FC12
:408480000298401CC0B2029002980528ECDB0D98D0F81802454A014602900D98FEF797FC4148006880470D99C1F844013F490D98FEF74FFB0D9890F8D30040B10D988069D1
:4084C0000290F6F783FD012801D1012100E000210D9880F840120D9890F8D30040B10D9880690290F6F772FD022801D1012100E000210D9880F841120D982AF1F5F90990AD
:408500000D98006C08B9012000E000200590049808B1059808B1012000E0002008900D9890F82901012815D10D9890EDA90AB8EE400A8DED020AD0F8180101900D98D0F8BF
:40854000180100684069002100909DED020ADDE9002090470D9890F82B01012816D10D98D0F8200102900D98D0F80801009033F164FA8DED010A02980068406900210090DB
:408580009DED010A009A0298904700BF0D9890F82A01012854D10D9890F82701C8B30D98D0F80401029003E018A01008BF18170833F1A3FA68B30D98D0F80401029033F135
:4085C00023FA30B30D98D0F80401029033F135FA0D98D0ED300AF8EE600AB4EEE00AF1EE10FA17D20D98D0F81C0102900D98D0F80401009033F121FA8DED010A02980068F6
:408600004069002100909DED010A009A0298904716E0FFE70D9890ED300AB8EE400A8DED020AD0F81C0101900D98D0F81C0100684069002100909DED020ADDE9002090477D
:408640000D9890F8DB00132881F04A81DFE810F013003101DF01E0016F0048090F035202CD03E7046105AB056006A9068A074008C0084809BA040D9890F83101B0B1002111
:408680000D98C0F834110D980068D0F89400029002990D988847032804D109210D98FEF7F4F903E000210D98FEF7EFF90D9829F178FF00B3FB4800688047012804D112214B
:4086C0000D9880F8DB1025E00D9890F8CB00012804D109210D9880F8DB101BE00D98806900F5D2700290F2F740FB022804D109210D9880F8DB100DE00D9890F8DC0001287F
:4087000004D10C210D9880F8DB1003E001210D9880F8DB100D9890F8DB1090F83001814203D000210D9880F8CB1001F0EAB80D9890F8310118B100210D98C0F834110D987F
:4087400029F12FFF20B900210D9880F8DB102BE0D44800688047012804D112210D9880F8DB1021E00D9890F8DC00012804D10C210D9880F8DB1017E00D9890F8400220B1AC
:4087800006210D9880F8DB100EE00D9890F8410220B107210D9880F8DB1005E0099818B901210D9880F8DB100D9890F8DB1090F8300181427CD10D98D0F8F800029027F1BA
:4087C00019FD042807D00D98D0F8F800029027F111FD012804D100210D98FEF756F967E00D9890F83101A8B30D98D0F8F800029027F100FD03282ED10D98D0F8F80002900D
:4088000027F16FFDB5EEC00AF1EE10FA50DD0D98D0F8F800029027F164FDB0EE408A0D98D0F8F800029027F13BFDB4EEC08AF1EE10FA0AD30D98D0F8F800029027F130FD24
:40884000B5EEC00AF1EE10FA32D108210D98FEF71CF92DE0FFE70D98D0F8F800029027F1C9FC03280CD10D9890F8CD0218B90D9890F8CC0220B10A210D98FEF706F917E0A4
:408880000D9890F8CA00012804D101210D98FEF7FCF80DE00D9890F8C900012804D102210D98FEF7F2F803E005210D98FEF7EDF83BE70D9890F8310118B100210D98C0F83B
:4088C00034110D9829F16DFE20B900210D9880F8DB103DE0734800688047012804D112210D9880F8DB1033E00D9890F8DC00012804D10C210D9880F8DB1029E0099820B1FD
:4089000004210D9880F8DB1022E00D9890F8400220B106210D9880F8DB1019E00D9890F8410220B107210D9880F8DB1010E00D9890F8CD0220B103210D9880F8DB1007E05F
:408940000D9890F8CC0218B102210D9880F8DB100D9890F8DB1090F83001814252D10D98D0F8E80028B10D98D0F8E800029029F1D3FA0D9890F8310158B30D98D0F8F80086
:40898000029027F137FC042823D10D98D0F8F800029027F185FCB5EEC00AF1EE10FA18D80D9890F8CD00A0B90D98D0F8F800029027F197FCB5EEC00AF1EE10FA04DD08218F
:4089C0000D98FEF762F821E007210D98FEF75DF81CE00D9890F8CA00012804D101210D98FEF753F812E00D9890F8C900012804D102210D98FEF749F808E005210D98FEF7E7
:408A000044F803E001210D98FEF768F88DE600BF0D9890F8310118B100210D98C0F834110D9829F1BEFD20B900210D9880F8DB1042E01C4800688047012804D112210D98D7
:408A400080F8DB1038E00D9890F8DC00012804D10D210D9880F8DB102EE00D9890F8400220B106210D9880F8DB1025E00D9890F8410220B107210D9880F8DB101CE00D98AA
:408A800090F8CD0220B103210D9880F8DB1013E00D9890F8CC0238B102210D9880F8DB100AE00000B00000200D9890F8CA0018B901210D9880F8DB100D9890F8301190F8BE
:408AC000DB00814211D10D9890F8CD0218B90D9890F8CC0220B10A210D98FDF7D6FF08E005210D98FDF7D1FF03E000210D98FDF7F5FF1AE60D9890F8310118B100210D98CE
:408B0000C0F834110D9829F14CFD20B900210D9880F8DB1021E0F84800688047012804D112210D9880F8DB1017E00D9890F8DC0001280AD10D9890F8410208B1089860B1A7
:408B40000C210D9880F8DB1007E00D9890F8410218B901210D9880F8DB100D9890F8DB1090F8300181427DD10D9890F8DC00012832D10D9890F8D90070B30D9890F82A01D6
:408B800002900D98D0F81C0101900146029A0D98FDF7C7FFF8B106210D98FDF776FF0D98D0F81C0102900D98D0F81C010068C06A0190DDE90110884704460D98D0F80401BD
:408BC000029032F1ACFF844250D2CC4B072205210D9854F143F849E00D98D0F8F800029027F108FB032822D10D98D0F8F800029027F177FBB5EEC00AF1EE10FA17D00D98E6
:408C0000D0F8F800029027F16CFBB0EE408A0D98D0F8F800029027F143FBB4EEC08AF1EE10FA04D208210D98FDF72FFF1EE00D98D0F8F800029027F1DDFA03280DD10D9881
:408C400090F8CD0218B90D9890F8CC0228B10A210D98FDF71AFF09E004E000210D98FDF714FF03E000210D98FDF738FF5DE50D9890F8310118B100210D98C0F834110D98DB
:408C800029F18FFC20B900210D9880F8DB1021E0994800688047012804D112210D9880F8DB1017E00D9890F8DC0001280AD10D9890F8400208B1089860B10C210D9880F89C
:408CC000DB1007E00D9890F8400218B901210D9880F8DB100D9890F8DB1090F8300181427ED10D9890F8DC00012833D10D9890F8D90070B30D9890F82A0102900D98D0F89F
:408D00001C0101900146029A0D98FDF70AFFF8B106210D98FDF7B9FE0D98D0F81C0102900D98D0F81C010068C06A0190DDE90110884704460D98D0F80401029032F1EFFE13
:408D4000844251D26D4B072205210D9853F186FF4AE0FFE70D98D0F8F800029027F14AFA032822D10D98D0F8F800029027F1B9FAB5EEC00AF1EE10FA17D00D98D0F8F800B0
:408D8000029027F1AEFAB0EE408A0D98D0F8F800029027F185FAB4EEC08AF1EE10FA04D208210D98FDF771FE1EE00D98D0F8F800029027F11FFA03280DD10D9890F8CD0264
:408DC00018B90D9890F8CC0228B10A210D98FDF75CFE09E004E000210D98FDF756FE03E000210D98FDF77AFE9FE40D9829F1D9FB20B900210D9880F8DB1023E03E480068B7
:408E00008047012804D112210D9880F8DB1019E00D9890F8DC00012810D1099848B1089838B90D9890F8400218B90D9890F8410240B10C210D9880F8DB1003E004210D9878
:408E400080F8DB100D9890F8DB1090F83001814250D10D9890F8D900F0B30D98D0F80401D0B30D98D0F8040102900CF08FF998B30D98806900F5D2700290F1F7F1FF012811
:408E80003ED00D98806900F5D2700290F1F7E8FF022835D00D9890F82A0102900D98D0F81C0101900146029A0D98FDF73AFE08B306210D98FDF7E9FD0D98D0F81C01029019
:408EC0000D98D0F81C010068C06A0190DDE90110884704460D9800E012E0D0F80401029032F11DFE84426CD2044B072205210D9853F1B4FE65E00000B0000020BF18170879
:408F00000D98D0F8F800029027F174F903283FD10D98D0F8F800029027F1E3F9B5EEC00AF1EE10FA34DD0D98D0F8F800029027F1D8F9B0EE408A0D98D0F8F800029027F1D1
:408F4000AFF9B4EEC08AF1EE10FA0AD30D98D0F8F800029027F1A4F9B5EEC00AF1EE10FA16D10D98806900F5D2700290F1F778FF01280DD00D98806900F5D2700290F1F7B3
:408F80006FFF022804D008210D98FDF77EFD18E00D98D0F8F800029027F12CF903280CD10D9890F8CD0218B90D9890F8CC0220B10A210D98FDF769FD03E000210D98FDF774
:408FC00064FDCEE20D9890F83101B0B100210D98C0F834110D980068D0F89400029002990D988847032804D109210D98FDF74DFD03E000210D98FDF748FD0D9829F1D1FA5A
:4090000020B900210D9880F8DB1007E0FC480068804718B909210D9880F8DB10A1E20D9890F83101D8B100210D98C0F834110D980068D0F89400029002990D98884703286E
:4090400004D109210D98FDF720FD03E000210D98FDF71BFD00210D9880F8CC1015E00D98806900F5D2700290F1F77FFE08B9012000E000200D9991F8CC10084308B10121A8
:4090800000E000210D9880F8CC100D9829F189FA20B900210D9880F8DB102EE00D98806900F5D2700290F1F760FE022825D0D44800688047012804D112210D9880F8DB1024
:4090C0001BE00D98806900F5D2700290F1F74DFE012812D10D9890F8CC0001280DD10D9890F8DC00012804D10C210D9880F8DB1003E001210D9880F8DB100D9890F8DB107E
:4091000090F83001814203D000210D98FDF7E6FCF7E30D9890F83101B0B100210D98C0F834110D980068D0F89400029002990D988847032804D109210D98FDF7A6FC03E095
:4091400000210D98FDF7A1FC0D9829F12AFA20B900210D9880F8DB1019E0A94800688047012804D112210D9880F8DB100FE00D9890F8DC00012806D1049840B10C210D980A
:4091800080F8DB1003E001210D9880F8DB100D9890F8DB1090F83001814203D000210D98FDF79CFCADE30D9890F8310118B100210D98C0F834110D9829F1F3F920B9002166
:4091C0000D9880F8DB1019E08D4800688047012804D112210D9880F8DB100FE00D9890F8DC00012806D1059840B90C210D9880F8DB1003E001210D9880F8DB100D9890F834
:40920000301190F8DB00814231D10D9890F8D90070B30D9890F82A0102900D98D0F81C0101900146029A0D98FDF77BFCF8B106210D98FDF72AFC0D98D0F81C0102900D9854
:40924000D0F81C010068C06A0190DDE90110884704460D98D0F80401029032F160FC844255D2684B072205210D9853F1F7FC4EE00D98D0F8F800029026F1BCFF03282DD188
:409280000D98D0F8F800029027F12BF8B5EEC00AF1EE10FA22DD0D98D0F8F800029027F120F8B0EE408A0D98D0F8F800029026F1F7FFB4EEC08AF1EE10FA0AD30D98D0F875
:4092C000F800029026F1ECFFB5EEC00AF1EE10FA04D108210D98FDF7D8FB18E00D98D0F8F800029026F186FF03280CD10D9890F8CD0218B90D9890F8CC0220B10A210D9826
:40930000FDF7C3FB03E000210D98FDF7BEFBF8E20D9829F146F920B900210D9880F8DB103EE0374800688047012804D112210D9880F8DB1034E00D9890F8DC0001282BD104
:40934000049820B90A210D9880F8DB1028E0059820B10B210D9880F8DB1021E00D9890F8400220B106210D9880F8DB1018E00D9890F8410220B107210D9880F8DB100FE0D3
:40938000099820B108210D9880F8DB1008E010210D9880F8DB1003E001210D9880F8DB10AFE20D9890F8310118B100210D98C0F834110D9829F1F5F820B900210D9880F89D
:4093C000DB104FE00E4800688047012804D112210D9880F8DB1045E00D9890F8DC0001283CD10D9890F8400228B90D9890F8410208B9089840B10C210D9880F8DB1031E0D9
:40940000B0000020BF181708099820B10F210D9880F8DB1026E00D9890F8CC0210B30D98D0ED940A9FEDF91A80EE810AF7EE000A70EE200A90EDA90AB8EE400A60EE800AF1
:4094400090ED120AB8EE400AF4EEC00AF1EE10FA08DB0E210D9880F8DB1003E001210D9880F8DB100D9890F8DB1090F8300181426DD10D98D0F8E80028B10D98D0F8E80052
:40948000029028F149FD0D9890F8310138B30D98D0F8F800029026F1ADFE04281FD10D98D0F8F800029026F1FBFEB5EEC00AF1EE10FA14D80D98D0F8F800029026F111FF35
:4094C000B5EEC00AF1EE10FA04DD08210D98FDF7DCFA46E007210D98FDF7D7FA41E00D98D0F8B80068B30D9890F8290102900D98D0F8180101900146029A0D98FDF711FBFC
:4095000000B306210D98FDF7C0FA0D98D0F8180102900D98D0F818010068C06A0190DDE90110884704460D98D0F8FC00029032F1F6FA844215D2B64B072205210D9853F159
:409540008DFB0EE000210D98FDF79FFA09E001210D98FDF7C3FAAF48006880470D99C1F83401CEE10D9890F8310118B100210D98C0F834110D9829F114F820B900210D9803
:4095800080F8DB1064E0A44800688047012804D112210D9880F8DB105AE00D9890F8DC00012851D10D9890F8400238B90D9890F8410218B9089808B9099820B10C210D98DC
:4095C00080F8DB1044E00D9890F82801C0B10D98D0F80801029032F190FA88B10D98D0F80801029032F110FA50B10D98D0F80801029032F122FAB5EEC00AF1EE10FA04D187
:409600000D210D9880F8DB1022E00D98D0ED940A9FED7E1A80EE810AF7EE000A70EE200A90EDA90AB8EE400A60EE800A90ED120AB8EE400AF4EEC00AF1EE10FA08D20D2140
:409640000D9880F8DB1003E001210D9880F8DB100D9890F8DB1090F83001814233D10D9890F82B0102900D98D0F8200101900146029A0D98FDF755FA00B306210D98FDF7F5
:4096800004FA0D98D0F8200102900D98D0F820010068C06A0190DDE90110884704460D98D0F80801029032F13AFA84420FD2584B072205210D9853F1D1FA08E000210D9891
:4096C000FDF7E3F903E001210D98FDF707FA18E10D9890F8310128B14E48006880470D99C1F838010D9828F15CFF20B900210D9880F8DB1042E0484800688047012804D173
:4097000012210D9880F8DB1038E00D9890F8DC0001282FD1099820B90D210D9880F8DB102CE00D98D0F84001F8B10D98D0F840016421484302900D98D0F83801019002996F
:40974000CDF084F888B90D9890F8CD0268B90D9890F8400248B90D9890F8410228B9089818B90D9890F8CC0240B10C210D9880F8DB1003E001210D9880F8DB100D9890F8C5
:40978000DB1090F83001814219D10D98D0F8F800029026F12FFD03280CD10D9890F8CD0218B90D9890F8CC0220B10A210D98FDF76CF90CE00B210D98FDF767F907E0052136
:4097C0000D98FDF762F901210D98FDF787F998E00D9890F8310128B10E48006880470D99C1F838010D9828F1DCFE20B900210D9880F8DB104FE008480068804701280DD11E
:4098000012210D9880F8DB1045E000000000C842BF18170818A01008B00000200D9890F8DC00012833D10D9890F8400238B90D9890F8410218B9089808B9099820B10C2151
:409840000D9880F8DB1026E00D98D0F83C01C8B10D98D0F83C016421484302900D98D0F8380101900299CCF0F1FF58B90D98D0F8340138B10D98D0F83401FE490290CCF01A
:40988000E5FF40B10D210D9880F8DB1003E001210D9880F8DB100D9890F8DB1090F83001814219D10D98D0F8F800029026F1A2FC03280CD10D9890F8CD0218B90D9890F864
:4098C000CC0220B10A210D98FDF7DFF807E005210D98FDF7DAF802E000210D98816610E0002211460D9828F160FE00210D98FDF7CCF800210D98C0F834110D9880F8DB1059
:4099000000BF00BF00210D9880F831110D9890F8DB1090F83001814215D00D980068006D029002990D98884701210D9880F831110D9890F8DB1080F83011CF4B07221A21C5
:409940000D9853F18BF90A980BB0BDEC028B18BD90ED8F0A70470146D1F81C0270472DE9F0472DED028B04460D46164600272046FFF7F1FFA84222D0C4F81C5233463A4601
:409980008021204653F16AF9B84614E0D4F8000168B12046D4F80091FCF72AFFB0EE408AD9F80000B44982694846904700BF08F1010000F0FF0894F826014045E6DC384694
:4099C000BDEC028BBDE8F087014691F8200270472DE9F0472DED028B04460D46164600272046FFF7F1FFA84222D084F8205233463A468121204653F131F9B84614E0D4F815
:409A0000000168B12046D4F80091FCF7F1FEB0EE408AD9F80000984982694846904700BF08F1010000F0FF0894F826014045E6DC3846BDEC028BBDE8F0872DE9F0410446F2
:409A40000D461646002794F8D002A84207D084F8D05233463A46AE21204653F1FFF83846BDE8F08138B504462046FEF785FB10B32046FDF7EFF9012804D02046FDF7EAF905
:409A8000032818D1206800221146D0F8EC3020469847012084F8B802774801230022114600902046FDF7DDFA9FED740A84ED920A002084F8B80238BD0146D1F8BC0270470D
:409AC0002DE9F04104460D4616460027D4F8BC02A84207D0C4F8BC5233463A467F21204653F1BCF83846BDE8F08190ED9F0A7047024602F50B7050F821007047014691F8D8
:409B0000280270472DE9F0472DED028B04460D46164600272068816D20468847A8422AD084F8285233463A462121204653F196F8B84615E0D4F8FC0070B1D4F8FC9020687C
:409B4000816E20468847B0EE408AD9F800004A4982694846904700BF08F1010000F0FF0894F825014045E5DCD4F8E80018B1D4F8E80027F12FFE3846BDEC028BBDE8F087B7
:409B80000146D1F8240270472DE9F0472DED028B04460D46164600272068016E20468847A8422AD0C4F8245233463A462021204653F154F8B84615E0D4F8FC0070B1D4F88A
:409BC000FC902068816E20468847B0EE408AD9F80000294982694846904700BF08F1010000F0FF0894F825014045E5DCD4F8E80018B1D4F8E80027F1EDFD3846BDEC028BA3
:409C0000BDE8F08700B503469FED1C0AB0EE401AD3F8240268B193F828121846FCF7ABFDD3ED890AF8EE600AC0EE201AB0EE611A03E09FED120AB0EE401AB0EE410A00BDCB
:409C40000146D1F8400170472DE9F04104460D4616460027D4F84001A84207D0C4F8405133463A464221204652F1F8FF3846BDE8F0810000C0D40100BF181708000000003F
:409C80000146D1F83C0170472DE9F04104460D4616460027D4F83C01A84207D0C4F83C5133463A464321204652F1D8FF3846BDE8F08190ED940A704770B52DED028B0446CD
:409CC000B0EE408A0D4600269FEDF70AB4EEC08AF1EE10FA04DD02269FEDF30AB0EE408A94F8290150B1D4F8180138B1D4F818010168CA692946B0EE480A904794F82A0134
:409D000050B1D4F81C0138B1D4F81C010168CA692946B0EE480A904794F82B0150B1D4F8200138B1D4F820010168CA692946B0EE480A904794ED940AB4EE480AF1EE10FA4B
:409D400007D084ED948A2B4632464821204652F185FF3046BDEC028B70BD90ED950A704770B52DED028B0446B0EE408A0D4600269FEDCE0AB4EEC08AF1EE10FA04DD022619
:409D80009FEDCA0AB0EE408AB5EEC08AF1EE10FA04D203261FED470AB0EE408A94F82401012809D1D4F8F80030B12946B0EE480AD4F8F80026F124FB94ED950AB4EE480A7B
:409DC000F1EE10FA07D084ED958A2B4632465121204652F143FF3046BDEC028B70BD31B1012907D0022908D003290CD108E090ED960A08E090ED970A05E090ED980A02E014
:409E000090ED990A00BF00BF70472DE9F0412DED028B0446B0EE408A0E46154600279FEDA30AB4EEC08AF1EE10FA04DD02279FED9F0AB0EE408AB5EEC08AF1EE10FA04D2F6
:409E400003271FED720AB0EE408A36B1012E4AD0022E7DD0032E7CD1D4E0D4F8180170B194F8290158B1D4F81801EFF72FF830B92946B0EE480AD4F8180127F12CFCD4F8F9
:409E80001C0170B194F82A0158B1D4F81C01EFF71DF830B92946B0EE480AD4F81C0127F11AFCD4F8200170B194F82B0158B1D4F82001EFF70BF830B92946B0EE480AD4F8A8
:409EC000200127F108FC94ED960AB4EE480AF1EE10FA07D084ED968A2B463A464421204652F1BCFEE5E0D4F8180170B194F8290158B1D4F81801EEF7E9FF30B92946B0EED4
:409F0000480AD4F8180127F104FCD4F81C0170B194F82A0158B1D4F81C01EEF7D7FF30B92946B0EE480AD4F81C0127F1F2FBD4F8200188B194F82B0170B1D4F82001EEF75D
:409F4000C5FF48B92946B0EE480AD4F8200101E012E0ADE027F1DDFB94ED970AB4EE480AF1EE10FA07D084ED978A2B463A464521204652F173FE9CE0D4F8180170B194F899
:409F8000290158B1D4F81801EEF7A0FF30B92946B0EE480AD4F8180127F1D9FBD4F81C0170B194F82A0158B1D4F81C01EEF78EFF30B92946B0EE480AD4F81C0127F1C7FBBC
:409FC000D4F8200170B194F82B0158B1D4F82001EEF77CFF30B92946B0EE480AD4F8200127F1B5FB94ED980AB4EE480AF1EE10FA07D084ED988A2B463A464621204652F1DD
:40A000002DFE56E0D4F8180170B194F8290158B1D4F81801EEF75AFF30B92946B0EE480AD4F8180127F1B1FBD4F81C01A0B194F82A0188B1D4F81C01EEF748FF60B9B2EEEE
:40A04000040AC8EE000AF0EE608A2946B0EE680AD4F81C0127F199FBD4F82001A0B194F82B0188B1D4F82001EEF730FF60B9B1EE040AC8EE000AF0EE608A2946B0EE680A39
:40A08000D4F8200127F181FB94ED990AB4EE480AF1EE10FA07D084ED998A2B463A464721204652F1DBFD04E00000C84200007A4400BF00BF3846BDEC028BBDE8F08101469E
:40A0C00091F86D0270472DE9F04104460D461646002794F86D02A84207D084F86D5233463A464B21204652F1B9FD3846BDE8F08190ED9C0A70472DE9F0412DED028B0446E9
:40A10000B0EE408A0D46002694ED9C0AB4EE480AF1EE10FA16D0FE4890ED000AB4EEC80AF1EE10FA02D884ED9C8A05E0F84890ED000A84ED9C0A03262B4632464F2120460E
:40A1400052F18CFD00270DE0D4F8F80040B1D4ED9C0AB0EE600A2946D4F8F80026F119F9781CC7B294F82401B842EDDC3046BDEC028BBDE8F08190ED9D0A70472DE9F0411A
:40A180002DED028B0446B0EE408A0D46002694ED9D0AB4EE480AF1EE10FA07D084ED9D8A2B4632464E21204652F158FD00270BE0D4F8F80030B12946B0EE480AD4F8F80029
:40A1C00026F1B0F8781CC7B294F82401B842EFDC3046BDEC028BBDE8F08190ED9E0A70472DE9F0412DED028B0446B0EE408A0D46002694ED9E0AB4EE480AF1EE10FA07D089
:40A2000084ED9E8A2B4632465021204652F126FD00270BE0D4F8F80030B12946B0EE480AD4F8F80026F160F8781CC7B294F82401B842EFDC3046BDEC028BBDE8F08101468A
:40A24000D1F8680270472DE9F04104460D461646072794F86D02012802D002281BD100BF002794F82401012808D1D4F8F80028B132462946D4F8F800EEF745FDD4F868023C
:40A28000A84207D0C4F8685233463A465221204652F1E4FC0AE0D4F86802A84205D033463A465221204652F1D9FC00BF00BF3846BDE8F08110B50346072021B9012483F8E8
:40A2C0006C42002000BF00BF10BD2DE9F04104460D4616460027D4F84C02A84207D0C4F84C5233463A468221204652F1B7FC3846BDE8F0812DE9F04104460D4616460027B6
:40A3000094F82F01A84207D084F82F5133463A468321204652F1A2FC3846BDE8F0812DE9F04105460C46164698460727052C11DA002705F5C27050F82400B0420AD005F53F
:40A34000C27040F8246004F18F0143463A46284652F184FC3846BDE8F0812DE9F04104460D4616461F464FF00708204627F1E9FE012810D1204627F173FE02280BD02046E0
:40A3800027F16EFE032806D03B46324629462046FFF7C5FF80464046BDE8F08102460020052903DA02F5CC7353F8210070472DE9F04105460C46164698460727052C11DAFA
:40A3C000002705F5CC7050F82400B0420AD005F5CC7040F8246004F1940143463A46284652F13CFC3846BDE8F08130B503460020052909DA032A07DA01EB410503F5EA74D1
:40A4000004EB850454F8220030BD2DE9F04706460C4615461F46DDF820904FF00708052C34DA032D32DA4FF0000804EB440106F5EA7000EB810050F82500B84226D004EBC8
:40A44000440106F5EA7000EB810040F8257025B1012D0AD0022D18D10FE004F199014B464246304652F1FAFB0FE004F19E014B464246304652F1F2FB07E004F1A3014B467B
:40A480004246304652F1EAFB00BF00BF4046BDE8F08702460020052903DA02F5D67353F8210070470146D1F81402704702460020052903DA02F5B87353F8210070470146A4
:40A4C000D1F8AC0270470146D1F8A402704710B50446204628F1ACFC08B9012010BD0020FCE72DE9F04104460D461646002794F8CF02A84213D084F8CF5294F8CF02012825
:40A5000004D1324602212046FFF797FA334601E0004417083A46AD21204652F19FFB3846BDE8F081014691F8DC027047014691F8D20270472DE9F04104460D4616460027B5
:40A5400094F8D202A84207D084F8D25233463A46AF21204652F182FB3846BDE8F0810146D1F8D80270472DE9F04104460D4616460027D4F8D802A84207D0C4F8D8523346C9
:40A580003A46B021204652F169FB3846BDE8F0810146D1F8D40270472DE9F04104460D4616460027D4F8D402A84207D0C4F8D45233463A46B121204652F150FB3846BDE87E
:40A5C000F081014691F8D10270472DE9F04104460D461646002794F8D102A84207D084F8D15233463A46B221204652F137FB3846BDE8F081014691F8DD0270472DE9F04182
:40A6000004460D461646002794F8DD02A84207D084F8DD5233463A46B321204652F11EFB3846BDE8F081014691F8DE0270472DE9F04104460F461546002684F8DE722B46F5
:40A640003246B421204652F109FB3046BDE8F08110B5044694F82501002809DDD4F8FC0030B1D4F8FC0031F1CAFA08B1012010BD0020FCE70146D1F8E00270472DE9F04194
:40A6800004460D4616460027D4F8E002A84207D0C4F8E05233463A46B521204652F1DEFA3846BDE8F081000010B50446204627F15AFE002004F58E74A0700120E070F74879
:40A6C0000068804760600020A060E060F34800688047A0610020E061082084F82000002060629FEDEF0A84ED0A0A9FEDED0A84ED0B0A84F8300084F83100606384F8680086
:40A70000A4F58E74002140F285100155204627F19EFE062802D0072813D107E0002084F88601062140F28710015512E0012084F88601042140F287100155DA48C4F8C000CB
:40A7400007E0062084F88601062140F28710015500BF00BF2068D44A00210369204698472068D14A01210369204698479FEDCC0A84ED680A002009E09FEDC90A04F5D2712E
:40A7800001EB800181ED000A411CC8B20528F3DB00214FF4DC700155401C0155002004F5DE742060BD480068804760600020A06020736073A073E07320746074A074E0748F
:40A7C000B6480068804760619FEDB50A84ED060AA4F5DE7410BDF8B504460F4615461E462B46012239462046009627F111FD0446AE48FC3444F8FC0C00F5807044F8F00CD6
:40A80000103044F8EC0C002044F8100C44F80C0C44F8080C44F8040C20606060A060E0602061606120766076A076E07620776077A077E07784F8200084F82100FC3C2046EF
:40A84000FFF732FF23462A469949204652F191F92046F8BD70B504469448206000F58070E0601030206100250BE0D4F8EC0038B1D4F8EC0020B1D4F8EC0002685168884713
:40A880006D1C94F81401A842EFD800250BE0D4F8F00038B1D4F8F00020B1D4F8F0000268516888476D1C94F81501A842EFD800250BE0D4F8F40038B1D4F8F40020B1D4F8DB
:40A8C000F4000268516888476D1C94F81601A842EFD800250BE0D4F8040138B1D4F8040120B1D4F804010268516888476D1C94F81A01A842EFD800250BE0D4F8080138B1B7
:40A90000D4F8080120B1D4F808010268516888476D1C94F81B01A842EFD800250BE0D4F80C0138B1D4F80C0120B1D4F80C010268516888476D1C94F81C01A842EFD8002579
:40A940000BE0D4F8100138B1D4F8100120B1D4F810010268516888476D1C94F81D01A842EFD8204627F190FC0446204670BD70B504462046FFF76EFF054657F1D3F870BD1B
:40A9800010B50446103C2046FFF7F1FF10BD10B504460C3C2046FFF7EAFF10BD10B50446103C2046FFF756FF10BD10B504460C3C2046FFF74FFF10BD70B50546012406E098
:40A9C000394B00222146284652F148F9641C7D2CF6D37E2406E0344B00222146284652F13DF9641C8B2CF6D370BD2DE9F0412DED028B0446B0EE408A0D46002694ED670AB7
:40AA0000B4EE480AF1EE10FA07D084ED678A2B4632468921204652F121F900270BE0D4F8F00030B12946B0EE480AD4F8F00025F15BFC781CC7B294F81501B842EFDC304689
:40AA4000BDEC028BBDE8F0812DE9F0412DED028B0446B0EE408A0D46002694ED630AB4EE480AF1EE10FA16D0124890ED000AB4EEC80AF1EE10FA02D884ED638A05E00D4810
:40AA800090ED000A84ED630A03262B4632468821204652F1E3F800271CE0000018A0100800000000549A3400B51817084C9F1708CD31140800441708D4F8F00040B1D4EDFC
:40AAC000630AB0EE600A2946D4F8F00025F161FC781CC7B294F81501B842EDDC3046BDEC028BBDE8F0812DE9F0412DED028B0446B0EE408A0D46002694ED650AB4EE480A12
:40AB0000F1EE10FA07D084ED658A2B4632468721204652F1A3F800270BE0D4F8F00030B12946B0EE480AD4F8F00025F1FBFB781CC7B294F81501B842EFDC3046BDEC028B2A
:40AB4000BDE8F08170B504460D46164615B1012D7AD1A6E0206832460021036F20469847206832460021836F2046984720683146B0EE080AD0F880202046904794F8860145
:40AB800005287DD2DFE800F0412203616200206831469FEDFE0AD0F8A8202046904720683146B0EE080AD0F8A02020469047206831461FED450AD0F8B020204690472068AE
:40ABC0003246294643692046984761E0206831469FEDEE0AD0F8A8202046904720683146B0EE080AD0F8A02020469047206831461FED550AD0F8B020204690472068324639
:40AC0000294643692046984742E0206831469FEDDF0AD0F8A82020469047206831469FEDDC0AD0F8A02020469047206831461FED640AD0F8B020204690472068324629465E
:40AC400043692046984723E0A4E000BF206831469FEDD00AD0F8A8202046904720683146B3EE0E0AD0F8A02020469047206831461FED750AD0F8B02020469047206800E027
:40AC800005E03246294643692046984700E000BF00BFC14B00224FF6FF71204651F1DEFF78E040F28710005D052869D2DFE800F0351C034E4F0031469FEDB40A2046FFF766
:40ACC00012FF3146B0EE080A2046FFF7BDFE31461FED8D0A2046FFF788FE2068324629464369204698474CE031469FEDA80A2046FFF7F9FE3146B0EE080A2046FFF7A4FE50
:40AD000031461FED990A2046FFF76FFE20683246294643692046984733E031469FED9B0A2046FFF7E0FE31469FED990A2046FFF78BFE31461FEDA60A2046FFF756FE2068D9
:40AD4000324629464369204698471AE000BF31469FED900A2046FFF7C6FE3146B3EE0E0A2046FFF771FE31461FEDB30A2046FFF73CFE20683246294643692046984700E074
:40AD800000BF00BF844B00224FF6FF71204651F165FF00BF00BF70BD2DE9F0412DED028B0446B0EE408A0E46154600279FED7B0AB4EEC08AF1EE10FA04DD02279FED770A45
:40ADC000B0EE408AB5EEC08AF1EE10FA04D203271FEDCD0AB0EE408A36B1012E26D0022E46D0032E7DD165E0D4F8080170B194F81B0158B1D4F80801EEF768F830B929469B
:40AE0000B0EE480AD4F8080126F165FC94ED590AB4EE480AF1EE10FA07D084ED598A2B463A467F21204651F119FF69E0D4F8080170B194F81B0158B1D4F80801EEF746F8B0
:40AE400030B92946B0EE480AD4F8080126F161FC94ED5B0AB4EE480AF1EE10FA07D084ED5B8A2B463A468021204651F1F7FE47E0D4F8080170B194F81B0158B1D4F808017F
:40AE8000EEF724F830B92946B0EE480AD4F8080126F15DFC94ED5D0AB4EE480AF1EE10FA07D084ED5D8A2B463A468121204651F1D5FE25E0D4F8080170B194F81B0158B156
:40AEC000D4F80801EEF702F830B92946B0EE480AD4F8080126F159FC94ED5F0AB4EE480A00E00BE0F1EE10FA07D084ED5F8A2B463A468221204651F1B1FE01E0072700BF99
:40AF000000BF3846BDEC028BBDE8F08170B52DED028B0446B0EE408A0D4607269FED1F0AB4EEC08AF1EE10FA05DD02269FED1B0AB0EE408A0BE0B5EEC08AF1EE10FA05D245
:40AF400003269FED170AB0EE408A00E0002694ED570AB4EE480AF1EE10FA07D084ED578A2B4632468A21204651F178FE94F81501012809D1D4F8F00030B12946B0EE480A52
:40AF8000D4F8F00025F13CFA30460BE00000C84200000C420000AA42B518170800007A4400000000BDEC028B70BD70B504460D461646002D74D104F5C2704155801C405D4D
:40AFC00005286ED2DFE800F06E3703A2A300206831469FEDFC0AD0F8882020469047206832460021B2EE0E0AD0F89030204698472068324601219FEDF30AD0F890302046C3
:40B0000098472068324602211FED1B0AD0F8903020469847206832460321B1EE0A0AD0F8903020469847206832460021D0F8B83020469847A0E0206831469FEDE20AD0F897
:40B04000882020469047206832460021B2EE0E0AD0F89030204698472068324601219FEDD90AD0F89030204698472068324602211FED350AD0F890302046984720683246AC
:40B080000321B1EE0A0AD0F8903020469847206832464FF4C871D0F8B830204698476BE073E068E0206831469FEDC60AD0F88820204690472068324600219FEDC20AD0F84C
:40B0C000903020469847206832460121B3EE040AD0F89030204698472068324602219FEDB90AD0F8903020469847206832460321B1EE040AD0F890302046984720683246D0
:40B100000021D0F8B8302046984735E000BF206831469FEDAC0AD0F88820204690472068324600219FEDA70AD0F8903020469847206832460121B2EE040AD0F8903020464E
:40B1400098472068324602211FED6B0AD0F89030204698472068324603219FED9B0AD0F8903020469847206832460021D0F8B8302046984700E000BF00BF944B00224FF6A3
:40B18000FF71204651F16AFD2EE0012D2CD1002104F5C270415531469FED8A0A2046FFF7B5FE32460021B3EE040A2046FFF7F4FD32460121B1EE040A2046FFF7EDFD3246B5
:40B1C00002211FED890A2046FFF7E6FD324603219FED7F0A2046FFF7DFFD7C4B00224FF6FF71204651F13AFD70BD10B50346002059B993F81441002C07DDD3F8EC4024B1BF
:40B20000D3F8EC40146001200CE001290AD193F81541002C06DDD3F8F0401CB1D3F8F0401460012010BD014691F8140191F815211044C0B2704770B504460D460026D4F8A7
:40B24000EC0038B1D4F8EC0024F1D4FFA84201D1701CC6B2D4F8EC0038B1D4F8EC0024F1C9FFA84201D1701CC6B2304670BD30B5044600206AB1012A02D0032A27D111E083
:40B2800094F81651012D03D1D4F8F4501D6001201EE094F81951012D03D1D4F800511D60012015E041B994F81751012D04DBD4F8FC501D60012009E0012907D194F81851B4
:40B2C000012D03DBD4F8F8501D60012000E000BF00BF30BD30B50446002000251D602AB919B9D4F8F4501D60012000E000BF00BF30BD10B50246002071B1012902D003292F
:40B300000DD102E092F816010AE092F8173192F818412344D8B203E092F8190100E000BF00BF10BD2DE9F84304460F4690461D46089E4FF00009B8F1000F1AD0B8F1010FF8
:40B3400003D0B8F1030F5AD127E094F8160101280ED16946D4F8F40030F1E4FB40B10098EDF735FEA84203D1009830604FF0010946E094F8190101280ED16946D4F80001D4
:40B3800030F1D0FB40B10098EDF721FEA84203D1009830604FF0010932E0DFB994F81701012817DB6946D4F8FC0030F1BBFB88B10098EDF70CFEA8420CD1009830604FF042
:40B3C00001091BE000004842CDCC4C3EB51817080AD7233E012F11D194F8180101280DDB6946D4F8F80030F19DFB38B10098EDF7EEFDA84202D100983060B94600E000BFA6
:40B4000000BF4846BDE8F8832DE9F84304460D4617461E464FF0000817B1012F3ED113E08DB994F8160101280DD16946D4F8F40030F178FB38B10098EDF7C9FD18B9009828
:40B4400030604FF001082AE09DB994F8170101280FDB6946D4F8FC0030F164FB48B10098EDF7B5FD012804D1009830604FF0010813E0012D11D194F8180102280DDB6946E8
:40B48000D4F8F80030F14EFB38B10098EDF79FFD012802D100983060A84600E000BF00BF4046BDE8F88330B50446002022B1012A03D0032A16D10AE015E039B994F81A514B
:40B4C000012D03D1D4F804511D6001200BE0012907D194F81B51012D03D1D4F808511D60012000E000BF00BF30BD014691F81A0191F81B211044C0B270470246002021B12F
:40B50000012903D0032907D103E006E092F81A0103E092F81B0100E000BF00BF70472DE9F04104460D461646002740F28710005DA84208D040F28710055533463A468521ED
:40B54000204651F18BFB3846BDE8F0812DE9F04104460E4615460027002D7DD0002E42D194F8140101283EDAC4F8EC5023460022F649D4F8EC0051F1FCFA94F81401401C56
:40B5800084F814010127D4ED620AB0EE600A2068EF49D0F8A02020469047D4ED640AB0EE600A2068EA49D0F8A8202046904794F886112068E64AD0F8983020469847D4EDE8
:40B5C000560AB0EE600A2068E149D0F8882020469047D4ED660AB0EE600A2068DC49D0F8B02020469047012E3BD194F81501012837DAC4F8F05023460122D449D4F8F00051
:40B6000051F1B7FA94F81501401C84F815010127D4ED630AB0EE600ACD492046FFF714FAD4ED650AB0EE600AC9492046FFF75BFA40F28710015DC64A2046FFF770FFD4EDEB
:40B64000570AB0EE600AC2492046FFF75FFCD4ED670AB0EE600A00E017E0BD492046FFF7C4F9D4F880112068B94AD0F8B830204698473146284624F1D2FD204626F1F2FE5C
:40B6800080464146284624F1BDFD012F05D1B04B00225321204651F1E1FA3846BDE8F0812DE9F0472DED028B04460E4615464FF00009002D5ED0284630F149FA60B30128B4
:40B6C00002D0032854D136E02EBB94F81601012821DA94F81601401C84F81601C4F8F450002712E0D4F8F40070B1D4F8F4802068816E20468847B0EE408AD8F800009449D5
:40B7000082694046904700BF7F1C94F81601B842E8D84FF001092CE066B994F81901012808DAC4F8005194F81901401C84F819014FF001091DE066B994F81701012808DA2C
:40B7400044F8FC5FE07E401CE076FC3C4FF001090DE0012E0BD194F81801012807DAC4F8F85094F81801401C84F81801B14600E000BF00BF4846BDEC028BBDE8F087F8B57E
:40B7800004460E461546002700200090002D7DD069462846EDF79DFB0028F8D0009830F1D6F920B1012803D003287AD13AE079E0BEBB94F81A01012833DAC4F8045194F885
:40B7C0001A01401C84F81A010127D4ED580AB0EE600A20685E4A0021D0F8903020469847D4ED5A0AB0EE600A2068594A0121D0F8903020469847D4ED5C0AB0EE600A2068CC
:40B80000534A0221D0F8903020469847D4ED5E0AB0EE600A20684E4A0321D0F89030204698473FE0012E01D1012000E0002094F81B11012901DA012100E00021084038B3E5
:40B84000C4F8085194F81B01401C84F81B010127D4ED590AB0EE600A3D4A00212046FFF79BFAD4ED5B0AB0EE600A394A01212046FFF792FAD4ED5D0AB0EE600A344A02219E
:40B880002046FFF789FAD4ED5F0A02E00BE008E006E0B0EE600A2E4A03212046FFF77CFA00E000BF00BF6DB12846EDF70FFB48B9D4ED550AB0EE600A20682549D0F880200F
:40B8C000204690473846F8BD0246002092F81C31012B07DAC2F80C1192F81C315B1C82F81C31012070470246002092F81C31012B03D1D2F80C310B6001207047014691F86F
:40B900001C01704770B504460D46002694F81D0101280EDA04F588742560607B401C607301262068A4F588740268B7EE000A91688847304670BD0246002092F81D31012BD8
:40B9400003D1D2F810310B600120704753311408B5181708014691F81D01704770B504460D4694F8C801A8420DD084F8C851D4F80C0140B1D4F80C01026800EE105AB8EEF6
:40B98000400A9168884770BD70B504460D4694F8150140B1D4F8F00028B100222946D4F8F00024F14CFD70BD70B504460D4694F8140140B1D4F8EC0028B100222946D4F844
:40B9C000EC0024F13CFD70BD70B52DED028B04460D46D4F8EC0098B15DB1D4F8EC0024F15FFCB0EE408A0021D4F8EC0024F15EFC06E000219FEDF90AD4F8EC0024F156FCDB
:40BA0000BDEC028B70BD2DE9F04104460D4617460126D4F80801B8B1B5B106212046FFF7B3FFFC34E0680268D16A8847804654F8FC0930F174F880450BD2E94B07220621AC
:40BA4000204651F10BF904E0002600212046FFF79BFF3046BDE8F0812DE9F04104460D4617460126D4F80401B8B1B5B106212046FFF79AFFF43420690268D16A884780465E
:40BA800054F8F40930F14BF880450BD2D44B07220521204651F1E2F804E0002600212046FFF782FF3046BDE8F08170B52DED028B04460D4694F81501B0B1D4F8F00098B142
:40BAC0005DB1D4F8F00024F1EBFBB0EE408A0021D4F8F00024F1EAFB06E000219FEDBF0AD4F8F00024F1E2FBBDEC028B70BD2DE9F04104460E461546002794F8150158B1C3
:40BB0000D4F8F00040B1012D06D100223146D4F8F00024F1B2FB01273846BDE8F0812DE9F04104460E461546002794F8140158B1D4F8EC0040B1012D06D100223146D4F85C
:40BB4000EC0024F19AFB01273846BDE8F08170B52DED028B0446B0EE408A0D460726D4F8080160B10026D4ED6F0AF8EE600AB0EE600AD4F8080101684A69002190472B467D
:40BB800032468321204651F169F8BDEC028B70BD2DE9F04104460E469046354694F81701002809DDD4F8FC0030B1D4F8FC002FF1A4FF08B1012000E0002007460FB90025CD
:40BBC00041E0D4F8FC002FF15AFFB0B1D4F8FC002FF16EFFF0EE400A00EE105AB8EE400AF4EEC00AF1EE10FA07DDD4F8FC002FF15FFFBCEEC00A10EE105AD4F8C000A842AC
:40BC000001D9D4F8C050D4F8FC002FF1FDFEB0B1D4F8FC002FF111FFF0EE400A00EE105AB8EE400AF4EEC00AF1EE10FA07D2D4F8FC002FF102FFBCEEC00A10EE105A6948BE
:40BC4000854200D905462846BDE8F0812DE9F0412DED028B04460F461646614A2046D4F8C010FFF795FF0546002F7CD0204626F198FC90B1A069F3F723F98046D3F09DFCEC
:40BC800041EC180B9FED580B53EC102B58F1F8FA03D3A069F3F714F938B9002084F8C90184F8CA01C4F8BC510FE194F8DC00C8BB94F8C901012817D1D4F8F00024F1F0FA56
:40BCC000B0EE408AD4F8F00024F160FBB4EE408AF1EE10FA02D194F8C90008B9012000E0002084F8C9010CE0D4F8EC0024F1DEFB20B194F8CA0008B1012000E0002084F8FC
:40BD0000C90194F8C90184F8CA0194F8C90150B1D4F8F8000268516A8847BCEEC00A84ED6F0AD2E004E0D4F8C000C4F8BC01CCE0002084F8C901D4F8F00000287DD0D4F885
:40BD4000EC00002879D094F8CD01E8B3D4F8F00024F11CFBB0EE408AD4F8F00024F1A0FAB4EEC08A00E0A9E0F1EE10FA0ADB002084F8CA01C4F8BC511D4800688047C4F813
:40BD80002801A2E094F8CA01012825D14FF47A71D4F82801CAF05AFDA8B1154800688047C4F82801D4F8BC1194ED6F0AB8EE400ADFED100A20EE200ABCEEC00A10EE100A37
:40BDC000081AC4F8BC0100E01BE0D4F8BC01A84212D2002084F8CA0177E0000000000000B5181708F473E7000000000000F06B4018A01008CDCCCC3D002E66D0C4F8BC5144
:40BE000063E016B1C4F8BC515FE0D4F8EC0024F14DFB50B394F8CA0120B9FD4800688047C4F8280142F21071D4F82801CAF00EFDB8B1F7480068804700E039E0C4F828012B
:40BE4000D4F8BC1194ED6F0AB8EE400A5FED170A20EE200ABCEEC00A10EE100A0844C4F8BC01012084F8CA012FE0D4F8EC0024F136FB10B342F21071D4F82801CAF0E6FCCB
:40BE8000D8B1E34800688047C4F82801D4F8BC1194ED6F0AB8EE400A5FED2A0A20EE200ABCEEC00A10EE100A081AC4F8BC010CE0C4F8BC51002084F8CA0106E0C4F8BC518D
:40BEC000002084F8C90184F8CA01D24A2046D4F8BC11FFF75DFEC4F8BC01BDEC028BBDE8F0812DE9F04104460D46164694F81701002814DDD4F8FC0088B1D4F8FC002FF17E
:40BF00009CFDDFEDC50AB4EEE00AF1EE10FA06DD00219FEDC10AD4F8FC002FF191FD94F81801002814DDD4F8F80088B1D4F8F8002FF183FDDFEDB80AB4EEE00AF1EE10FA65
:40BF400006DD00219FEDB40AD4F8F8002FF178FD2DB3D4F8FC002FF1D0FD00B3D4F8FC002FF152FDD8B1D4F8FC002FF166FDB5EEC00AF1EE10FA12DDD4F8FC002FF17BFD22
:40BF800068B1D4F8FC002FF139FD07464FF47A71CAF05CFC18B1012084F8CE0102E0002084F8CE01BDE8F08180F8CC1170472DE9F04F2DED028B81B004460D4616461F468E
:40BFC000DDE90C9B0020009094F81901002809DDD4F8000130B1D4F800012FF18EFD08B1012000E0002082462068C16C20468847F0B3D4ED131AF8EE611AB0EE611AD4EDF2
:40C00000101AF8EE611AF0EE610A94F8390001EE900AF8EE611AB0EE610A26F167FF28B1216CE06C884201D9012000E0002080462068784A4146D0F8F43020469847D4EDF7
:40C04000131AF8EE611AB0EE611AD4ED101AF8EE611AF0EE610A94F8390001EE900AF8EE611AB0EE610A26F141FF38B1216C00E00EE0E06C884201D2012000E00020804661
:40C080002068644A4146D0F8F030204698470DE02068604A0021D0F8F4302046984720685C4A0021D0F8F030204698471DB3BAF1000F20D0D4F800012FF1A6FCD8B1D4F84B
:40C0C00000012FF1BAFCB5EEC00AF1EE10FA12DDD4F800012FF1CFFC68B1D4F800012FF18DFC80464FF47A71CAF0B0FB18B1012084F8CD0102E0002084F8CD016B4603222E
:40C100001146A069F0F796F930B1009809F03EF80B2801D1012000E000208046E5B3DEB3D4F8F00024F1BCF8B0EE408AD4F8F00024F1F5F8B4EEC08AF1EE10FA2DDB5FB3D2
:40C14000B9F1000F29D0F83460680268516A8847B0EE408A54F8F8090268516A8847DFED2F0A30EE200AB4EEC08AF1EE10FA14D8B8F1000F0ED0B8F1010F0ED10098006840
:40C18000416A00988847F8EE000AB4EEE00AF1EE10FA02D2012001E0FFE7002084F8CF0194F8CF0120B91A4800688047C4F8D00194F8CF0158B143F69821D4F8D001CAF0DF
:40C1C00045FB20B100221146204626F1EEF9204626F12EFE00EE100AB8EE408A204626F126FD00EE100AF8EE400A88EE200ADFED0C0A60EE200A94ED0F0AB8EE400AF4EEF2
:40C20000C00AF1EE10FA0DD8012084F8D8000CE018A01008B5181708F473674BC0A9064800007A44002084F8D80001B0BDEC028BBDE8F08F2DE9F0412DED028B82B00446D2
:40C240000E46174698462068816E20468847B0EE408A0025D4F8B80000287CD0002EFCD000200190D4F8F40070B101A9D4F8F4002FF158FC40B101980068016901988847D0
:40C28000054601982FF1BFF8D4F8F4002FF1B7FCD8B1204626F148FA00EE100AB8EE400A1FED211AC0EE010A00EE107AB8EE400A20EE800ABCEEC00AB8EE400AD4ED750A4C
:40C2C00030EE200A84ED750A09E0D4ED750A00EE105AB8EE400A48EE000AC4ED750A94ED750A5FED310AB4EEE00AF1EE10FA55DB00BF94ED750A5FED360A80EE201ABCEE5C
:40C30000C10A10EE105AD4F8A400A84205D9D4F8A400401BC4F8A40002E00020C4F8A40054F8A80F2844206054F8A809FE49884204D3D4F8A800401AC4F8A80054F8AC0FF8
:40C340002844206054F8AC09F749884206D3D4F8AC00401A00E022E0C4F8AC0054F89C0F2844206060692844606160699C3CEE49884204D3D4F8B000401AC4F8B000D4ED7C
:40C38000750A4FF47A7105FB01F000EE100AB8EE400A30EEC00A84ED750A00BF0FE076B100200190D4F8F40040B101A9D4F8F4002FF1B8FB10B101982FF125F800BF02B093
:40C3C000BDEC028BBDE8F08170B504460D46164620680121C26A20469047A84208DDC4F8406105F12201D14B0022204650F136FC70BD2DE9F0412DED0E8B04460D46164644
:40C400009FEDCB0AB0EE408A9FEDC90AF0EE408A2068816E20468847B0EE408A94F8160110B1D4F8F40048B99FEDC10AF0EE408A002211462046FFF7C7FF5BE0D4F8F4005E
:40C440002FF1DDFBA0B3012802D002283ED111E0002D0AD9D4F8F4002FF133FC00EE100AB8EE400AF0EE408A03E09FEDB10AF0EE408A30E0B5EEC08AF1EE10FA19DD94ED5E
:40C48000100AF8EE400A00EE106AB8EE401A00EE105AB8EE400A21EE000A20EE800ADFEDA50A68EE200A80EE201AF0EE418A04E004E09FED9F0AF0EE408A0CE0D4F8F40034
:40C4C0000268116A8847F0EE408A04E09FED980AF0EE408A00BF00BFD4F8F4000268116A8847BCEEC00A10EE107A3A4600212046FFF76AFF28EE880ABCEEC00A84ED120A29
:40C50000002E1ED9002D1CD994ED120AB8EE400ADFED890A20EE200ADFED880A60EE200A00EE106AB8EE401A00EE105AB8EE400A21EE000A80EE801ABCEEC10A84ED130AE6
:40C5400001E00020E0642846D3F037F841EC1B0B3046D3F032F841EC1D0B206CD3F02DF841EC1E0B53EC1D2BD3F03AF841EC1C0B53EC1B2BD3F034F841EC1A0B9FED700BA4
:40C5800053EC102BD2F028FE41EC190BD2F0E8FFC4F8C401BDEC0E8BBDE8F0812DE9F04104460E461746DEB90020E064A064002511E0D4F8F40068B1D4F8F4000268116A71
:40C5C0008847BCEEC00A10EE108AE9B242462046FFF7FAFE6D1C94F81601A842E9D806E02046D4F85021D4F8B810FFF702FF3B4600225521204650F131FB3B4600225621F8
:40C60000204650F12BFBBDE8F0812DE9F04F2DED028B87B0044600200690012501260590824680464FF0010983460027E06ECAF0FDF80490444800688047E066D4F8B80025
:40C64000C4F8BC00204625F10DFF0290A16901F13000029905F0ADFEC4F8B800A069F2F72FFCC4F850010020059094F8160100280FDDD4F8F40010B90320069009E0D4F8C0
:40C68000F4002FF13AFA10B90120069001E00120059094F81801002809DDD4F8F80030B1D4F8F8002FF129FA08B1012000E00020824694F81701002809DDD4F8FC0030B1BF
:40C6C000D4F8FC002FF119FA08B1012000E00020804694F81501002804DDD4F8F00008B1012000E00020834694F88401012805D120680E4A002143692046984740F28510CC
:40C70000005D012805D12068084A0121436920469847204626F1DDFC0598F0B12068816E2046884712E00000FA592E87B51817080000000020BCBE4C0000C84200247449B9
:40C740000000000084D7974118A01008B5EEC00AF1EE10FA01DD012000E000200746F94A39462046FFF71AFFF649204626F166FDF449204626F18EFD204626F101FEF14BC1
:40C7800039462046049AFFF755FDD4F8B8202046049926F113FC4FF4FA71D4F83401CAF055F820B3D4F8A4102068E64AD0F8EC3020469847E34A2046D4F8A81026F1FEFAD1
:40C7C000E04A2046D4F8AC1026F1B2FADD4A2046D4F8B01026F111FBDA4A2046D4F89C1026F1D3FAD84800688047C4F83401204625F12DFE072801D1012000E000200290A1
:40C80000D04853465A46CDE9008020460299FFF7CEFB2068D0F894102046884750B9CB48806A00F00070B0F1007F03D103212046FFF7BAFB94F8D30028B1A069F2F7C6FB0E
:40C84000012800D100E0002084F84C0194F8D30030B1A069F2F7BAFB022801D1012000E0002084F84D01204626F13EF80546206C08B9012000E00020814617B1B9F1000F73
:40C8800001D0012000E000200646AE4A41462046FFF727FBBBF1000F21D0204625F1D7FD07281CD1BAF1000F19D0D4F8F8002FF1E6F878B154F8F80F2FF1FAF8B0EE408ACA
:40C8C00054F8F8090268516A8847B4EEC08AF1EE10FA04D8B8F1000F01D0012000E0002003902A4620460399FFF7B0F9D4F8040158B1D4ED710AF8EE600AB0EE600AD4F8BE
:40C90000040101684A6900219047D4ED6F0AF8EE600AB0EE600A00212046FFF718F994F81A212046D4F80411FFF7F9F894F81B212046D4F80811FFF7DAF894F8DB0013284C
:40C9400072D2DFE810F01300260142024302CA0082001603C7026703DE0350049D04E704230571007100B1057100B10394F81F0150B10020C4F8200100212046FFF714F878
:40C9800009212046FFF700F8204625F10AFE10B36F4800688047012803D1122084F8DB001DE094F8CB00012803D1092084F8DB0015E0A16901F5D270EEF7D7F9022803D18B
:40C9C000092084F8DB000AE094F8DC00012803D10C2084F8DB0002E0052084F8DB0094F8DB0094F81E1188422ED1594800688047012803D094F8CC01032808D109212046E3
:40CA0000FEF7D2FF09212046FEF7BEFF1CE094F8CC01012809D100212046FEF7C5FF00212046FEF7B1FF0FE0F6E394F8CC0102280AD194F8860138B903212046FEF7B4FFCE
:40CA400000212046FEF7A0FF43E294F81F0150B10020C4F8200100212046FEF7A5FF00212046FEF791FF204625F19BFD28B3384800688047012803D1122084F8DB001FE07D
:40CA800094F8DC00012803D10C2084F8DB0017E094F8CA0018B1012084F8DB0010E094F84C0118B1062084F8DB0009E094F84D0130B1072084F8DB0002E0002084F8DB0076
:40CAC00094F8CC01032807D109212046FEF76CFF09212046FEF758FFB6E794F81F0150B10020C4F8200100212046FEF75DFF00212046FEF749FF204625F153FD18B900206E
:40CB000084F8DB002AE0124800688047012803D1122084F8DB0021E094F8DC00012803D10C2084F8DB0019E094F84C0118B1062084F8DB0012E094F84D0158B1072084F80C
:40CB4000DB000BE0B518170818A01008C0230010B000002015B9012084F8DB0094F8CC01032807D109212046FEF71EFF09212046FEF70AFF94F8DB0094F81E11884207D0DB
:40CB800094F8DB00012803D000212046FEF78DFF5AE794F81F0190B10020C4F82001039850B1D4F8F00023F17EFBB5EEC00AF1EE10FA01D0012000E0002084F8CB01204604
:40CBC00025F1EFFC18B9002084F8DB003CE0F84800688047012803D1122084F8DB0033E094F8DC00012803D10C2084F8DB002BE07DB1D4F8EC0023F1FDFA012805D0D4F81A
:40CC0000EC0023F1F7FA042803D1042084F8DB001AE094F84C0118B1062084F8DB0013E094F84D0118B1072084F8DB000CE094F8CE0118B1032084F8DB0005E094F8CD0192
:40CC400010B1022084F8DB0094F8DB0094F81E11884271D194F81F0120B3D4F8EC0023F1C9FA04281ED1D4F8EC0023F119FBB5EEC00AF1EE10FA15D894F8CD0090B9D4F892
:40CC8000EC0023F12EFBB5EEC00AF1EE10FA04DD08212046FEF788FE96E007212046FEF783FE91E094F8C900B8B1002084F8CB0194F8C90140B102212046FEF765FE0321AD
:40CCC0002046FEF771FE7FE000212046FEF75CFE02212046FEF768FE76E094F8CB0160B3D4F8EC0023F1E2FBE8B1012084F8C90107212046FEF748FE03212046FEF754FE4D
:40CD0000D4F8F00023F1CFFAB0EE408AD4F8F00023F1C6FAB4EE408AF1EE10FA54D1002084F8CB0150E004212046FEF72DFE03212046FEF739FE47E030E0FFE794F8CA007C
:40CD4000B8B1002084F8CB0194F8C90140B101212046FEF719FE03212046FEF725FE33E000212046FEF710FE01212046FEF71CFE2AE094F8C90140B105212046FEF704FE5D
:40CD800003212046FEF710FE1EE000212046FEF7FBFD05212046FEF707FE15E094F8DB00042801D1012000E0002001462046FEF77CFE2068D0F8941020468847042803D12E
:40CDC00001212046FEF700FED9E300BF94F81F0110B10020C4F82001204625F1E2FB18B9002084F8DB0037E0714800688047012803D1122084F8DB002EE094F8DC0001280E
:40CE000003D10D2084F8DB0026E01DB1042084F8DB0021E094F84C0118B1062084F8DB001AE094F84D0118B1072084F8DB0013E094F8CE0118B1032084F8DB000CE094F807
:40CE4000CD0118B1022084F8DB0005E094F8CA0010B9012084F8DB0094F81E0194F8DB1088422BD194F8CE0110B994F8CD0180B194F8C90140B10A212046FEF785FD03211C
:40CE80002046FEF791FD24E000212046FEF77CFD1FE094F8C90140B105212046FEF774FD03212046FEF780FD13E000212046FEF76BFD05212046FEF777FD0AE02068D0F856
:40CEC000941020468847042803D100212046FEF77BFD54E394F81F0150B10020C4F8200100212046FEF760FD00212046FEF74CFD204625F156FB18B9002084F8DB001AE0D7
:40CF00002B4800688047012803D1122084F8DB0011E094F8DC00012807D194F84D0100B14EB10C2084F8DB0005E094F84D0110B9052084F8DB0094F8CC01032807D10921D8
:40CF40002046FEF731FD09212046FEF71DFD94F81E0194F8DB1088420AD02068D0F8941020468847042803D100212046FEF72CFD05E394F81F0150B10020C4F82001002142
:40CF80002046FEF711FD00212046FEF7FDFC204625F107FB18B9002084F8DB001CE0044800688047012805D1122084F8DB0013E0B000002094F8DC00012807D194F84C01C9
:40CFC00000B14EB10C2084F8DB0005E094F84C0110B9052084F8DB0094F8CC01032807D109212046FEF7E0FC09212046FEF7CCFC94F81E0194F8DB1088420AD02068D0F8DB
:40D00000941020468847042803D100212046FEF7DBFCB4E2204625F1C4FA18B9002084F8DB001BE0FE4800688047012803D1122084F8DB0012E094F8DC0001280BD135B171
:40D040002EB994F84C0110B994F84D0130B10C2084F8DB0002E0042084F8DB0094F8CC01032808D109212046FEF79EFC09212046FEF78AFC17E094F81E0194F8DB10884222
:40D0800011D100212046FEF78FFC94F8CA01012805D1E44A41462046FEF7B5FC03E000212046FEF771FC6AE294F81F0168B10020C4F8200100212046FEF776FC0921204618
:40D0C000FEF762FC002084F8C901204625F169FA18B9002084F8DB0006E0D1480068804710B9092084F8DB0094F8CC01032807D109212046FEF758FC09212046FEF744FCDF
:40D100003DE294F81F0180B10020C4F8200100212046FEF749FC09212046FEF735FC002084F8C90184F8CC0011E0A16901F5D270EDF71BFE08B9012000E0002094F8CC1057
:40D14000084308B1012000E0002084F8CC00204625F127FA18B9002084F8DB0025E0A16901F5D270EDF701FE02281ED0AC4800688047012803D1122084F8DB0015E0A16973
:40D1800001F5D270EDF7F1FD01280ED194F8CC0001280AD194F8DC00012803D10C2084F8DB0002E0052084F8DB0094F8CC01032807D109212046FEF7F7FB09212046FEF763
:40D1C000E3FB94F8DB0094F81E1188420AD02068D0F8941020468847042803D100212046FEF7F2FBCBE194F81F0168B10020C4F8200109212046FEF7D7FB09212046FEF7AF
:40D20000C3FB002084F8C901204625F1CAF920B9002084F8DB0015E09EE1814800688047012803D1122084F8DB000BE094F8DC00012804D137B10C2084F8DB0002E001208A
:40D2400084F8DB0094F8CC01032807D109212046FEF7AAFB09212046FEF796FB94F8DB0094F81E1188420AD02068D0F8941020468847042803D100212046FEF7A5FB7EE151
:40D2800094F81F0110B10020C4F82001204625F188F918B9002084F8DB0016E0604800688047012803D1122084F8DB000DE094F8DC00012806D1B9F1000F06D10C2084F8DF
:40D2C000DB0002E0012084F8DB0094F8CC01032807D109212046FEF767FB09212046FEF753FB94F8DB0094F81E11884211D100212046FEF759FB94F8CA01012805D1494A5C
:40D3000041462046FEF77FFB03E000212046FEF73BFB34E1204625F144F918B9002084F8DB0032E03E4800688047012803D1122084F8DB0029E094F8DC00012822D11FB934
:40D340000A2084F8DB0020E0B9F1000F03D00B2084F8DB0019E094F84C0118B1062084F8DB0012E094F84D0118B1072084F8DB000BE01DB1082084F8DB0006E0102084F829
:40D38000DB0002E0052084F8DB00F8E094F81F0120B10020C4F8200184F8CB01204625F100F918B9002084F8DB001FE01C4800688047012803D1122084F8DB0016E094F843
:40D3C000DC0001280FD194F84C0118B994F84D0100B91EB10C2084F8DB0007E035B1082084F8DB0002E0012084F8DB0094F8DB0094F81E11884246D194F81F0138B3D4F8AD
:40D40000EC0022F1F7FE042821D1D4F8EC0022F147FFB5EEC00AF1EE10FA18D804E00000B0000020B5181708D4F8EC0022F159FFB5EEC00AF1EE10FA04DD08212046FEF705
:40D44000B3FA30E007212046FEF7AEFA2BE0D4F8B80020B905212046FEF7A6FA04E0FD4A39462046FEF7F8FA94F8CA01012805D1F84A41462046FEF7C6FA14E0002120468F
:40D48000FEF782FA0FE02068D0F8941020468847042803D101212046FEF796FAEE4800688047C4F820016AE094F81F0120B1EA4800688047C4F82401204625F172F818B9D4
:40D4C000002084F8DB0035E0E44800688047012803D1122084F8DB002CE094F8DC00012825D194F84C0120B994F84D0108B906B91DB10C2084F8DB001CE0D4F82C0190B199
:40D500006423D4F82C2102FB03F1D4F82401C9F09DF940B9D4F8200128B1D149D4F82001C9F094F930B10D2084F8DB0002E0012084F8DB0094F8DB0094F81E11884208D18A
:40D5400005212046FEF730FA05212046FEF71CFA01E00020A06612E000221146204625F124F809212046FEF71FFA09212046FEF70BFA0020C4F8200184F8DB0000BF00BF65
:40D58000002084F81F0194F8DB0094F81E11884215D0002084F8CB0084F8CC012068016D20468847012084F81F0194F8DB0084F81E01A84B07221A2120464FF14FFB94F871
:40D5C000DB00142818D2DFE800F00A1D1E1F0C0D0E0F101112131C2021142215160B00BF00BF00BF00BF00BF00BF00BF00BF00BF00BF00BF00BF00BF00212046FEF7AEF9F4
:40D6000011E010E000BF00BF00BF00BF00BFD4F8B800002801D9012000E0002001462046FEF79CF900BF00BF069807B0BDEC028BBDE8F08F014691F8C8017047DFED890A94
:40D64000B0EE600A092933D2DFE801F0050A0F14191E23282D00DFED840AB0EE600A28E0DFED820AB0EE600A23E0DFED810AB0EE600A1EE0DFED7F0AB0EE600A19E0DFED86
:40D680007E0AB0EE600A14E0DFED7C0AB0EE600A0FE0DFED7B0AB0EE600A0AE0DFED790AB0EE600A05E0DFED780AB0EE600A00E000BF00BF704790ED680A704702460020A5
:40D6C00009B9D2F840017047014691F83C0170472DE9F0472DED028B04460D46164600272068816D20468847A84223D084F83C5133463A46212120464FF1B0FAB84615E0BF
:40D70000D4F8F40070B1D4F8F4902068816E20468847B0EE408AD9F800004E4982694846904700BF08F1010000F0FF0894F816014045E5DC3846BDEC028BBDE8F08701463C
:40D74000D1F8380170472DE9F0472DED028B04460D46164600272068016E20468847A84223D0C4F8385133463A46202120464FF175FAB84615E0D4F8F40070B1D4F8F4901B
:40D780002068816E20468847B0EE408AD9F80000304982694846904700BF08F1010000F0FF0894F816014045E5DC3846BDEC028BBDE8F08700B503469FED2A0AB0EE401A9C
:40D7C000D3F8380168B193F83C111846FFF736FFD3ED4E0AF8EE600AC0EE201AB0EE611A03E09FED200AB0EE401AB0EE410A00BD0146D1F8300170472DE9F04104460D462F
:40D8000016460027D4F83001A84207D0C4F8305133463A46422120464FF120FA3846BDE8F0810146D1F82C0170472DE9F04104460D4616460027D4F82C01A84207D0C4F8E9
:40D840002C5133463A46432120464FF107FA3846BDE8F081B518170818A01008B0000020C0D4010000000000002474498096184B0F0B674AE966104C58BC8A4A00007A44FC
:40D880000F0BE74626FADD46E76C8A4A90ED550A704770B52DED028B0446B0EE408A0D4600269FEDFE0AB4EEC08AF1EE10FA04DD02269FEDFA0AB0EE408A94F81A0150B11B
:40D8C000D4F8040138B1D4F804010168CA692946B0EE480A904794F81B0150B1D4F8080138B1D4F808010168CA692946B0EE480A904794ED550AB4EE480AF1EE10FA07D029
:40D9000084ED558A2B463246482120464FF1A6F93046BDEC028B70BD90ED560A704770B52DED028B0446B0EE408A0D4607261FED2D0AB4EEC08AF1EE10FA05DD02261FED67
:40D94000310AB0EE408A0BE0B5EEC08AF1EE10FA05D203261FED3D0AB0EE408A00E0002694ED560AB4EE480AF1EE10FA07D084ED568A2B463246512120464FF16FF994F8A7
:40D980001401012809D1D4F8EC0030B12946B0EE480AD4F8EC0022F133FD3046BDEC028B70BD90ED570A70475FED520AB0EE600A31B1012909D002290CD0032914D10EE053
:40D9C000D0ED580AB0EE600A0EE0D0ED5A0AB0EE600A09E0D0ED5C0AB0EE600A04E0D0ED5E0AB0EE600A00BF00BF70472DE9F0412DED028B0446B0EE408A0E461546002719
:40DA00001FED620AB4EEC08AF1EE10FA04DD02271FED660AB0EE408AB5EEC08AF1EE10FA04D203271FED710AB0EE408A36B1012E26D0022E46D0032E7DD165E0D4F80401FF
:40DA400070B194F81A0158B1D4F80401EBF73EFA30B92946B0EE480AD4F8040123F13BFE94ED580AB4EE480AF1EE10FA07D084ED588A2B463A46442120464FF1EFF869E06E
:40DA8000D4F8040170B194F81A0158B1D4F80401EBF71CFA30B92946B0EE480AD4F8040123F137FE94ED5A0AB4EE480AF1EE10FA07D084ED5A8A2B463A46452120464FF1AE
:40DAC000CDF847E0D4F8040170B194F81A0158B1D4F80401EBF7FAF930B92946B0EE480AD4F8040123F133FE94ED5C0AB4EE480AF1EE10FA07D084ED5C8A2B463A4646214A
:40DB000020464FF1ABF825E0D4F8040170B194F81A0158B1D4F80401EBF7D8F930B92946B0EE480AD4F8040123F12FFE94ED5E0AB4EE480A00E00BE0F1EE10FA07D084ED3E
:40DB40005E8A2B463A46472120464FF187F801E0072700BF00BF3846BDEC028BBDE8F0815FEDC00AB0EE600A31B1012909D002290CD0032914D10EE0D0ED590AB0EE600AB7
:40DB80000EE0D0ED5B0AB0EE600A09E0D0ED5D0AB0EE600A04E0D0ED5F0AB0EE600A00BF00BF7047014691F8860170472DE9F04104460D461646002794F88601A84207D0A8
:40DBC00084F8865133463A464B2120464FF146F83846BDE8F081014640F28710405C704790ED620A70472DE9F0412DED028B0446B0EE408A0D46002694ED620AB4EE480AF8
:40DC0000F1EE10FA16D0264890ED000AB4EEC80AF1EE10FA02D884ED628A05E0204890ED000A84ED620A03262B4632464F2120464FF114F800270DE0D4F8EC0040B1D4ED29
:40DC4000620AB0EE600A2946D4F8EC0022F1A1FB781CC7B294F81401B842EDDC3046BDEC028BBDE8F08190ED640A70472DE9F0412DED028B0446B0EE408A0D46002694EDEB
:40DC8000640AB4EE480AF1EE10FA0DD084ED648A2B4632464E21204604E000000000C842004417084EF1DAFF00270BE0D4F8EC0030B12946B0EE480AD4F8EC0022F132FBB4
:40DCC000781CC7B294F81401B842EFDC3046BDEC028BBDE8F08190ED660A70472DE9F0412DED028B0446B0EE408A0D46002694ED660AB4EE480AF1EE10FA07D084ED668A2C
:40DD00002B463246502120464EF1A8FF00270BE0D4F8EC0030B12946B0EE480AD4F8EC0022F1E2FA781CC7B294F81401B842EFDC3046BDEC028BBDE8F08190ED630A7047B6
:40DD400090ED650A704790ED670A70470146D1F8800170472DE9F04104460D461646072794F88601012802D002281BD100BF002794F81401012808D1D4F8EC0028B13246EF
:40DD80002946D4F8EC00EAF7BEFFD4F88001A84207D0C4F8805133463A46522120464EF15DFF0AE0D4F88001A84205D033463A46522120464EF152FF00BF00BF3846BDE89D
:40DDC000F08130B50346002011B101290BD104E0012483F88441002005E0012540F28514E554002000BF00BF30BD0146D1F8C40170470146D1F8BC017047014691F8CF01E9
:40DE000070470146C86B70472DE9F04104460D4616460027E06BA84206D0E56333463A46722120464EF11AFF3846BDE8F0810146C86B70472DE9F04104460D4616460027CA
:40DE4000E06BA84206D0E56333463A46722120464EF104FF3846BDE8F08110B5044694F81601002809DDD4F8F40030B1D4F8F4002DF1C5FE08B1012010BD0020FCE70000DB
:40DE800010B50446204624F16EFA204624F1DFFA0F2803D1062084F8100102E0042084F81001132084F811012068FE4A0021036920469847002004F5A0742060FA48006811
:40DEC00080476060F84800688047E06000202061F5480068804760610020A06120626062A06284F83400012084F83600002084F8370084F83800A4F5A074204624F1A7FAE4
:40DF00000F2801D1E948206410BDF8B504460F4615461E462B46052239462046009624F177F90446E248DC3444F8DC0C00F5907044F8D00C103044F8CC0C00202061606148
:40DF4000A06120776077A07720626062A062E0622063DC3C2046FFF793FF23462A46D54920464EF106FE2046F8BD70B50446D048206000F59070E06010302061002513E03A
:40DF8000D4F8EC0050F8250068B1D4F8EC0050F8250040B1D4F8EC2052F8250052F825201268516888476D1C94F8F800A842E7D8002513E0D4F8F00050F8250068B1D4F859
:40DFC000F00050F8250040B1D4F8F02052F8250052F825201268516888476D1C94F8F900A842E7D8002513E0D4F8F40050F8250068B1D4F8F40050F8250040B1D4F8F420E4
:40E0000052F8250052F825201268516888476D1C94F8FA00A842E7D854F8EC0F53F17EFD606853F17BFDA06853F178FD206953F175FD606953F172FDA06953F16FFDE06920
:40E0400053F16CFD206AEC3C53F168FD204624F11BF90446204670BD70B504462046FFF784FF054653F15EFD70BD10B50446103C2046FFF7F1FF10BD10B504460C3C204696
:40E08000FFF7EAFF10BD10B50446103C2046FFF76CFF10BD10B504460C3C2046FFF765FF10BD70B50546012406E07E4B0022214628464EF1D3FD641C7D2CF6D37E2406E01D
:40E0C000784B0022214628464EF1C8FD641CE72CF6D370BD70B504460D461646002D7CD120683246036F20469847206832460021836F2046984794F8100105286ED2DFE861
:40E1000000F0512A037B7C0020683146B0EE080AD0F8802020469047206831469FED660AD0F8A8202046904720683146B0EE080AD0F8A02020469047206831469FED5F0AF6
:40E14000D0F8B0202046904720683246294643692046984779E020683146B0EE080AD0F8802020469047206831469FED530AD0F8A8202046904720683146B0EE080AD0F891
:40E18000A02020469047206831469FED4C0AD0F8B0202046904720683246294643692046984752E020683146B0EE080AD0F8802020469047206831469FED3F0AD0F8A82062
:40E1C00020469047206831469FED3D0AD0F8A020204690472068314601E03EE034E09FED370AD0F8B0202046904720683246294643692046984728E000BF20683146B0EED3
:40E20000000AD0F8802020469047206831469FED2A0AD0F8A8202046904720683146B7EE000AD0F8A02020469047206831469FED230AD0F8B0202046904720683246294634
:40E2400043692046984700E000BF00BF154B00224FF6FF7120464EF101FD70BD70B504460D461646002D7DD1002084F8770194F81001052877D2DFE800F0824A03B6B70095
:40E28000206831469FED0F0AD0F8882020469047206832460021B2EE0E0AD0F890302046984711E0C918170818A010089421010090A51008CD3114080000C842000000007F
:40E2C00000000C42000048422068324601211FED030AD0F89030204698472068324602211FED0A0AD0F8903020469847206832460321B2EE040AD0F8903020469847206807
:40E3000032460021D0F8B83020469847A1E0206831461FED140AD0F8882020469047206832460021B2EE0E0AD0F89030204698472068324601211FED1D0AD0F8903020460F
:40E3400098472068324602211FED240AD0F8903020469847206832460321B2EE040AD0F8903001E07DE073E020469847206832464FF4C871D0F8B8302046984769E0206822
:40E3800031461FED300AD0F88820204690472068324600211FED350AD0F8903020469847206832460121B3EE040AD0F89030204698472068324602211FED3E0AD0F890301D
:40E3C00020469847206832460321B1EE040AD0F8903020469847206832460021D0F8B8302046984735E000BF206831461FED4B0AD0F88820204690472068324600211FED16
:40E400004F0AD0F8903020469847206832460121B2EE040AD0F89030204698472068324602211FED5A0AD0F89030204698472068324603219FEDFA0AD0F890302046984738
